:020000040000FA
:04000000D1EF06F046
:08000800000EFA6EFB6A2734BA
:100010000E0BF926010C020C040C080C100C200C21
:10002000400C800C0A6E1E501A5C02E11D50195CD7
:10003000040ED8B0010ED8B4020E0A14D8A4010ED2
:100040001200086A216E226A00960850D8B4008611
:10005000050E076E270E1E6E100E0CD8030E1E6EB8
:10006000E80E08D81E6A640E05D81E6A0A0E02D869
:10007000215008D01D6E22501A6E2150196E32EC9C
:1000800002F01950196E074E0096085003E0075C05
:10009000D8B008D01950D8A4009600B603D0300FBD
:1000A0000AEF01F012000096085003E100860A0EE4
:1000B000086E2EC01CF02DC01BF02CC01AF02BC0F7
:1000C00019F0076A246A236A226A0A0E216ED2ECAA
:1000D00001F0072A0750085CD8A4F4D72150D8A40F
:1000E000009600A602D0082C04D02150300F0AEC54
:1000F00001F0082EDED7120005C019F006C01AF074
:10010000010E1D6E1E6A0F0EEA6E02C0E9FF0000AE
:100110002AD8D8A015D01D2EFAD7FF0E1E26D8B08B
:10012000F6D71926D8A01A26D8A01200640E1D6E84
:100130001E6AEDD70F0EEA6E02C0E9FF14D8FEE288
:1001400056D8276A080E1E6E53D80DD8D8B0273E51
:100150001D321E2EF9D72AAA276A2ABA1D9E48D810
:10016000D8801D501200120EE9260950EF1202C06D
:10017000E9FFEF142ABC0918FF0F1200256E0F0EBD
:10018000EA6EE26E0250E96E120FE16E800E0A1600
:10019000080E266ED890D8B00A3E12D82532262EE8
:1001A000FAD700002ABA0A300BD800D000D000D00D
:1001B000D88006D806501E6E055083EC01F0120060
:1001C0002AAE0BD0EF5009102AAC0918EF6EE75099
:1001D0000910D8A00918E76E0BD0EF500910D8A06D
:1001E00009182ABC0918EF6E091CE71601D00A8C01
:1001F0002A501F0B000F1A6E2950050FD8B01A2A6B
:100200000AAC90EF01F00A9C196E020E8DEC02F020
:1002100090EF01F001BABEEF00F001B202D001B0E0
:100220002DEF01F0008800A8009800BA03D0008AE2
:1002300033D827E2009444D8C58642D8C95000B4C8
:1002400007D000B804D0C588C5B8FED700B819D803
:10025000D8901D6E1DD0008800A8009800BC05D065
:10026000FE0B0A6E008CD89013D000BE06D0256E0F
:10027000008E14D8D8B005D0255014D802E200A8BA
:1002800007D0C584C5B4FED7009C009E009A009498
:100290002780D8A0279012000DD801D005D80A5089
:1002A00000BA0109C96E0AD094869488C580C5B089
:1002B000FED71200C582C5B2FED71200C7B4FED762
:1002C0001D68C5501F0B00D0D890D8B412001D2E49
:1002D000F8D7D8801200AA6AA96EA66AA680A8508C
:1002E000A94AAA2A1200AA6AA86EA66AA684550E6E
:1002F000A76EAA0EA76EA682A6B2FED7A694A94A9A
:10030000AA2A12001E6A1D6EFF0E1D261E2200D094
:10031000D8A01200030E1A6EE30E02D8F5D71A6A9F
:10032000F40F196E1A1EFE0ED8A003D01926D8B0ED
:10033000FDD7192600001A3EF9D7000019B000D0E9
:1003400019B000D012000009D8B41200276E19C0ED
:10035000E9FF1AC0EAFF1A6A196A27BE07D0EE50F1
:10036000196E27A21200EF501A6E120004EC00F072
:10037000EF14D8A4192A1200010F266E0A0E1D6E62
:100380001E6A70D8262EFDD721501200010F066E6E
:100390000A0E216E226A236A246A04D8062EF8D730
:1003A000215012001C502418800BF46E1CAE06D095
:1003B000D880000E19561A561B561C5624AE06D06D
:1003C000D880000E21562256235624561D6A1E6AD6
:1003D0001F6A206A316A326A336A346A24502310F1
:1003E0002210211023E0200EF36ED89019361A3611
:1003F0001B361C3631363236333634362150315CBA
:1004000022503258235033582450345809E3215095
:10041000315E2250325A2350335A2450345AD880F5
:100420001D361E361F362036F32EDFD7F4AE06D02B
:10043000D880000E1D561E561F5620561DC019F09E
:100440001EC01AF01FC01BF020C01CF031C021F0EC
:1004500032C022F033C023F034C024F012001A6AF4
:100460001E6A1D6E226A216A100EF36E1A3421363E
:1004700022361D50215C1E50225805E31D50215E7E
:100480001E50225AD88019361A36F32EEFD719503B
:100490001200200E256E316A326A336A346AD890AF
:1004A00019A00ED0215031262250D8B0223C32263D
:1004B0002350D8B0233C33262450D8B0243C3426D3
:1004C00034323332323231321C321B321A32193268
:1004D000252EE5D712001D6A1E6A04D01A32193281
:1004E0001D361E36FF0FFAE21EC01AF01D50196E9F
:1004F0001200196E1CBE02D819501200191E1A1EC5
:100500001B1E1C1E192AD8B01A2AD8B01B2AD8B014
:100510001C2A1200D8901A321932FF0FFBE2195030
:100520001200FC0EDBCFE6FFFD0EDBCFE6FFFE0E7A
:10053000DBCFE6FFFF0EDBCFE6FFDD52DD52DD5203
:10054000DD521200FE0EDBCFE6FFFF0EDBCFE6FF33
:10055000DD52DD521200010E00D0216E37C023F0B3
:10056000378C246A216602D012BE248E129E880E19
:100570001160378A14C019F013C01AF012C01BF0B2
:1005800011C01CF0830E186EF90E176E220E166E37
:100590007F0E156EDEEC05F0379C2EEC06F0378CE6
:1005A00014A004D0142A000E13221222070E1414D1
:1005B000226E030E226404D0800E241A040E225EE2
:1005C000116A8EEC06F01150206E6DE014C01DF023
:1005D00013C01EF012C01FF0186A0F0E176EC90E5E
:1005E000166E7E0E156EDEEC05F019C018F01AC0FE
:1005F00017F01BC016F01CC015F0DCEC04F014C0A2
:1006000019F013C01AF012C01BF011C01CF01DC06D
:1006100014F01EC013F01FC012F020C011F0186AB1
:10062000A20E176EDA0E166E6E0E156EDEEC05F06B
:1006300019C018F01AC017F01BC016F01CC015F036
:10064000DCEC04F014C019F013C01AF012C01BF057
:1006500011C01CF01DC014F01EC013F01FC012F01A
:1006600020C011F0200E186EA20E176E850E166EA9
:100670005C0E156EDEEC05F019C018F01AC017F00C
:100680001BC016F01CC015F0DCEC04F011501C6E01
:10069000156E12501B6E166E13501A6E176E145094
:1006A000196E186E0CD01C50116E156E1B50126E08
:1006B000166E1A50136E176E1950146E186EDEEC0B
:1006C00005F014C01DF013C01EF012C01FF011C0C1
:1006D00020F022302218010B211851E0CE0E186EA6
:1006E000F50E176E4C0E166E6F0E156EDEEC05F0E5
:1006F0001A0E186E060E176EB60E166E750E156E65
:10070000DCEC04F01DC018F01EC017F01FC016F07E
:1007100020C015F0DEEC05F0A50E186EAA0E176EBF
:100720002A0E166E7A0E156EDCEC04F01DC018F061
:100730001EC017F01FC016F020C015F0DEEC05F04B
:100740001DC018F01EC017F01FC016F020C015F015
:10075000DEEC05F01DC018F01EC017F01FC016F02B
:1007600020C015F015661506DAEC04F0379C186AFF
:10077000176A166A7F0E156EDCEC04F05AD0F90E7B
:10078000186E680E176E360E166E6C0E156EDEEC59
:1007900005F0C00E186E070E176ED00E166E720E94
:1007A000156EDCEC04F01DC018F01EC017F01FC061
:1007B00016F020C015F0DEEC05F0840E186E880EE1
:1007C000176E080E166E780E156EDCEC04F01DC068
:1007D00018F01EC017F01FC016F020C015F0DEEC98
:1007E00005F0AB0E186EAA0E176E166E7C0E156E07
:1007F000DCEC04F01DC018F01EC017F01FC016F08E
:1008000020C015F0DEEC05F019C018F01AC017F082
:100810001BC016F01CC015F0DEEC05F0379C19C0AB
:1008200018F01AC017F01BC016F01CC015F0DCEC55
:1008300004F0800E215202E022B2241A24BE121AC1
:1008400023BC378C1450120012BEB1D01152D8B450
:10085000AFD011C022F037C023F0378C7F0E116E5D
:10086000186A176A166A156EDAEC04F014C019F0EB
:1008700013C01AF012C01BF011C01CF0130E186E3A
:10088000CB0E176E030E166E840E156EDCEC04F0A4
:1008900019C018F01AC017F01BC016F01CC015F0D4
:1008A000DEEC05F0BC0E186E5A0E176E050E166EB5
:1008B000860E156EDCEC04F019C018F01AC017F0A3
:1008C0001BC016F01CC015F0DEEC05F0830E186E90
:1008D000300E176E720E166E850E156EDCEC04F07F
:1008E00014C01DF013C01EF012C01FF011C020F084
:1008F00019C014F01AC013F01BC012F01CC011F084
:100900008E0E186ED70E176E6B0E166E810E156E4C
:10091000DEEC05F0B50E186E290E176E4E0E166E33
:10092000840E156EDCEC04F019C018F01AC017F034
:100930001BC016F01CC015F0DEEC05F0800E186E22
:10094000300E176E720E166E840E156EDCEC04F00F
:100950001DC018F01EC017F01FC016F020C015F003
:1009600076EC05F019C018F01AC017F01BC016F08D
:100970001CC015F0DEEC05F0186A176A166A7F0EC7
:10098000156EDCEC04F022B00AD0F30E186E040EE3
:10099000176E350E166E7F0E156EDEEC05F07F0EAF
:1009A00022262230116E23BC03D0379C01D0378A17
:1009B00014501200800E161A1550115C366E19E292
:1009C000366C11C038F015C011F038C015F012C0E7
:1009D00038F016C012F038C016F013C038F017C047
:1009E00013F038C017F014C038F018C014F038C035
:1009F00018F01A0E366078D0155276E0356A12502B
:100A0000386E1618396E128E168E080E365E08E392
:100A100018C035F017C018F016C017F0166AF5D7D1
:100A2000362607E0D8901632173218323532362E75
:100A3000F9D739AE35D01850145E1750135A1650E6
:100A4000125A07E2D880000E145613561256800E22
:100A5000381A356C04E01406000E135A125A040EAC
:100A6000366E12660DD013C012F014C013F035C0EC
:100A700014F0356A080E115E2DE3362EF2D72AD017
:100A800012BE08D0D8903536143613361236112ED1
:100A9000F7D720D037AC26D035AE24D0356A11D068
:100AA00018501426175013221650122206E3123241
:100AB000133214323532114A0FD037AC13D035AE61
:100AC00011D0143E0FD0133E0DD0123E0BD0D88063
:100AD0001490EDD7116A02D037821168146A136A34
:100AE000800E126E38AE129E145012001250336EE9
:100AF0001618396E155053E0115254E0115E7F0EF6
:100B000003E2112603E24DD011264EE214C031F06B
:100B100013C032F0338E168E180E386E146A136AB4
:100B2000126A0BD01850315C1750325811E3326EF4
:100B3000336A1850315E0BD004E21650335CF2E099
:100B400007E31850315E1750325A1650335AD88086
:100B5000143613361236313632363336382EECD759
:100B600012BE07D011521DE039321106382A39362B
:100B7000E3D737AC1FD007E21850315E1750325A16
:100B80001650335A17E3143E15D0133E13D0123EBD
:100B900011D0123213321432113E0CD005D03786E8
:100BA00004D03784116A02D037821168146A136A3C
:100BB000800E126E39AE129E145012001250336E17
:100BC0001618396E1150D8A415503CE011267E0E2F
:100BD00003E3115E03E338D0115E33E314C031F058
:100BE00013C032F0338E168E146A136A126A180E0E
:100BF000386E33323232313206E318501426175031
:100C0000132216501222123213321432382EF1D718
:100C100012BE07D0143613361236115212E01106E6
:100C2000333437AC17D016E3143E14D0133E12D031
:100C3000123E10D0D880123213321432113E0AD034
:100C400003D03784116A02D037821168146A136A9C
:100C5000800E126E39AE129E1450120012C039F07E
:100C60007F0E115C386E3FE3128E116A316A1708ED
:100C7000386E0BE2080E382638E312C011F013C0AC
:100C800012F014C013F0146A0CD0080E385E08E39A
:100C900014C031F013C014F012C013F0126AF5D76B
:100CA0003826385208E0D8901132123213321432FA
:100CB0003132382EF8D711BE18D037AC0BD031AE48
:100CC00009D0143E07D0133E05D0123E03D0122A9D
:100CD00011BE0BD039AE10D0D880000E145613566A
:100CE0001256115609D0000E02D03782FF0E116E37
:100CF000126E136E146E119E14501200116E126A51
:100D0000136A146A11C035F014C011F035C014F024
:100D100013C035F012C013F035C012F0960E386EC5
:100D2000396A11AE07D0D880000E145613561256E9
:100D30001156398E115218E037AC0DD014AE0BD0CD
:100D4000133E09D0123E07D0113E05D0D880113293
:100D500012321332382A080E382613C014F012C08B
:100D600013F011C012F015D0126613D0080E385EC1
:100D7000135005E1080E385E145011E0146A126E2B
:100D800014C013F0146A05D0D890143613361236F6
:100D9000380612AEF9D738C011F039AE129E145091
:100DA0001200F86A400E376E006AAB6A280EC66EF3
:100DB000040EC86E800EC76E070EB46E0F0EC16EA5
:100DC0002FEE20F0860ED56E2E0E926E070E936ECD
:100DD000870E946E956A966A7E0E976E200E986EB8
:100DE0007B6B7A6B896B010E8B6F900E8A6F0A0E8C
:100DF000816F836B846B8095856B0501BD6B0001F2
:100E00008091A66BA56BA86BA76B809B580E070102
:100E10009E6F010E0001A96F010EAA6FBB6B0A0E37
:100E2000826F80998097BE6BC16BC46BCA6BC96BB4
:100E3000C86BC76B7C6B800E7C5DD8B02CEF07F065
:100E400001EEB9F0D8907C35E926000EEA22EE6A70
:100E5000EF6A7C2BD8A4EFD77C6B800E7C5DD8B07A
:100E60003EEF07F002EEB9F0D8907C35E926000E8F
:100E7000EA22EE6AEF6A7C2BD8A4EFD77C6B800E57
:100E80007C5DD8B050EF07F003EEB9F0D8907C3518
:100E9000E926000EEA22EE6AEF6A7C2BD8A4EFD78F
:100EA0007C6B150E7C5DD8B062EF07F001EE3BF075
:100EB000D8907C35E926000EEA22EE6AEF6A7C2B98
:100EC000D8A4EFD77C6B150E7C5DD8B074EF07F01B
:100ED00001EE65F0D8907C35E926000EEA22EE6A34
:100EE000EF6A7C2BD8A4EFD77C6B150E7C5DD8B055
:100EF00086EF07F001EE8FF0D8907C35E926000EE2
:100F0000EA22EE6AEF6A7C2BD8A4EFD7FAEF6DF0F5
:100F10007B53D8A4C2EF07F0800E026E040E096E58
:100F2000400E2A6EBC0E296E070E066ED00E056EA0
:100F30007CEC00F0D8A053EF50F05208D8A4F8D7BA
:100F40007CEC00F0D8A053EF50F04D08D8A4F0D7B7
:100F50007CEC00F0D8A053EF50F04308D8A4E8D7B9
:100F60000B6AD8807CEC00F0D8A053EF50F007EE6D
:100F7000A0F00B501DC0EBFF0B2A0B504008F1E115
:100F8000DBEF08F0470E0701A06F500EA16F520E65
:100F9000A26F4D0EA36F430EA46F2C0EA56F300EE3
:100FA000A66F310EA76F310EA86F340EA96F330EE6
:100FB000AA6F370EAB6F2E0EAC6F300EAD6F300ECA
:100FC000AE6F300EAF6F2C0EB06F410EB16F2C0EA6
:100FD000B26F340EB36F320EB46F340EB56F340E81
:100FE000B66F2E0EB76F300EB86F300EB96F300E71
:100FF000BA6F300EBB6F2C0EBC6F4E0EBD6F2C0E39
:10100000BE6F300EBF6F380EC06F330EC16F300E23
:10101000C26F300EC36F2E0EC46F300EC56F300E10
:10102000C66F300EC76F300EC86F2C0EC96F570ECB
:10103000CA6F2C0ECB6FE56B05EEBEF0D8900501A4
:10104000BD35E926000EEA22EECF19F0EFCF1AF0F7
:10105000030EBCEC01F00701E56FE5C7CCF7E56BCB
:1010600005EEBEF0D8900501BD35E926000EEA2256
:10107000EECF19F0EFCF1AF0020EBCEC01F0070131
:10108000E56FE5C7CDF72E0ECE6FE56B05EEBEF032
:10109000D8900501BD35E926000EEA22EECF19F001
:1010A000EFCF1AF0010EBCEC01F00701E56FE5C7C8
:1010B000CFF7E56B05EEBEF0D8900501BD35E9260A
:1010C000000EEA22EECF19F0EFCF1AF0000EBCECC2
:1010D00001F00701E56FE5C7D0F72C0ED16FE56B86
:1010E00006EEAEF0D8900501BD35E926000EEA22E5
:1010F000EECF19F0EFCF1AF0020EBCEC01F00701B1
:10110000E56FE5C7D2F7E56B06EEAEF0D8900501C6
:10111000BD35E926000EEA22EECF19F0EFCF1AF026
:10112000010EBCEC01F00701E56FE5C7D3F7E56BF5
:1011300006EEAEF0D8900501BD35E926000EEA2294
:10114000EECF19F0EFCF1AF0000EBCEC01F0070162
:10115000E56FE5C7D4F72E0ED56F380ED66F350E76
:10116000D76F2C0ED86F320ED96F300EDA6F300E6B
:10117000DB6F380EDC6F300EDD6F380EDE6F2C0E3D
:10118000DF6F2C0EE06F2A0EE16F310EE26F360E2C
:10119000E36F360EE46F0501BD2B780EBD5D0001D7
:1011A000D8A0D5EF08F00501BD6B0001030E1E6E3F
:1011B000200E83EC01F007019F6B0001400E070138
:1011C0009F5D0001D8B01EEF09F007EEA0F0070107
:1011D0009F51EBCF0BF000EE3AF09F510BC0EBFFAD
:1011E00007EEA0F09F51EB500D6E140EF66E120E2E
:1011F000F76E1D681D2A1D5009080001D8A014EFC4
:1012000009F00900F55009000D5CF4E11DC00BF078
:1012100014EF09F0300C310C320C330C340C350C5B
:10122000360C370C380C390C00EE3AF007019F51A0
:101230000BC0EBFF9F2B0001D8A4BFD71200070102
:10124000E66B00010A0E0701E65D0001D8B045EF2C
:1012500009F00701E62903EEB9F0D890E836E9264F
:10126000000EEA22EECF0BF0EFCF0CF007EEE9F024
:10127000D890E635E926000EEA220BC0EEFF0CC03E
:10128000EFFFE62B0001D8A4DCD70701E66B0001D5
:101290000A0E0701E65D0001D8B0D4EF09F0B9C32A
:1012A00019F0BAC31AF0020EBCEC01F00B6E030E7B
:1012B0000B5CD8A48FEF09F007EEE9F0D890070196
:1012C000E635E926000EEA22EECF19F0EFCF1AF04C
:1012D000020EBCEC01F00B6E0B520001D8A48EEF95
:1012E00009F007EEE9F0D8900701E635E926000E8F
:1012F000EA22EECF0DF0EFCF0EF0680E0D240B6E4C
:10130000010E0E200C6E07EEE9F0D890E635E926C6
:10131000000EEA220BC0EEFF0CC0EFFF0001B9C3C4
:1013200019F0BAC31AF0020EBCEC01F00B6E0B52AE
:10133000D8A4CFEF09F007EEE9F0D8900701E63521
:10134000E926000EEA22EECF19F0EFCF1AF0020ED6
:10135000BCEC01F00B6E030E0B5C0001D8A4CEEFC9
:1013600009F007EEE9F0D8900701E635E926000E0E
:10137000EA22EECF0DF0EFCF0EF00D5068080B6EA5
:10138000010E0E540C6E07EEE9F0D890E635E92612
:10139000000EEA220BC0EEFF0CC0EFFF00010701B8
:1013A000E62B0001D8A473D70701E86BE76BE66B67
:1013B00000010A0E0701E65D0001D8B0F4EF09F064
:1013C00007EEE9F0D8900701E635E926000EEA229B
:1013D000EECF0BF0EFCF0CF00B50E7270C50E823CB
:1013E000E62B0001D8A4E4D7E8C71AF0E7C719F044
:1013F0001E6A0A0E1D6E32EC02F00701E76F1AC07A
:10140000E8F7B9C30BF0BAC30CF00B50E75D0C5012
:10141000E8590001D8B01BEF0AF0B9C30BF0BAC30A
:101420000CF00701E7510B5CFD6FE8510C58FE6FA3
:10143000000126EF0AF0B9C30BF0BAC30CF00B5051
:101440000701E75DFD6F0C50E859FE6F00010701D1
:10145000FE530001D8A43AEF0AF0060E0701FD5D25
:101460000001D8B03AEF0AF0B9C3E7F7BAC3E8F71A
:101470003FEF0AF0010E0701E86F680EE76F000109
:10148000E7C7DEFFE8C7DEFF120018EE06F0A2ECA9
:1014900002F018EE04F0A2EC02F00801016B006B00
:1014A00005C81AF004C819F0020EBCEC01F0016B7B
:1014B000006F036B026B07C81AF006C819F0020E22
:1014C000BCEC01F0036B026F0001809F0801025128
:1014D000005D0B6E035101590C6E0B50030A0C108A
:1014E0000001D8A485EF0AF0808F08010451680834
:1014F000046F010E0555056F04510625086F05514F
:101500000721096F4C0E00017D6F08010051025D3B
:101510000B6E015103590C6E0B50030A0C100001A5
:10152000D8A4A2EF0AF0808F680E08010427010EEC
:1015300005230651045D086F07510559096F520EC6
:1015400000017D6FD89680BFD886D8B6D6EF0AF056
:1015500008010451065D055107590001D8B0BDEFDF
:101560000AF008010651045D086F07510559096F1B
:10157000520E00017D6FD6EF0AF008010651045D9E
:10158000075105590001D8B0D2EF0AF00801045103
:10159000065D086F05510759096F4C0E00017D6FFC
:1015A000D5EF0AF00801096B086B0001809F08C89D
:1015B000DEFF09C8DEFF1200B9C30BF0BAC30CF09E
:1015C0000BC0DEFF0CC0DEFF8AC0DEFF8BC0DEFF7B
:1015D0005CDF18EE0BF0A2EC02F00BC811F00CC8A7
:1015E00012F080EC06F0D00E186E0F0E176E490E3A
:1015F000166E800E156EDEEC05F014C016F813C0E2
:1016000015F812C014F811C013F8186A176A340ECE
:10161000166E860E156E16C814F015C813F014C891
:1016200012F013C811F076EC05F014C016F813C0D0
:1016300015F812C014F811C013F816C814F015C824
:1016400013F014C812F013C811F0ABEC02F014C080
:1016500012F813C011F812C010F811C00FF80801E9
:10166000109FB9C20BF0BAC20CF00BC011F00CC045
:1016700012F080EC06F012C818F011C817F010C86C
:1016800016F00FC815F0DEEC05F02EEC06F013C0D6
:101690000EF80D6F0DC8DEFF0EC8DEFF0001120050
:1016A000D89680ADD886D8B65BEF0BF00801206BDA
:1016B0001F6B0001809DB9C317F8BAC318F818C88A
:1016C0001AF017C819F0020EBCEC01F008011A6BF1
:1016D000196FBBC31BF8BCC31CF81CC81AF01BC88D
:1016E00019F0020EBCEC01F01E6B1D6F1D51195D4F
:1016F0000B6E1E511A590C6E0B50030A0C10000190
:10170000D8A48AEF0BF008011B5168081B6F010E6B
:101710001C551C6F0001080119511D5D0B6E1A51FB
:101720001E590C6E0B50030A0C100001D8A49EEF3A
:101730000BF0680E08011727010E1823000108019D
:1017400017511B5D18511C590001D8B0BAEF0BF0AE
:1017500008011F2B040E205D0001D8A0B7EF0BF08D
:101760008081B9C37EF0BAC37FF0B9EF0BF00801F6
:10177000206B000108011B51175D1C511859000115
:10178000D8B0D5EF0BF00801202B040E1F5D00012F
:10179000D8A0D2EF0BF08081B9C37EF0BAC37FF03E
:1017A000D4EF0BF008011F6B0001120018EE6DF072
:1017B00091EC02F018EE69F091EC02F018EE64F092
:1017C00091EC02F018EE5EF091EC02F018EE5AF097
:1017D00091EC02F018EE56F091EC02F0C1517EEC63
:1017E00006F0DB0E186E0F0E176E490E166E800E89
:1017F000156EDEEC05F014C02EF013C02DF012C0F3
:101800002CF011C02BF0186A176A340E166E860E73
:10181000156E2EC014F02DC013F02CC012F02BC08A
:1018200011F076EC05F014C080F813C07FF812C0F8
:101830007EF811C07DF880C814F07FC813F07EC810
:1018400012F07DC811F0ABEC02F014C07CF813C0AC
:101850007BF812C07AF811C079F8146A136A7A0E0C
:10186000126E880E116E7CC818F07BC817F07AC80B
:1018700016F079C815F0DEEC05F02EEC06F011C07C
:1018800078F812C077F813C076F80801756F70C841
:101890001CF06FC81BF06EC81AF06DC819F0246AEE
:1018A000236A226A060E216ED2EC01F01CC070F889
:1018B0001BC06FF81AC06EF819C06DF86CC81CF028
:1018C0006BC81BF06AC81AF069C819F0246A236A49
:1018D000226A060E216ED2EC01F01CC06CF81BC00F
:1018E0006BF81AC06AF819C069F867C81CF066C8B6
:1018F0001BF065C81AF064C819F0246A236A226ACA
:10190000060E216ED2EC01F01CC067F81BC066F811
:101910001AC065F819C064F861C81CF060C81BF0F3
:101920005FC81AF05EC819F0246A236A226A060E9C
:10193000216ED2EC01F01CC061F81BC060F81AC027
:101940005FF819C05EF85DC81CF05CC81BF05BC88E
:101950001AF05AC819F0246A236A226A060E216E08
:10196000D2EC01F01CC05DF81BC05CF81AC05BF83B
:1019700019C05AF859C81CF058C81BF057C81AF0BB
:1019800056C819F0246A236A226A060E216ED2EC28
:1019900001F01CC059F81BC058F81AC057F819C0FC
:1019A00056F85A51645D226F5B516559236F5C5143
:1019B0006659246F5D516759256F25C81CF024C8EE
:1019C0001BF023C81AF022C819F078C824F077C891
:1019D00023F076C822F075C821F049EC02F01CC053
:1019E0002EF01BC02DF01AC02CF019C02BF02EC009
:1019F0001CF02DC01BF02CC01AF02BC019F0246A6B
:101A0000236A030E226EE80E216ED2EC01F01CC098
:101A100029F81BC028F81AC027F819C026F8695100
:101A2000565D2A6F6A5157592B6F6B5158592C6F5D
:101A30006C5159592D6F6D515A5D2E6F6E515B5916
:101A40002F6F6F515C59306F70515D59316F31C8D4
:101A50001CF030C81BF02FC81AF02EC819F078C837
:101A600024F077C823F076C822F075C821F049EC3D
:101A700002F01CC02EF01BC02DF01AC02CF019C0B3
:101A80002BF02EC01CF02DC01BF02CC01AF02BC068
:101A900019F0246A236A030E226EE80E216ED2EC3E
:101AA00001F01CC035F81BC034F81AC033F819C057
:101AB00032F856515E5D366F57515F59376F585146
:101AC0006059386F59516159396F29C81CF028C8BD
:101AD0001BF027C81AF026C819F02DC824F02CC80E
:101AE00023F02BC822F02AC821F049EC02F01CC0D8
:101AF0003DF81BC03CF81AC03BF819C03AF835C88D
:101B00001CF034C81BF033C81AF032C819F039C8B9
:101B100024F038C823F037C822F036C821F049EC49
:101B200002F01CC041F81BC040F81AC03FF819C0B1
:101B30003EF83E513A5D196E3F513B591A6E405185
:101B40003C591B6E41513D591C6E7AEC02F0426FBC
:101B50001AC043F81BC044F81CC045F829C81CF043
:101B600028C81BF027C81AF026C819F029C824F085
:101B700028C823F027C822F026C821F049EC02F03B
:101B80001CC049F81BC048F81AC047F819C046F8ED
:101B900039C81CF038C81BF037C81AF036C819F01D
:101BA00039C824F038C823F037C822F036C821F0ED
:101BB00049EC02F01CC04DF81BC04CF81AC04BF8A1
:101BC00019C04AF84A5146254E6F4B5147214F6F75
:101BD0004C514821506F4D514921516F51C814F05B
:101BE00050C813F04FC812F04EC811F082EC06F046
:101BF00024EC04F02EEC06F011C055F812C054F895
:101C000013C053F8526F45C81CF044C81BF043C8BA
:101C10001AF042C819F0246A236A226A640E216EFF
:101C200049EC02F01CC02EF01BC02DF01AC02CF0A5
:101C300019C02BF02EC01CF02DC01BF02CC01AF0C8
:101C40002BC019F055C824F054C823F053C822F013
:101C500052C821F0D2EC01F01CC074F81BC073F81C
:101C60001AC072F819C071F80001BF53D8A487EFE9
:101C70000EF074C81CF073C81BF072C81AF071C85B
:101C800019F0246A236A226A6F0E216E49EC02F071
:101C90001CC02EF01BC02DF01AC02CF019C02BF068
:101CA0002EC01CF02DC01BF02CC01AF02BC019F058
:101CB000246A236A226A640E216ED2EC01F01CC0F1
:101CC00074F81BC073F81AC072F819C071F8D8966E
:101CD000080174BFD8860001D8B684EF0EF03D0E1F
:101CE0000801715D860E7259010E7359000E745908
:101CF0000001D8A084EF0EF00801746B010E736F21
:101D0000860E726F3C0E716F0001A0EF0FF0010E96
:101D1000BF5DD8A409EF0FF074C81CF073C81BF0A6
:101D200072C81AF071C819F0246A236A226A6F0E09
:101D3000216E49EC02F01CC02EF01BC02DF01AC021
:101D40002CF019C02BF02EC01CF02DC01BF02CC0A5
:101D50001AF02BC019F0246A236A226A640E216EDD
:101D6000D2EC01F01CC074F81BC073F81AC072F8F2
:101D700019C071F874C81CF073C81BF072C81AF04F
:101D800071C819F0246A236A010E226E4D0E216E6D
:101D900049EC02F01CC074F81BC073F81AC072F84A
:101DA00019C071F874C81CF073C81BF072C81AF01F
:101DB00071C819F0246A236A226A640E216ED2EC7B
:101DC00001F01CC074F81BC073F81AC072F819C077
:101DD00071F8D896080174BFD8860001D8B606EF0E
:101DE0000FF03D0E0801715D860E7259010E735998
:101DF000000E74590001D8A006EF0FF00801746BB3
:101E0000010E736F860E726F3C0E716F0001A0EFB2
:101E10000FF0020EBF5DD8A4A0EF0FF074C81CF045
:101E200073C81BF072C81AF071C819F0246A236ACB
:101E3000226A6F0E216E49EC02F01CC02EF01BC00E
:101E40002DF01AC02CF019C02BF02EC01CF02DC0A4
:101E50001BF02CC01AF02BC019F0246A236A226AE6
:101E6000640E216ED2EC01F01CC074F81BC073F834
:101E70001AC072F819C071F874C81CF073C81BF04E
:101E800072C81AF071C819F0246A236A010E226E12
:101E90004D0E216E49EC02F01CC074F81BC073F8A3
:101EA0001AC072F819C071F874C81CF073C81BF01E
:101EB00072C81AF071C819F0246A236A226A640E83
:101EC000216ED2EC01F01CC074F81BC073F81AC06C
:101ED00072F819C071F874C81CF073C81BF072C88E
:101EE0001AF071C819F0246A236A226AC0C021F06E
:101EF000D2EC01F01CC074F81BC073F81AC072F861
:101F000019C071F8D896080174BFD8860001D8B6F8
:101F10009FEF0FF03D0E0801715D860E7259010EA4
:101F20007359000E74590001D8A09FEF0FF00801FB
:101F3000746B010E736F860E726F3C0E716F000131
:101F4000820E026E400E096E2A6A540E296E066ACF
:101F5000056A200E016E440EBEEC00F0490EBEEC88
:101F600000F0530EBEEC00F0540EBEEC00F05F0E1D
:101F7000BEEC00F0320EBEEC00F0300EBEEC00F015
:101F8000300EBEEC00F0200EBEEC00F0640EBEEC95
:101F900000F06F0EBEEC00F06E0EBEEC00F0650EB1
:101FA000BEEC00F03D0EBEEC00F0820E026E400E64
:101FB000096E2A6A540E296E066A056A200E016EA1
:101FC000086A74C82EF073C82DF072C82CF071C85E
:101FD0002BF053EC00F0820E026E400E096E2A6A5E
:101FE000540E296E066A056A200E016E0D0EBEECB7
:101FF00000F0820E026E400E096E2A6A540E296E9F
:10200000066A056A200E016E0A0EBEEC00F071C869
:10201000DEFF72C8DEFF73C8DEFF74C8DEFF120089
:10202000020E0501BF6FD80EBE6F020EC16FDB0E30
:10203000C06F020EC36FDE0EC26F020EC56FE10EDF
:10204000C46F020EC76FE40EC66F020EC96FE70EB3
:10205000C86F020ECB6FEA0ECA6F020ECD6FED0E87
:10206000CC6F020ECF6FF00ECE6F020ED16FF30E5B
:10207000D06F020ED36FF60ED26F020ED56FF90E2F
:10208000D46F020ED76FFC0ED66F020ED96FD869CF
:10209000030EDB6F020EDA6F030EDD6F050EDC6FD1
:1020A000030EDF6F080EDE6F030EE16F0B0EE06FA5
:1020B000030EE36F0E0EE26F030EE56F110EE46F79
:1020C000030EE76F140EE66F030EE96F170EE86F4D
:1020D000030EEB6F1A0EEA6F030EED6F1D0EEC6F21
:1020E000030EEF6F200EEE6F030EF16F230EF06FF5
:1020F000030EF36F260EF26F030EF56F290EF46FC9
:10210000030EF76F2C0EF66F030EF96F2F0EF86F9C
:10211000030EFB6F320EFA6F030EFD6F350EFC6F70
:10212000030EFF6F380EFE6F030E0601016F3B0EAC
:10213000006F030E036F3E0E026F030E056F410E1C
:10214000046F030E076F440E066F030E096F470EF0
:10215000086F030E0B6F4A0E0A6F030E0D6F4D0EC4
:102160000C6F030E0F6F500E0E6F030E116F530E98
:10217000106F030E136F560E126F030E156F590E6C
:10218000146F030E176F5C0E166F030E196F5F0E40
:10219000186F030E1B6F620E1A6F030E1D6F650E14
:1021A0001C6F030E1F6F680E1E6F030E216F6B0EE8
:1021B000206F030E236F6E0E226F030E256F710EBC
:1021C000246F030E276F740E266F030E296F770E90
:1021D000286F030E2B6F7A0E2A6F030E2D6F7D0E64
:1021E0002C6F030E2F6F800E2E6F030E316F830E38
:1021F000306F030E336F860E326F030E356F890E0C
:10220000346F030E376F8C0E366F030E396F8F0EDF
:10221000386F030E3B6F920E3A6F030E3D6F950EB3
:102220003C6F030E3F6F980E3E6F030E416F9B0E87
:10223000406F030E436F9E0E426F030E456FA10E5B
:10224000446F030E476FA40E466F030E496FA70E2F
:10225000486F030E4B6FAA0E4A6F030E4D6FB20EFE
:102260004C6F030E4F6FBA0E4E6F030E516FC20EBE
:10227000506F030E536FCA0E526F030E556FD20E7E
:10228000546F030E576FDA0E566F030E596FE20E3E
:10229000586F030E5B6FEA0E5A6F030E5D6FF20EFE
:1022A0005C6F030E5F6FFA0E5E6F040E616F020EBD
:1022B000606F040E636F0A0E626F040E656F120E7C
:1022C000646F040E676F1A0E666F040E696F220E3C
:1022D000686F040E6B6F2A0E6A6F040E6D6F320EFC
:1022E0006C6F040E6F6F270E6E6F040E716F1C0EF5
:1022F000706F040E736F110E726F040E756F060E01
:10230000746F030E776FFB0E766F030E796FF00E0E
:10231000786F030E7B6FE50E7A6F030E7D6FDA0E1A
:102320007C6F030E7F6FCF0E7E6F030E816FC40E26
:10233000806F030E836FB90E826F030E856FAE0E32
:10234000846F030E876FA30E866F030E896F980E3E
:10235000886F030E8B6F8D0E8A6F030E8D6F820E4A
:102360008C6F030E8F6F770E8E6F030E916F6C0E56
:10237000906F030E936F610E926F030E956F560E62
:10238000946F030E976F4B0E966F030E996F400E6E
:10239000986F030E9B6F350E9A6F030E9D6F2A0E7A
:1023A0009C6F030E9F6F1F0E9E6F030EA16F140E86
:1023B000A06F030EA36F090EA26F020EA56FFE0E93
:1023C000A46F020EA76FF30EA66F020EA96FE80EA0
:1023D000A86F020EAB6FDD0EAA6F020EAD6FD20EAC
:1023E000AC6FAF6B730EAE6FB16B720EB06FB36B41
:1023F000720EB26FB56B730EB46FB76B740EB66FAF
:10240000B96B750EB86FBB6B760EBA6FBD6B770E7E
:10241000BC6FBF6B780EBE6FC16B790EC06FC36BA4
:102420007A0EC26FC56B7B0EC46FC76B7C0EC66F16
:10243000C96B7D0EC86FCB6B7E0ECA6FCD6B7F0EE6
:10244000CC6FCF6B800ECE6FD16B810ED06FD36B04
:10245000820ED26FD56B830ED46FD76B840ED66F7E
:10246000D96B850ED86FDB6B860EDA6FDD6B870E4E
:10247000DC6FDF6B880EDE6FE16B890EE06FE36B64
:102480008A0EE26FE56B8B0EE46FE76B8C0EE66FE6
:10249000E96B8D0EE86FEB6B8E0EEA6FED6B8F0EB6
:1024A000EC6FEF6B900EEE6FF16B910EF06FF36BC4
:1024B000920EF26FF56B930EF46FF76B940EF66F4E
:1024C000F96B950EF86FFB6B960EFA6FFD6B970E1E
:1024D000FC6FFF6B980EFE6F0701016B990E006F8A
:1024E000036B9A0E026F056B9B0E046F076B9C0EBD
:1024F000066F096B9D0E086F0B6B9E0E0A6F0D6BBE
:102500009F0E0C6F0F6BA00E0E6F116BA10E106F54
:10251000136BA20E126F156BA30E146F176BA40E24
:10252000166F196BA50E186F1B6BA60E1A6F1D6B1D
:10253000A70E1C6F1F6BA80E1E6F216BA90E206FBC
:10254000236BAA0E226F256BAB0E246F276BAC0E8C
:10255000266F296BAD0E286F2B6BAC0E2A6F2D6B7F
:10256000AB0E2C6F2F6BAA0E2E6F316BA90E306F36
:10257000336BA80E326F356BA70E346F376BA60E18
:10258000366F396BA50E386F3B6BA40E3A6F3D6BFF
:10259000A30E3C6F3F6BA20E3E6F416BA10E406FCE
:1025A000436BA00E426F456B9F0E446F476B9E0EB0
:1025B000466F496B9D0E486F4B6B9C0E4A6F4D6B7F
:1025C0009B0E4C6F4F6B9A0E4E6F516B990E506F66
:1025D000536B980E526F556B970E546F576B960E48
:1025E000566F596B950E586F5B6B940E5A6F5D6BFF
:1025F000930E5C6F5F6B920E5E6F616B910E606FFE
:10260000636B900E626F656B8F0E646F676B8E0EDF
:10261000666F696B8D0E686F6B6B8C0E6A6F6D6B7E
:102620008B0E6C6F6F6B8A0E6E6F716B890E706F95
:10263000736B880E726F756B870E746F776B860E77
:10264000766F796B850E786F7B6B840E7A6F7D6BFE
:10265000830E7C6F7F6B820E7E6F816B810E806F2D
:10266000836B800E826F856B7F0E846F876B7E0E0F
:10267000866F896B7D0E886F8B6B7C0E8A6F8D6B7E
:102680007B0E8C6F8F6B7A0E8E6F916B790E906FC5
:10269000936B780E926F956B770E946F976B760EA7
:1026A000966F996B750E986F9B6B740E9A6F9D6BFE
:1026B000730E9C6F00011200A30E0801A26FA20E00
:1026C000A36FAB0EA46FAA0EA56F010110510A0DE6
:1026D000F3CF2BF0F4CF2CF011512B240B6E0BC049
:1026E00081F812510A0DF3CF2BF0F4CF2CF01351D7
:1026F0002B240B6E0BC082F814510A0DF3CF2BF074
:10270000F4CF2CF015512B240B6E0BC083F817510E
:102710000A0DF3CF2BF0F4CF2CF018512B240B6EB5
:102720000BC084F819510A0DF3CF2BF0F4CF2CF025
:102730001A512B240B6E0BC085F81B510A0DF3CFD9
:102740002BF0F4CF2CF01C512B240B6E0BC086F811
:102750001D510A0DF3CF2BF0F4CF2CF01E512B247A
:102760000B6E0BC087F84E0E1F5D0001D8A4BDEFA5
:1027700013F030C188F8C3EF13F00A0E01013025C1
:102780000B6E0BC088F80001010120510A0DF3CF38
:102790002BF0F4CF2CF021512B240B6E0BC089F8B9
:1027A00022510A0DF3CF2BF0F4CF2CF023512B2420
:1027B0000B6E0BC08AF824510A0DF3CF2BF0F4CF27
:1027C0002CF025512B240B6E0BC08BF826510A0DD3
:1027D000F3CF2BF0F4CF2CF027512B240B6E0BC032
:1027E0008CF8450E295D0001D8A400EF14F0140EFA
:1027F000010128250B6E0BC08DF8000106EF14F0C7
:102800001E0E010128250B6E0BC08DF80001010181
:102810002A510A0DF3CF2BF0F4CF2CF02B512B249F
:102820000B6E0BC08EF82C510A0DF3CF2BF0F4CFAA
:102830002CF02D512B240B6E0BC08FF831510A0D4B
:10284000F3CF2BF0F4CF2CF032512B240B6E0BC0B6
:1028500090F835510A0DF3CF2BF0F4CF2CF0365110
:102860002B240B6E0BC091F837510A0DF3CF2BF0D0
:10287000F4CF2CF038512B240B6E0BC092F8395149
:102880000A0DF3CF2BF0F4CF2CF03A512B240B6E22
:102890000BC093F80401B9510A0DF3CF2BF0F4CF1C
:1028A0002CF0BA512B240B6E0BC094F8BB510A0DBF
:1028B000F3CF2BF0F4CF2CF0BC512B240B6E0BC0BC
:1028C00095F8EA0E0801966F976B0001160E080145
:1028D000975D0001D8B0F0EF14F0D896AEBFD8865F
:1028E000D8B680EF14F0FE0EAB5DFF0EAC59010EB2
:1028F000AD59000EAE59D8A080EF14F051EF15F08D
:10290000D896AEBFD886D8B6CEEF14F0000EAE5D26
:10291000D8A0CEEF14F011E1000EAD5DD8A0CEEF3F
:1029200014F00BE1FF0EAC5DD8A0CEEF14F005E182
:10293000FE0EAB5DD8A0CEEF14F0AB2B000EAC2397
:10294000AD23AE23FF0EAB5D0801986FFF0E0001B3
:10295000AC590801996F000E0001AD5908019A6F3A
:10296000000E0001AE5908019B6F99C89DF898C8E8
:102970009CF8A5512DEC01F09D512DEC01F09C51DE
:102980002DEC01F008EE81F09751EB502BEC01F0AB
:10299000050E82EC01F00001EAEF14F0AB2B000E03
:1029A000AC23AD23AE23ACC09DF8ABC09CF80801AE
:1029B000A3512DEC01F09D512DEC01F09C512DEC1B
:1029C00001F008EE81F09751EB502BEC01F0050E71
:1029D00082EC01F000010801972B0001D8A475D703
:1029E000AEC09EF8ADC09FF8ACC0A0F8ABC0A1F8D7
:1029F0000801A3512DEC01F00001B0512DEC01F0C4
:102A0000AF512DEC01F008019E512BEC01F0050EA9
:102A100082EC01F0A3512DEC01F0010E0001AF2575
:102A20002B6E000EB0212C6E2C502DEC01F02B5093
:102A30002DEC01F008019F512BEC01F0050E82EC0A
:102A400001F0A3512DEC01F0020E0001AF252B6E19
:102A5000000EB0212C6E2C502DEC01F02B502DECE3
:102A600001F00801A0512BEC01F0050E82EC01F001
:102A7000A3512DEC01F0030E0001AF252B6E000ECB
:102A8000B0212C6E2C502DEC01F02B502DEC01F0D0
:102A90000801A1512BEC01F0050E82EC01F00001C0
:102AA00012000A0E816F56EF15F012008083CDECF4
:102AB00069F01A6A81C019F0000EBCEC01F00B6ECF
:102AC0000B52D8B468EF15F081C082F06AEF15F0B0
:102AD0000B0E826F0A0E815DD8A47BEF15F070ECAF
:102AE0005FF09D0EDE6E200EDE6E010EDE6EF1ECEE
:102AF00054F08AEF19F00B0E815DD8A48CEF15F01D
:102B000037EC5FF02F0EDE6E0C0EDE6E020EDE6E08
:102B1000F1EC54F08AEF19F00C0E815DD8A49DEF12
:102B200015F037EC5FF02D0EDE6E1B0EDE6E020E22
:102B3000DE6EF1EC54F08AEF19F00D0E815DD8A431
:102B4000AEEF15F037EC5FF02B0EDE6E0E0EDE6E84
:102B5000020EDE6EF1EC54F08AEF19F0140E815D76
:102B6000D8A4BEEF15F070EC5FF09F0EDE6E140E71
:102B7000DE6EDE6AF1EC54F08AEF19F0150E815D1D
:102B8000D8A4D6EF15F099EC5FF0250EDE6E1B0E83
:102B9000DE6EDE6AF1EC54F0330EDE6E0E0EDE6E8B
:102BA0000C0EDE6EF1EC54F08AEF19F0160E815D1A
:102BB000D8A4EEEF15F099EC5FF0270EDE6E0C0E48
:102BC000DE6EDE6AF1EC54F0350EDE6E1B0EDE6E4C
:102BD0000C0EDE6EF1EC54F08AEF19F0170E815DE9
:102BE000D8A406EF16F099EC5FF0270EDE6E0C0EFF
:102BF000DE6EDE6AF1EC54F0330EDE6E0E0EDE6E2B
:102C00000C0EDE6EF1EC54F08AEF19F01E0E815DB1
:102C1000D8A417EF16F070EC5FF0A30EDE6E110E65
:102C2000DE6E010EDE6EF1EC54F08AEF19F01F0E2D
:102C3000815DD8A42FEF16F099EC5FF0250EDE6EC3
:102C40001B0EDE6EDE6AF1EC54F0970EDE6E210E86
:102C5000DE6E0C0EDE6EF1EC54F08AEF19F0200EF1
:102C6000815DD8A447EF16F099EC5FF0250EDE6E7B
:102C70001B0EDE6EDE6AF1EC54F0950EDE6E210E58
:102C8000DE6E0C0EDE6EF1EC54F08AEF19F0210EC0
:102C9000815DD8A45FEF16F099EC5FF0250EDE6E33
:102CA0001B0EDE6EDE6AF1EC54F0930EDE6E210E2A
:102CB000DE6E0C0EDE6EF1EC54F08AEF19F0220E8F
:102CC000815DD8A477EF16F099EC5FF0250EDE6EEB
:102CD0001B0EDE6EDE6AF1EC54F0990EDE6E210EF4
:102CE000DE6E0C0EDE6EF1EC54F08AEF19F0230E5E
:102CF000815DD8A48FEF16F099EC5FF0270EDE6EA1
:102D00000C0EDE6EDE6AF1EC54F0950EDE6E210ED6
:102D1000DE6E0C0EDE6EF1EC54F08AEF19F0240E2C
:102D2000815DD8A4A7EF16F099EC5FF0270EDE6E58
:102D30000C0EDE6EDE6AF1EC54F0930EDE6E210EA8
:102D4000DE6E0C0EDE6EF1EC54F08AEF19F0250EFB
:102D5000815DD8A4BFEF16F099EC5FF0270EDE6E10
:102D60000C0EDE6EDE6AF1EC54F0970EDE6E210E74
:102D7000DE6E0C0EDE6EF1EC54F08AEF19F0260ECA
:102D8000815DD8A4D7EF16F099EC5FF0270EDE6EC8
:102D90000C0EDE6EDE6AF1EC54F0990EDE6E210E42
:102DA000DE6E0C0EDE6EF1EC54F08AEF19F0270E99
:102DB000815DD8A4EFEF16F099EC5FF0230EDE6E84
:102DC0000E0EDE6EDE6AF1EC54F0930EDE6E210E16
:102DD000DE6E0C0EDE6EF1EC54F08AEF19F0280E68
:102DE000815DD8A407EF17F099EC5FF0230EDE6E3B
:102DF0000E0EDE6EDE6AF1EC54F0950EDE6E210EE4
:102E0000DE6E0C0EDE6EF1EC54F08AEF19F0290E36
:102E1000815DD8A41FEF17F099EC5FF0230EDE6EF2
:102E20000E0EDE6EDE6AF1EC54F0970EDE6E210EB1
:102E3000DE6E0C0EDE6EF1EC54F08AEF19F02A0E05
:102E4000815DD8A437EF17F099EC5FF0230EDE6EAA
:102E50000E0EDE6EDE6AF1EC54F0990EDE6E210E7F
:102E6000DE6E0C0EDE6EF1EC54F08AEF19F0320ECD
:102E7000815DD8A448EF17F070EC5FF0A50EDE6E10
:102E80000F0EDE6E010EDE6EF1EC54F08AEF19F0DB
:102E9000330E815DD8A458EF17F037EC5FF0140EB5
:102EA000DE6E200EDE6EDE6AF1EC54F08AEF19F071
:102EB000340E815DD8A4AEEF17F037EC5FF0EB0E67
:102EC000DE6E2A0EDE6EDE6AF1EC54F0010EA95DB4
:102ED000D8A47EEF17F0DE6A0F0EDE6E380EDE6EBF
:102EE000040EDE6E18EC5FF04D0EDE6E3F0EDE6EF1
:102EF000040EDE6EF1EC54F0ACEF17F0020EA95D9B
:102F0000D8A496EF17F0DE6A0F0EDE6E380EDE6E76
:102F1000040EDE6E18EC5FF0590EDE6E450EDE6EAE
:102F2000040EDE6EF1EC54F0ACEF17F0030EA95D69
:102F3000D8A4ACEF17F0DE6A0F0EDE6E380EDE6E30
:102F4000040EDE6E18EC5FF0550EDE6E380EDE6E8F
:102F5000040EDE6EF1EC54F08AEF19F0350E815D4F
:102F6000D8A4CEEF17F0550EDE6E380EDE6EDE6A98
:102F7000F1EC54F0570EDE6E360EDE6E020EDE6E93
:102F8000F1EC54F0850EDE6E2F0EDE6E040EDE6E5A
:102F9000F1EC54F037EC5FF08AEF19F0360E815DFA
:102FA000D8A4DEEF17F037EC5FF0180EDE6E1E0EC1
:102FB000DE6EDE6AF1EC54F08AEF19F0370E815DB7
:102FC000D8A4EEEF17F037EC5FF0160EDE6E250E8C
:102FD000DE6EDE6AF1EC54F08AEF19F03C0E815D92
:102FE000D8A4FFEF17F070EC5FF0ED0EDE6E1F0E51
:102FF000DE6E010EDE6EF1EC54F08AEF19F03D0E3C
:10300000815DD8A40FEF18F037EC5FF0F30EDE6EA1
:103010001A0EDE6EDE6AF1EC54F08AEF19F03E0E05
:10302000815DD8A427EF18F037EC5FF0E90EDE6E73
:103030001C0EDE6EDE6AF1EC54F0ED0EDE6E1F0E3D
:10304000DE6E040EDE6EF1EC54F08AEF19F03F0EE6
:10305000815DD8A43FEF18F037EC5FF0EB0EDE6E29
:103060002A0EDE6EDE6AF1EC54F0ED0EDE6E1F0EFF
:10307000DE6E040EDE6EF1EC54F08AEF19F0400EB5
:10308000815DD8A458EF18F037EC5FF0890EDE6E42
:10309000200EDE6E010EDE6EF1EC54F0ED0EDE6EF3
:1030A0001F0EDE6E040EDE6EF1EC54F08AEF19F0A6
:1030B000410E815DD8A487EF18F037EC5FF0A30EC6
:1030C000DE6E110EDE6EDE6AF1EC54F0080EDE6E7E
:1030D000130EDE6E030EDE6EF1EC54F0010EBE5DDB
:1030E000D8A47DEF18F0F50EDE6E390EDE6E060EFA
:1030F000DE6EF1EC54F085EF18F0F70EDE6E390E4F
:10310000DE6E060EDE6EF1EC54F08AEF19F0420E20
:10311000815DD8A4AFEF18F037EC5FF0020EDE6EE1
:10312000240EDE6E010EDE6EF1EC54F0010E7B5DBE
:10313000D8A4A5EF18F0F50EDE6E390EDE6E060E81
:10314000DE6EF1EC54F0ADEF18F0F70EDE6E390ED6
:10315000DE6E060EDE6EF1EC54F08AEF19F0430ECF
:10316000815DD8A4C8EF18F037EC5FF0120EDE6E68
:10317000150EDE6E010EDE6EF1EC54F0ED0EDE6E1D
:103180001F0EDE6E040EDE6EF1EC54F08AEF19F0C5
:10319000440E815DD8A4FFEF18F037EC5FF0850E88
:1031A000DE6E2F0EDE6EDE6AF1EC54F0550EDE6E32
:1031B000120EDE6E030EDE6EF1EC54F0630EDE6E68
:1031C000460EDE6E030EDE6EF1EC54F0010E855DF0
:1031D000D8A4F5EF18F0F50EDE6E390EDE6E060E91
:1031E000DE6EF1EC54F0FDEF18F0F70EDE6E390EE6
:1031F000DE6E060EDE6EF1EC54F08AEF19F0460E2C
:10320000815DD8A441EF19F01B0EDE6E0D0EDE6E4F
:10321000030EDE6EF1EC54F0630EDE6E190EDE6E00
:103220000A0EDE6EF1EC54F0D70EDE6E6E0EDE6E20
:10323000090EDE6EF1EC54F0D90EDE6E6E0EDE6E0F
:103240000B0EDE6EF1EC54F04F0EDE6E3F0EDE6EB6
:103250000E0EDE6EF1EC54F0DF0EDE6E780EDE6EDA
:103260000E0EDE6EF1EC54F0DB0EDE6E6D0EDE6ED9
:103270000E0EDE6EF1EC54F0C80E82EC01F08AEF17
:1032800019F0470E815DD8A488EF19F01B0EDE6E91
:103290000D0EDE6E030EDE6EF1EC54F0E10EDE6E0E
:1032A0003F0EDE6E0A0EDE6EF1EC54F0D70EDE6ECF
:1032B0006E0EDE6E080EDE6EF1EC54F0D90EDE6E90
:1032C0006E0EDE6E0C0EDE6EF1EC54F0DF0EDE6E76
:1032D000800EDE6E0A0EDE6EF1EC54F0DB0EDE6E5A
:1032E000650EDE6E0A0EDE6EF1EC54F04F0EDE6EF1
:1032F0003F0EDE6E0E0EDE6EF1EC54F0DD0EDE6E75
:10330000650EDE6E0E0EDE6EF1EC54F08AEF19F0F3
:1033100056EF15F0C20ED76EF70ED66EF294080176
:10332000BF6BBE6B010E1E6EF40E83EC01F000014C
:10333000F2A4A3EF19F0C20ED76EF70ED66EF29478
:103340000801BE4BBF2B0001030E0801BF5D000149
:10335000D8A0B7EF19F0D8A4B5EF19F0850E080181
:10336000BE5D0001D8A0B7EF19F053EC50F0080192
:10337000BA9300018C6B80A0C3EF19F00801BA83E7
:10338000030E00018C6F81A2CBEF19F00801BA8304
:10339000040E00018C6F80AAD3EF19F00801BA83E4
:1033A000010E00018C6F82A2DBEF19F00801BA83D5
:1033B000020E00018C6F82A0E3EF19F00801BA83BE
:1033C000050E00018C6FD8960801BAB3D8860001AB
:1033D000D8B665EF1AF0810E026E010E096E400E2E
:1033E0002A6E200E296E066A640E056E0B6AD8805E
:1033F0007CEC00F0D8A09BD708EEAAF00B501DC0C3
:10340000EBFF0B2A0B501008F2E10801BB6B000127
:10341000100E0801BB5D0001D8B065EF1AF008EE90
:10342000AAF00801BB51EB500B6E030E0B5C0001C0
:10343000D8A460EF1AF0030E0801BB2508EEAAF02D
:10344000EB50BD6F1A6ABDC819F0080E6BEC02F0A4
:10345000BC6F800EBC5D0001D8A433EF1AF0010EE2
:103460008C6F60EF1AF0400E0801BC5D0001D8A41B
:103470003EEF1AF0020E8C6F60EF1AF0200E08017A
:10348000BC5D0001D8A449EF1AF0030E8C6F60EF09
:103490001AF0100E0801BC5D0001D8A454EF1AF018
:1034A000040E8C6F60EF1AF0080E0801BC5D00017D
:1034B000D8A45FEF1AF0050E8C6F60EF1AF08C6BDA
:1034C0000801BB2B0001D8A4A2D7010E8C5DD8A4A3
:1034D000A5EF1AF0470E815DD8A471EF1AF053EFF3
:1034E00050F00A0EF66E350EF76E1D681D2A1D503F
:1034F0000908D8A08FEF1AF00900F5500900815D86
:10350000F5E11DC089F08FEF1AF0630C0C0C150C5F
:10351000160C1F0C200C210C220C250C290C280E3B
:10352000815DD8A496EF1AF07DEF1FF01A6A81C072
:1035300019F0000EBCEC01F00B6E0B52D8B4A3EFE7
:103540001AF07DEF1FF058EF1BF0020E8C5DD8A42F
:10355000C9EF1AF081C019F00A0E2FEC02F0816F4A
:1035600081510A0DF3CF2BF0F4CF2CF00A0E2B244F
:10357000816F280E815DD8A4C0EF1AF0320E816FE2
:10358000500E815DD8A4C7EF1AF00A0E816F58EF74
:103590001BF0030E8C5DD8A4ECEF1AF081C019F07B
:1035A0000A0E2FEC02F0816F81510A0DF3CF2BF040
:1035B000F4CF2CF00A0E2B5C816F280E815DD8A40D
:1035C000E4EF1AF01E0E816F8153D8A4EAEF1AF0CF
:1035D000460E816F58EF1BF0040E8C5DD8A41EEFD1
:1035E0001BF0812B0E0E815DD8A4F9EF1AF00A0EA4
:1035F000816F180E815DD8A400EF1BF0140E816F4F
:103600002B0E815DD8A407EF1BF01E0E816F380EC4
:10361000815DD8A40EEF1BF0320E816F450E815DE7
:10362000D8A415EF1BF03C0E816F480E815DD8A425
:103630001CEF1BF0460E816F58EF1BF0050E8C5DE2
:10364000D8A450EF1BF08107090E815DD8A42BEFA1
:103650001BF00D0E816F130E815DD8A432EF1BF0AD
:10366000170E816F1D0E815DD8A439EF1BF02A0E55
:10367000816F310E815DD8A440EF1BF0370E816F52
:103680003B0E815DD8A447EF1BF0440E816F450EC1
:10369000815DD8A44EEF1BF0470E816F58EF1BF0F1
:1036A0008C53D8A457EF1BF042D658EF1BF03FD6EF
:1036B000CDEC69F00A0E815DD8A46BEF1BF070ECC5
:1036C0005FF09D0EDE6E200EDE6E010EDE6EF1EC02
:1036D00054F07AEF1FF00B0E815DD8A47CEF1BF045
:1036E00037EC5FF02F0EDE6E0C0EDE6E020EDE6E1D
:1036F000F1EC54F07AEF1FF00C0E815DD8A48DEF41
:103700001BF037EC5FF02D0EDE6E1B0EDE6E020E30
:10371000DE6EF1EC54F07AEF1FF00D0E815DD8A44F
:103720009EEF1BF037EC5FF02B0EDE6E0E0EDE6EA2
:10373000020EDE6EF1EC54F07AEF1FF0140E815D94
:10374000D8A4AEEF1BF070EC5FF09F0EDE6E140E8F
:10375000DE6EDE6AF1EC54F07AEF1FF0150E815D3B
:10376000D8A4C6EF1BF099EC5FF0250EDE6E1B0EA1
:10377000DE6EDE6AF1EC54F0330EDE6E0E0EDE6E9F
:103780000C0EDE6EF1EC54F07AEF1FF0160E815D38
:10379000D8A4DEEF1BF099EC5FF0270EDE6E0C0E66
:1037A000DE6EDE6AF1EC54F0350EDE6E1B0EDE6E60
:1037B0000C0EDE6EF1EC54F07AEF1FF0170E815D07
:1037C000D8A4F6EF1BF099EC5FF0270EDE6E0C0E1E
:1037D000DE6EDE6AF1EC54F0330EDE6E0E0EDE6E3F
:1037E0000C0EDE6EF1EC54F07AEF1FF01E0E815DD0
:1037F000D8A407EF1CF070EC5FF0A30EDE6E110E84
:10380000DE6E010EDE6EF1EC54F07AEF1FF01F0E4B
:10381000815DD8A41FEF1CF099EC5FF0250EDE6EE1
:103820001B0EDE6EDE6AF1EC54F0970EDE6E210E9A
:10383000DE6E0C0EDE6EF1EC54F07AEF1FF0200E0F
:10384000815DD8A437EF1CF099EC5FF0250EDE6E99
:103850001B0EDE6EDE6AF1EC54F0950EDE6E210E6C
:10386000DE6E0C0EDE6EF1EC54F07AEF1FF0210EDE
:10387000815DD8A44FEF1CF099EC5FF0250EDE6E51
:103880001B0EDE6EDE6AF1EC54F0930EDE6E210E3E
:10389000DE6E0C0EDE6EF1EC54F07AEF1FF0220EAD
:1038A000815DD8A467EF1CF099EC5FF0250EDE6E09
:1038B0001B0EDE6EDE6AF1EC54F0990EDE6E210E08
:1038C000DE6E0C0EDE6EF1EC54F07AEF1FF0230E7C
:1038D000815DD8A47FEF1CF099EC5FF0270EDE6EBF
:1038E0000C0EDE6EDE6AF1EC54F0950EDE6E210EEB
:1038F000DE6E0C0EDE6EF1EC54F07AEF1FF0240E4B
:10390000815DD8A497EF1CF099EC5FF0270EDE6E76
:103910000C0EDE6EDE6AF1EC54F0930EDE6E210EBC
:10392000DE6E0C0EDE6EF1EC54F07AEF1FF0250E19
:10393000815DD8A4AFEF1CF099EC5FF0270EDE6E2E
:103940000C0EDE6EDE6AF1EC54F0970EDE6E210E88
:10395000DE6E0C0EDE6EF1EC54F07AEF1FF0260EE8
:10396000815DD8A4C7EF1CF099EC5FF0270EDE6EE6
:103970000C0EDE6EDE6AF1EC54F0990EDE6E210E56
:10398000DE6E0C0EDE6EF1EC54F07AEF1FF0270EB7
:10399000815DD8A4DFEF1CF099EC5FF0230EDE6EA2
:1039A0000E0EDE6EDE6AF1EC54F0930EDE6E210E2A
:1039B000DE6E0C0EDE6EF1EC54F07AEF1FF0280E86
:1039C000815DD8A4F7EF1CF099EC5FF0230EDE6E5A
:1039D0000E0EDE6EDE6AF1EC54F0950EDE6E210EF8
:1039E000DE6E0C0EDE6EF1EC54F07AEF1FF0290E55
:1039F000815DD8A40FEF1DF099EC5FF0230EDE6E11
:103A00000E0EDE6EDE6AF1EC54F0970EDE6E210EC5
:103A1000DE6E0C0EDE6EF1EC54F07AEF1FF02A0E23
:103A2000815DD8A427EF1DF099EC5FF0230EDE6EC8
:103A30000E0EDE6EDE6AF1EC54F0990EDE6E210E93
:103A4000DE6E0C0EDE6EF1EC54F07AEF1FF0320EEB
:103A5000815DD8A438EF1DF070EC5FF0A50EDE6E2E
:103A60000F0EDE6E010EDE6EF1EC54F07AEF1FF0F9
:103A7000330E815DD8A448EF1DF037EC5FF0140ED3
:103A8000DE6E200EDE6EDE6AF1EC54F07AEF1FF08F
:103A9000340E815DD8A49EEF1DF037EC5FF0EB0E85
:103AA000DE6E2A0EDE6EDE6AF1EC54F0010EA95DC8
:103AB000D8A46EEF1DF0DE6A0F0EDE6E380EDE6EDD
:103AC000040EDE6E18EC5FF04D0EDE6E3F0EDE6E05
:103AD000040EDE6EF1EC54F09CEF1DF0020EA95DB9
:103AE000D8A486EF1DF0DE6A0F0EDE6E380EDE6E95
:103AF000040EDE6E18EC5FF0590EDE6E450EDE6EC3
:103B0000040EDE6EF1EC54F09CEF1DF0030EA95D87
:103B1000D8A49CEF1DF0DE6A0F0EDE6E380EDE6E4E
:103B2000040EDE6E18EC5FF0550EDE6E380EDE6EA3
:103B3000040EDE6EF1EC54F07AEF1FF0350E815D6D
:103B4000D8A4BEEF1DF0550EDE6E380EDE6EDE6AB6
:103B5000F1EC54F0570EDE6E360EDE6E020EDE6EA7
:103B6000F1EC54F0850EDE6E2F0EDE6E040EDE6E6E
:103B7000F1EC54F037EC5FF07AEF1FF0360E815D18
:103B8000D8A4CEEF1DF037EC5FF0180EDE6E1E0EDF
:103B9000DE6EDE6AF1EC54F07AEF1FF0370E815DD5
:103BA000D8A4DEEF1DF037EC5FF0160EDE6E250EAA
:103BB000DE6EDE6AF1EC54F07AEF1FF03C0E815DB0
:103BC000D8A4EFEF1DF070EC5FF0ED0EDE6E1F0E6F
:103BD000DE6E010EDE6EF1EC54F07AEF1FF03D0E5A
:103BE000815DD8A4FFEF1DF037EC5FF0F30EDE6EC1
:103BF0001A0EDE6EDE6AF1EC54F07AEF1FF03E0E24
:103C0000815DD8A417EF1EF037EC5FF0E90EDE6E91
:103C10001C0EDE6EDE6AF1EC54F0ED0EDE6E1F0E51
:103C2000DE6E040EDE6EF1EC54F07AEF1FF03F0E04
:103C3000815DD8A42FEF1EF037EC5FF0EB0EDE6E47
:103C40002A0EDE6EDE6AF1EC54F0ED0EDE6E1F0E13
:103C5000DE6E040EDE6EF1EC54F07AEF1FF0400ED3
:103C6000815DD8A448EF1EF037EC5FF0890EDE6E60
:103C7000200EDE6E010EDE6EF1EC54F0ED0EDE6E07
:103C80001F0EDE6E040EDE6EF1EC54F07AEF1FF0C4
:103C9000410E815DD8A477EF1EF037EC5FF0A30EE4
:103CA000DE6E110EDE6EDE6AF1EC54F0080EDE6E92
:103CB000130EDE6E030EDE6EF1EC54F0010EBE5DEF
:103CC000D8A46DEF1EF0F50EDE6E390EDE6E060E18
:103CD000DE6EF1EC54F075EF1EF0F70EDE6E390E6D
:103CE000DE6E060EDE6EF1EC54F07AEF1FF0420E3F
:103CF000815DD8A49FEF1EF037EC5FF0020EDE6E00
:103D0000240EDE6E010EDE6EF1EC54F0010E7B5DD2
:103D1000D8A495EF1EF0F50EDE6E390EDE6E060E9F
:103D2000DE6EF1EC54F09DEF1EF0F70EDE6E390EF4
:103D3000DE6E060EDE6EF1EC54F07AEF1FF0430EED
:103D4000815DD8A4B8EF1EF037EC5FF0120EDE6E86
:103D5000150EDE6E010EDE6EF1EC54F0ED0EDE6E31
:103D60001F0EDE6E040EDE6EF1EC54F07AEF1FF0E3
:103D7000440E815DD8A4EFEF1EF037EC5FF0850EA6
:103D8000DE6E2F0EDE6EDE6AF1EC54F0550EDE6E46
:103D9000120EDE6E030EDE6EF1EC54F0630EDE6E7C
:103DA000460EDE6E030EDE6EF1EC54F0010E855D04
:103DB000D8A4E5EF1EF0F50EDE6E390EDE6E060EAF
:103DC000DE6EF1EC54F0EDEF1EF0F70EDE6E390E04
:103DD000DE6E060EDE6EF1EC54F07AEF1FF0460E4A
:103DE000815DD8A431EF1FF01B0EDE6E0D0EDE6E6E
:103DF000030EDE6EF1EC54F0630EDE6E190EDE6E15
:103E00000A0EDE6EF1EC54F0D70EDE6E6E0EDE6E34
:103E1000090EDE6EF1EC54F0D90EDE6E6E0EDE6E23
:103E20000B0EDE6EF1EC54F04F0EDE6E3F0EDE6ECA
:103E30000E0EDE6EF1EC54F0DF0EDE6E780EDE6EEE
:103E40000E0EDE6EF1EC54F0DB0EDE6E6D0EDE6EED
:103E50000E0EDE6EF1EC54F0C80E82EC01F07AEF3B
:103E60001FF0470E815DD8A478EF1FF01B0EDE6EA9
:103E70000D0EDE6E030EDE6EF1EC54F0E10EDE6E22
:103E80003F0EDE6E0A0EDE6EF1EC54F0D70EDE6EE3
:103E90006E0EDE6E080EDE6EF1EC54F0D90EDE6EA4
:103EA0006E0EDE6E0C0EDE6EF1EC54F0DF0EDE6E8A
:103EB000800EDE6E0A0EDE6EF1EC54F0DB0EDE6E6E
:103EC000650EDE6E0A0EDE6EF1EC54F04F0EDE6E05
:103ED0003F0EDE6E0E0EDE6EF1EC54F0DD0EDE6E89
:103EE000650EDE6E0E0EDE6EF1EC54F07AEF1FF012
:103EF00056EF15F097EF19F01200A30E0901386F75
:103F0000A20E396FAB0E3A6FAA0E3B6F360E000150
:103F1000815DD8B092EF1FF088EC07F00AEC32F028
:103F200095EF1FF0C80E82EC01F07A6BD89680A353
:103F3000D886D8B69EEF1FF0CDEC69F0440E815DB7
:103F4000D8B43AEF20F0010E855DD8A43AEF20F006
:103F5000330E815DD8B43AEF20F0360E815DD8B4CF
:103F60003AEF20F08353D8A4BAEF1FF081C083F05A
:103F7000C6EF1FF08453D8A4C6EF1FF08351815DB4
:103F8000D8B4C6EF1FF081C084F08085D89680A594
:103F9000D886D8B63AEF20F081C086F0B9C30BF0CE
:103FA000BAC30CF08A510B5C8B510C58D8A0E9EFC6
:103FB0001FF0B9C30BF0BAC30CF08A510B5C0901B6
:103FC0002F6F00018B510C580901306F0001F6EF83
:103FD0001FF0B9C30BF0BAC30CF00B508A5D090196
:103FE0002F6F0C5000018B590901306F000109013E
:103FF00030530001D8A406EF20F05B0E09012F5DBD
:104000000001D8B006EF20F083C081F0010E090155
:10401000305D0001D8A019EF20F0D8A417EF20F0F0
:104020000E0E09012F5D0001D8A019EF20F083C00A
:1040300081F0090130530001D8A426EF20F05B0E77
:1040400009012F5D0001D8A032EF20F0010E090117
:10405000305D0E0ED8B42F5D0001D8B032EF20F0E5
:1040600084C081F08151865DD8B43AEF20F080831E
:10407000CDEC69F00B0E815DD8A4B1EF20F012EC0D
:104080004AF0010E8C5DD8A448EF20F056EF15F0F1
:10409000050E8C5DD8A455EF20F082C02EF981C0AA
:1040A00082F02EC981F0808328D7D89680A3D88645
:1040B000D8B665EF20F00801BA95270EDE6E180E0F
:1040C000DE6EDE6A0001F1EC54F050EC61F0BBC230
:1040D0000BF0BCC20CF00BC0DEFF0CC0DEFFB9C29F
:1040E0000BF0BAC20CF00BC0DEFF0CC0DEFF75ECAB
:1040F00044F0FF0EDB50DD520801BA85E8A0BA9506
:10410000D896BAA5D8860001D8B69BEF20F0B9C2E0
:104110000BF0BAC20CF00BC0DEFF0CC0DEFFBBC25E
:104120000BF0BCC20CF00BC0DEFF0CC0DEFF78EC65
:1041300045F0ADEF20F0B9C20BF0BAC20CF00BC0E5
:10414000DEFF0CC0DEFFBBC20BF0BCC20CF00BC02C
:10415000DEFF0CC0DEFF40EC45F08093CED608EFCA
:1041600032F0170E815DD8A40FEF21F012EC4AF067
:10417000010E8C5DD8A4BFEF20F056EF15F0050EB0
:104180008C5DD8A4CCEF20F082C02EF981C082F0E3
:104190002EC981F08083B1D6D89680A3D886D8B6B0
:1041A000E1EF20F0D10EDE6E050EDE6EDE6AF1EC80
:1041B00054F03F0EDE6E860EDE6E0A0EDE6EF1EC01
:1041C00054F0BBC20BF0BCC20CF00BC0DEFF0CC045
:1041D000DEFFB9C20BF0BAC20CF00BC0DEFF0CC0A0
:1041E000DEFF010EDE6EDE6AB5EC45F0BBC30BF000
:1041F000BCC30CF00BC0DEFF0CC0DEFFB9C30BF07C
:10420000BAC30CF00BC0DEFF0CC0DEFFDE6A010E8D
:10421000DE6EB5EC45F0809370D608EF32F0230ED9
:10422000815DD8A45CEF21F012EC4AF0010E8C5DA8
:10423000D8A41DEF21F056EF15F0050E8C5DD8A423
:104240002AEF21F082C02EF981C082F02EC981F0C0
:10425000808353D6D89680A3D886D8B63FEF21F076
:10426000D10EDE6E050EDE6EDE6AF1EC54F0D30E7A
:10427000DE6E8E0EDE6E090EDE6EF1EC54F0BBC209
:104280000BF0BCC20CF00BC0DEFF0CC0DEFFB9C2ED
:104290000BF0BAC20CF00BC0DEFF0CC0DEFF010E4B
:1042A000DE6EDE6AB5EC45F0010EDE6EB9EC62F052
:1042B000809323D608EF32F0250E815DD8A4C3EF9A
:1042C00021F012EC4AF0010E8C5DD8A46CEF21F0C5
:1042D00056EF15F082EF21F0020E8C5DD8A478EF36
:1042E00021F0CDEC69F0808315EF4FF082EF21F0E3
:1042F000030E8C5DD8A482EF21F0CDEC69F08083B1
:1043000015EF4FF0050E8C5DD8A490EF21F082C020
:104310002EF981C082F02EC981F080837DEF1FF0DD
:10432000D89680A3D886D8B6A5EF21F0D10EDE6E40
:10433000050EDE6EDE6AF1EC54F0CF0EDE6E900EEE
:10434000DE6E080EDE6EF1EC54F0BBC20BF0BCC2A8
:104350000CF00BC0DEFF0CC0DEFFB9C20BF0BAC21E
:104360000CF00BC0DEFF0CC0DEFF010EDE6EDE6A5D
:10437000B5EC45F0020EDE6EB9EC62F080937DEF95
:104380001FF008EF32F0240E815DD8A412EF22F066
:1043900012EC4AF0010E8C5DD8A4D1EF21F056EF5B
:1043A00015F0050E8C5DD8A4DFEF21F082C02EF948
:1043B00081C082F02EC981F080837DEF1FF0D896F6
:1043C00080A3D886D8B6F4EF21F0D10EDE6E050EAC
:1043D000DE6EDE6AF1EC54F03F0EDE6E860EDE6EAF
:1043E0000A0EDE6EF1EC54F0BBC20BF0BCC20CF056
:1043F0000BC0DEFF0CC0DEFFB9C20BF0BAC20CF07E
:104400000BC0DEFF0CC0DEFF010EDE6EDE6AB5EC17
:1044100045F0030EDE6EB9EC62F080937DEF1FF085
:1044200008EF32F0260E815DD8A469EF22F012EC7D
:104430004AF0010E8C5DD8A420EF22F056EF15F063
:10444000040E8C5DD8A42AEF22F08081B9C37EF0DF
:10445000BAC37FF0050E8C5DD8A438EF22F082C07D
:104460002EF981C082F02EC981F080837DEF1FF08C
:10447000D89680A3D886D8B64DEF22F0D10EDE6E46
:10448000050EDE6EDE6AF1EC54F0490EDE6E640E4F
:10449000DE6E0E0EDE6EF1EC54F0BBC20BF0BCC251
:1044A0000CF00BC0DEFF0CC0DEFFB9C20BF0BAC2CD
:1044B0000CF00BC0DEFF0CC0DEFF010EDE6EDE6A0C
:1044C000B5EC45F095EC43F080937DEF1FF008EFDD
:1044D00032F0160E815DD8A4E0EF22F012EC4AF023
:1044E000010E8C5DD8A479EF22F056EF15F08FEF16
:1044F00022F0020E8C5DD8A485EF22F0CDEC69F09D
:10450000808315EF4FF08FEF22F0030E8C5DD8A45F
:104510008FEF22F0CDEC69F0808315EF4FF0050EA0
:104520008C5DD8A49DEF22F082C02EF981C082F06C
:104530002EC981F080837DEF1FF0D89680A3D886A6
:10454000D8B6B2EF22F0D10EDE6E050EDE6EDE6A58
:10455000F1EC54F0CF0EDE6E900EDE6E080EDE6EC5
:10456000F1EC54F0BBC20BF0BCC20CF00BC0DEFF90
:104570000CC0DEFFB9C20BF0BAC20CF00BC0DEFFFC
:104580000CC0DEFF010EDE6EDE6AB5EC45F0BBC18D
:104590000BF0BCC10CF00BC0DEFF0CC0DEFFB9C1DC
:1045A0000BF0BAC10CF00BC0DEFF0CC0DEFFDE6A00
:1045B000DE6AB5EC45F080937DEF1FF008EF32F036
:1045C0000C0E815DD8A471EF23F012EC4AF0010EBD
:1045D0008C5DD8A4F0EF22F056EF15F006EF23F033
:1045E000020E8C5DD8A4FCEF22F0CDEC69F0808344
:1045F00015EF4FF006EF23F0030E8C5DD8A406EF05
:1046000023F0CDEC69F0808315EF4FF0050E8C5D43
:10461000D8A414EF23F082C02EF981C082F02EC9F5
:1046200081F080837DEF1FF0D89680A3D886D8B61E
:1046300024EF23F00801BA95250EDE6E180EDE6E0B
:10464000DE6A0001F1EC54F050EC61F0BBC10BF0FC
:10465000BCC10CF00BC0DEFF0CC0DEFFB9C10BF01B
:10466000BAC10CF00BC0DEFF0CC0DEFF75EC44F0ED
:10467000FF0EDB50DD520801BA85E8A0BA95D89646
:10468000BAA5D8860001D8B65AEF23F0B9C10BF00D
:10469000BAC10CF00BC0DEFF0CC0DEFFBBC10BF0DB
:1046A000BCC10CF00BC0DEFF0CC0DEFF78EC45F0A7
:1046B0006CEF23F0B9C10BF0BAC10CF00BC0DEFFF8
:1046C0000CC0DEFFBBC10BF0BCC10CF00BC0DEFFA9
:1046D0000CC0DEFF40EC45F080937DEF1FF008EF4B
:1046E00032F0150E815DD8A4E8EF23F012EC4AF009
:1046F000010E8C5DD8A481EF23F056EF15F097EFF3
:1047000023F0020E8C5DD8A48DEF23F0CDEC69F080
:10471000808315EF4FF097EF23F0030E8C5DD8A444
:1047200097EF23F0CDEC69F0808315EF4FF0050E85
:104730008C5DD8A4A5EF23F082C02EF981C082F051
:104740002EC981F080837DEF1FF0D89680A3D88694
:10475000D8B6B9EF23F0CD0EDE6EDE6ADE6AF1EC7C
:1047600054F03F0EDE6E860EDE6E0A0EDE6EF1EC4B
:1047700054F0BBC10BF0BCC10CF00BC0DEFF0CC091
:10478000DEFFB9C10BF0BAC10CF00BC0DEFF0CC0EC
:10479000DEFF010EDE6EDE6AB5EC45F0BBC30BF04A
:1047A000BCC30CF00BC0DEFF0CC0DEFFB9C30BF0C6
:1047B000BAC30CF00BC0DEFF0CC0DEFFDE6A010ED8
:1047C000DE6EB5EC45F080937DEF1FF008EF32F020
:1047D0001F0E815DD8A44EEF24F012EC4AF0010EBA
:1047E0008C5DD8A4F8EF23F056EF15F00EEF24F00F
:1047F000020E8C5DD8A404EF24F0CDEC69F0808328
:1048000015EF4FF00EEF24F0030E8C5DD8A40EEFE1
:1048100024F0CDEC69F0808315EF4FF0050E8C5D30
:10482000D8A41CEF24F082C02EF981C082F02EC9DA
:1048300081F080837DEF1FF0D89680A3D886D8B60C
:1048400030EF24F0CD0EDE6EDE6ADE6AF1EC54F05D
:10485000CF0EDE6E900EDE6E080EDE6EF1EC54F0C2
:10486000BBC10BF0BCC10CF00BC0DEFF0CC0DEFF07
:10487000B9C10BF0BAC10CF00BC0DEFF0CC0DEFFFB
:10488000010EDE6EDE6AB5EC45F0020EDE6EB9ECAE
:1048900062F080937DEF1FF008EF32F0200E815D13
:1048A000D8A4B4EF24F012EC4AF0010E8C5DD8A429
:1048B0005EEF24F056EF15F074EF24F0020E8C5DDD
:1048C000D8A46AEF24F0CDEC69F0808315EF4FF0A7
:1048D00074EF24F0030E8C5DD8A474EF24F0CDECBB
:1048E00069F0808315EF4FF0050E8C5DD8A482EF40
:1048F00024F082C02EF981C082F02EC981F080831D
:104900007DEF1FF0D89680A3D886D8B696EF24F016
:10491000CD0EDE6EDE6ADE6AF1EC54F0D30EDE6E92
:104920008E0EDE6E090EDE6EF1EC54F0BBC10BF0A4
:10493000BCC10CF00BC0DEFF0CC0DEFFB9C10BF038
:10494000BAC10CF00BC0DEFF0CC0DEFF010EDE6E44
:10495000DE6AB5EC45F0010EDE6EB9EC62F08093D4
:104960007DEF1FF008EF32F0210E815DD8A41AEF21
:1049700025F012EC4AF0010E8C5DD8A4C4EF24F0AF
:1049800056EF15F0DAEF24F0020E8C5DD8A4D0EFCC
:1049900024F0CDEC69F0808315EF4FF0DAEF24F0CE
:1049A000030E8C5DD8A4DAEF24F0CDEC69F080839F
:1049B00015EF4FF0050E8C5DD8A4E8EF24F082C00F
:1049C0002EF981C082F02EC981F080837DEF1FF027
:1049D000D89680A3D886D8B6FCEF24F0CD0EDE6E34
:1049E000DE6ADE6AF1EC54F03F0EDE6E860EDE6E9D
:1049F0000A0EDE6EF1EC54F0BBC10BF0BCC10CF042
:104A00000BC0DEFF0CC0DEFFB9C10BF0BAC10CF069
:104A10000BC0DEFF0CC0DEFF010EDE6EDE6AB5EC01
:104A200045F0030EDE6EB9EC62F080937DEF1FF06F
:104A300008EF32F0220E815DD8A48AEF25F012EC47
:104A40004AF0010E8C5DD8A42AEF25F056EF15F040
:104A50004CEF25F0020E8C5DD8A436EF25F0CDEC9E
:104A600069F0808315EF4FF04CEF25F0030E8C5D5D
:104A7000D8A442EF25F0CDEC69F0808315EF4FF01C
:104A80004CEF25F0040E8C5DD8A44CEF25F080810E
:104A9000B9C37EF0BAC37FF0050E8C5DD8A45AEF7F
:104AA00025F082C02EF981C082F02EC981F080836A
:104AB0007DEF1FF0D89680A3D886D8B66EEF25F08C
:104AC000CD0EDE6EDE6ADE6AF1EC54F0490EDE6E6B
:104AD000640EDE6E0E0EDE6EF1EC54F0BBC10BF018
:104AE000BCC10CF00BC0DEFF0CC0DEFFB9C10BF087
:104AF000BAC10CF00BC0DEFF0CC0DEFF010EDE6E93
:104B0000DE6AB5EC45F095EC43F080937DEF1FF045
:104B100008EF32F00D0E815DD8A4D6EF25F012EC2F
:104B20004AF0010E8C5DD8A498EF25F056EF15F0F1
:104B3000050E8C5DD8A4A6EF25F082C02EF981C0A9
:104B400082F02EC981F080837DEF1FF0D89680A37C
:104B5000D886D8B6BCEF25F0230EDE6E0E0EDE6EC4
:104B6000010EDE6EF1EC54F03D0EDE6E860EDE6E52
:104B7000060EDE6EF1EC54F0BBC30BF0BCC30CF0C0
:104B80000BC0DEFF0CC0DEFFB9C30BF0BAC30CF0E4
:104B90000BC0DEFF0CC0DEFFDE6A010EDE6EB5EC80
:104BA00045F080937DEF1FF008EF32F0270E815D16
:104BB000D8A427EF26F012EC4AF0010E8C5DD8A4A1
:104BC000E4EF25F056EF15F0050E8C5DD8A4F2EF5A
:104BD00025F082C02EF981C082F02EC981F0808339
:104BE0007DEF1FF0D89680A3D886D8B608EF26F0C0
:104BF0003D0EDE6E860EDE6E010EDE6EF1EC54F0C2
:104C00003F0EDE6E860EDE6E0A0EDE6EF1EC54F0A6
:104C1000BBC30BF0BCC30CF00BC0DEFF0CC0DEFF4F
:104C2000B9C30BF0BAC30CF00BC0DEFF0CC0DEFF43
:104C3000010EDE6E010EDE6EB5EC45F0030EDE6E8B
:104C4000B9EC62F080937DEF1FF008EF32F0280E90
:104C5000815DD8A478EF26F012EC4AF0010E8C5D4D
:104C6000D8A435EF26F056EF15F0050E8C5DD8A4CC
:104C700043EF26F082C02EF981C082F02EC981F068
:104C800080837DEF1FF0D89680A3D886D8B659EFE1
:104C900026F03D0EDE6E860EDE6E010EDE6EF1EC4F
:104CA00054F0D30EDE6E8E0EDE6E090EDE6EF1EC6B
:104CB00054F0BBC30BF0BCC30CF00BC0DEFF0CC048
:104CC000DEFFB9C30BF0BAC30CF00BC0DEFF0CC0A3
:104CD000DEFF010EDE6E010EDE6EB5EC45F0010E5C
:104CE000DE6EB9EC62F080937DEF1FF008EF32F0DA
:104CF000290E815DD8A4E1EF26F012EC4AF0010EF6
:104D00008C5DD8A488EF26F056EF15F09EEF26F0C4
:104D1000020E8C5DD8A494EF26F0CDEC69F0808370
:104D200015EF4FF09EEF26F0030E8C5DD8A49EEF9A
:104D300026F0CDEC69F0808315EF4FF0050E8C5D09
:104D4000D8A4ACEF26F082C02EF981C082F02EC923
:104D500081F080837DEF1FF0D89680A3D886D8B6E7
:104D6000C2EF26F03D0EDE6E860EDE6E010EDE6EAA
:104D7000F1EC54F0CF0EDE6E900EDE6E080EDE6E9D
:104D8000F1EC54F0BBC30BF0BCC30CF00BC0DEFF66
:104D90000CC0DEFFB9C30BF0BAC30CF00BC0DEFFD2
:104DA0000CC0DEFF010EDE6E010EDE6EB5EC45F0CE
:104DB000020EDE6EB9EC62F080937DEF1FF008EF1B
:104DC00032F02A0E815DD8A43AEF27F012EC4AF0B7
:104DD000010E8C5DD8A4EFEF26F056EF15F0040E0F
:104DE0008C5DD8A4F9EF26F08081B9C37EF0BAC3F8
:104DF0007FF0050E8C5DD8A407EF27F082C02EF956
:104E000081C082F02EC981F080837DEF1FF0D8969B
:104E100080A3D886D8B61DEF27F03D0EDE6E860E35
:104E2000DE6E010EDE6EF1EC54F0490EDE6E640EA5
:104E3000DE6E0E0EDE6EF1EC54F0BBC30BF0BCC3A5
:104E40000CF00BC0DEFF0CC0DEFFB9C30BF0BAC321
:104E50000CF00BC0DEFF0CC0DEFF010EDE6E010E9B
:104E6000DE6EB5EC45F095EC43F080937DEF1FF0DE
:104E700008EF32F0330E815DD8A43FEF2BF012EC37
:104E80004AF0010E8C5DD8A448EF27F056EF15F0DC
:104E9000020E8C5DD8A454EF27F080839CEC69F05F
:104EA00097EC4EF09CEC69F0030E8C5DD8A460EF9B
:104EB00027F080839CEC69F0D6EC4EF09CEC69F016
:104EC000D89680A3D886D8B69CEF27F0D89680BB1A
:104ED000D886D8B676EF27F0CDEC69F0D4EC43F065
:104EE000A66BA56BA86BA76B9CEF27F0890EDE6EF7
:104EF000DE6ADE6AF1EC54F08A0EDE6E0F0EDE6EB4
:104F0000030EDE6EF1EC54F0D70EDE6E840EDE6E14
:104F1000020EDE6EF1EC54F0D90EDE6E840EDE6E03
:104F2000060EDE6EF1EC54F01A0EDE6E790EDE6EB9
:104F3000040EDE6EF1EC54F095C0DEFF96C0DEFF8D
:104F400097C0DEFF98C0DEFF99C0DEFF9AC0DEFF8B
:104F50009BC0DEFF9CC0DEFF9DC0DEFF9EC0DEFF6B
:104F60009FC0DEFFA0C0DEFFA1C0DEFFA2C0DEFF4B
:104F7000A3C0DEFFA4C0DEFF8DC0DEFF8EC0DEFF5B
:104F80008FC0DEFF90C0DEFF91C0DEFF92C0DEFF6B
:104F900093C0DEFF94C0DEFFD6EC0BF018EEC0F03D
:104FA00091EC02F0CA51C911C811C711D8B4F4EF7D
:104FB00027F00801C0510001C75D09011A6F0801FF
:104FC000C1510001C85909011B6F0801C2510001FC
:104FD000C95909011C6F0801C3510001CA590901CF
:104FE0001D6F0001F9EF27F009011D6B1C6B1B6B96
:104FF0001A6B0001C3C8CAF0C2C8C9F0C1C8C8F062
:10500000C0C8C7F0BAC01FF9B9C01EF9C6C021F99F
:10501000C5C020F91FC91AF01EC919F0020EBCEC58
:1050200001F00B6E030E0B5CD8A429EF28F021C908
:105030001AF020C919F0020EBCEC01F00B6E0B52F5
:10504000D8A428EF28F0680E09012027010E21239B
:1050500000011FC91AF01EC919F0020EBCEC01F0C4
:105060000B6E0B52D8A448EF28F021C91AF020C9C2
:1050700019F0020EBCEC01F00B6E030E0B5CD8A411
:1050800047EF28F0680E09011E27010E1F230001BB
:1050900009011E51205D1F5121590001D8B058EF60
:1050A00028F0090120511E5D226F21511F59236FE5
:1050B0000001090120511E5D21511F590001D8B086
:1050C00069EF28F009011E51205D226F1F512159FF
:1050D000236F0001A651640DF3CF29F9A551640D8A
:1050E000F3CF28F9F450090129270001A851640DD4
:1050F000F3CF2BF9A751640DF3CF2AF9F45009012E
:105100002B270001C051640DF3CF2BF0F4CF2CF00E
:10511000D8902C3009012D6F2B302C6F0001BF531C
:10512000D8A4ADEF28F009012D510A0DF3CF2CF0D2
:105130002C510A0DF3CF2BF0F4502C262CC01AF072
:105140002BC019F01E6A210E1D6E32EC02F02C6F7E
:105150001AC02DF90001D7EF28F0010EBF5DD8A4C9
:10516000B4EF28F0D7EF28F0020EBF5DD8A4BFEF50
:1051700028F009012D6B2C6B0001D6EF28F00901F6
:105180002D510A0DF3CF2CF02C510A0DF3CF2BF03B
:10519000F4502C262CC01AF02BC019F01E6A210ED8
:1051A0001D6E32EC02F02C6F1AC02DF90001D8965A
:1051B00009011DAFD8860001D8B629EF29F00901F1
:1051C00023530001D8A428EF29F0B40E0901225D71
:1051D0000001D8B028EF29F009012C510801C025A1
:1051E0000901246F2D510801C1210901256F000E0D
:1051F0000801C2210901266F000E0801C32109011F
:10520000276F2851245F2951255B000E265B000E75
:10521000275B2A5124272B512523000E26232723E1
:105220001A51245F1B51255B1C51265B1D51275BC6
:1052300027C91CF026C91BF025C91AF0245179ECA6
:1052400002F0246F1AC025F91BC026F91CC027F9EB
:105250000001D89609011DBFD8860001D8B697EF86
:1052600029F009011A511B111C111D110001D8B49C
:1052700097EF29F0D89609011DBFD8860001D8B64E
:1052800097EF29F009011B511C111D1106E1010EB8
:105290001A5D0001D8A097EF29F0090123530001FE
:1052A000D8A496EF29F0B40E0901225D0001D8B010
:1052B00096EF29F009012C510801C05D0901246F06
:1052C0002D510801C1590901256F000E0801C2596D
:1052D0000901266F000E0801C3590901276F2851E3
:1052E000242729512523000E262327232A51245F12
:1052F0002B51255B000E265B000E275B1A51245FA5
:105300001B51255B1C51265B1D51275B27C91CF0D7
:1053100026C91BF025C91AF0245179EC02F0246F3C
:105320001AC025F91BC026F91CC027F90001D89620
:1053300009011DAFD8860001D8B6E9EF29F00901AF
:1053400023530001D8A4ACEF29F0B50E0901225D6A
:105350000001D8A0E8EF29F009012C510801C0256F
:105360000901246F2D510801C1210901256F000E8B
:105370000801C2210901266F000E0801C32109019D
:10538000276F2851242729512523000E2623272360
:105390002A51245F2B51255B000E265B000E275BF4
:1053A0001A51245F1B51255B1C51265B1D51275B45
:1053B00027C91CF026C91BF025C91AF0245179EC25
:1053C00002F0246F1AC025F91BC026F91CC027F96A
:1053D0000001D89609011DBFD8860001D8B657EF45
:1053E0002AF009011A511B111C111D110001D8B41A
:1053F00057EF2AF0D89609011DBFD8860001D8B60C
:1054000057EF2AF009011B511C111D1106E1010E75
:105410001A5D0001D8A057EF2AF0090123530001BB
:10542000D8A41AEF2AF0B50E0901225D0001D8A018
:1054300056EF2AF009012C510801C05D0901246FC3
:105440002D510801C1590901256F000E0801C259EB
:105450000901266F000E0801C3590901276F285161
:10546000245F2951255B000E265B000E275B2A5125
:1054700024272B512523000E262327231A51245F8E
:105480001B51255B1C51265B1D51275B27C91CF056
:1054900026C91BF025C91AF0245179EC02F0246FBB
:1054A0001AC025F91BC026F91CC027F90001080104
:1054B000C66BC86BC96BCA6B27C91CF026C91BF029
:1054C00025C91AF024C919F0040EC6EC01F0C66F04
:1054D00027C91CF026C91BF025C91AF024C919F0E8
:1054E000030EC6EC01F0C86F27C91CF026C91BF0DB
:1054F00025C91AF024C919F0020EC6EC01F0C96FD3
:1055000027C91CF026C91BF025C91AF024C919F0B7
:10551000010EC6EC01F0CA6F27C91CF026C91BF0AA
:1055200025C91AF024C919F0000EC6EC01F0CB6FA2
:10553000C6530001D8B4E0EF2AF00801C7530001B8
:10554000D8A4A6EF2AF09CEC69F080832C6AC6C828
:105550002BF02C50640DF3CF2CF02B50640DF3CFB7
:105560002BF0F4502C26306AC8C82FF030500A0DAA
:10557000F3CF30F02F500A0DF3CF2FF0F450302638
:105580002F502B2630502C220801C9512B24C46FD8
:10559000000E2C20C56FBBC30BF0BCC30CF00BC0BE
:1055A000DEFF0CC0DEFFC4C8DEFFC5C8DEFFDE6A5A
:1055B000010EDE6E0001B5EC45F0809338EF2BF064
:1055C0000801C7530001D8B4E9EF2AF09CEC69F058
:1055D00080832C6AC8C82BF02CC028F02B50276E73
:1055E000E80DF3CF2BF0F4CF2CF02850E80DF3505A
:1055F0002C262750030DF3502C26306AC9C82FF0F3
:105600003050640DF3CF30F02F50640DF3CF2FF0F6
:10561000F45030262F502B2630502C22306ACAC826
:105620002FF030500A0DF3CF30F02F500A0DF3CF8A
:105630002FF0F45030262F502B2630502C2208010A
:10564000CB512B24C46F000E2C20C56FBBC10BF0B7
:10565000BCC10CF00BC0DEFF0CC0DEFFC4C8DEFF17
:10566000C5C8DEFFDE6ADE6A0001B5EC45F0809356
:10567000C6C8C7F880937DEF1FF008EF32F0340EF4
:10568000815DD8A451EF2BF012EC4AF0010E8C5D35
:10569000D8A44DEF2BF056EF15F0ADEF50F008EF1A
:1056A00032F0350E815DD8A45EEF2DF012EC4AF099
:1056B000010E8C5DD8A461EF2BF056EF15F0B4EF1E
:1056C0002BF0020E8C5DD8A491EF2BF0B9C331F909
:1056D000BAC332F9CDEC69F00901356B0001150E42
:1056E0000901355D0001D8B08DEF2BF01CEC6DF099
:1056F000640E82EC01F05B0EDE6E360EDE6E080E7E
:10570000DE6EF1EC54F023EC6DF0640E82EC01F0EF
:105710000901352B0001D8A4E1D7CDEC69F0B4EF35
:105720002BF0030E8C5DD8A4A8EF2BF009013251A9
:10573000010A680ED8B431190001D8B4A6EF2BF0D5
:10574000B9C333F9BAC334F9CDEC69F0B4EF2BF037
:10575000040E8C5DD8A4AFEF2BF0B4EF2BF0050E48
:105760008C5DD8A4B4EF2BF0D89680A3D886D8B699
:10577000C7EF2BF0010E0901326F680E316F010E79
:10578000346F680E336F010E376F680E366F00018D
:105790003F0EDE6E860EDE6E0A0EDE6EF1EC54F00B
:1057A0008083BBC30BF0BCC30CF00BC0DEFF0CC08E
:1057B000DEFFB9C30BF0BAC30CF00BC0DEFF0CC0A8
:1057C000DEFFDE6A010EDE6EB5EC45F08093090166
:1057D0003251010A680ED8B431190001D8A42AEF59
:1057E0002CF01FEC09F019EE31F0A2EC02F00901E7
:1057F0003251010A680ED8B431190001D8B42AEF29
:105800002CF0B9C331F9BAC332F9CDEC69F0090112
:10581000356B0001150E0901355D0001D8B028EF88
:105820002CF01CEC6DF0640E82EC01F05B0EDE6E71
:10583000360EDE6E080EDE6EF1EC54F023EC6DF0E9
:10584000640E82EC01F00901352B0001D8A4E1D7E8
:10585000CDEC69F009013251010A680ED8B4311952
:105860000001D8B4C9EF2CF009013451010A680EC7
:10587000D8B433190001D8A4C9EF2CF01FEC09F0FB
:1058800019EE33F0A2EC02F009013451010A680E5E
:10589000D8B433190001D8B4C9EF2CF0B9C333F927
:1058A000BAC334F932C91AF031C919F0020EBCEC8E
:1058B00001F00B6E030E0B5CD8A471EF2CF034C911
:1058C0001AF033C919F0020EBCEC01F00B6E0B524A
:1058D000D8A470EF2CF0680E09013327010E342391
:1058E000000132C91AF031C919F0020EBCEC01F006
:1058F0000B6E0B52D8A490EF2CF034C91AF033C9B8
:1059000019F0020EBCEC01F00B6E030E0B5CD8A478
:105910008FEF2CF0680E09013127010E32230001B0
:1059200009013151335D325134590001D8B0B2EF21
:105930002CF009013351315D0B6E345132590C6E2C
:105940000C520001D8A4AFEF2CF0280E0B5CD8B09D
:10595000AFEF2CF0010E0901346F680E336F0001B8
:10596000C9EF2CF009013151335D0B6E32513459BE
:105970000C6E0C520001D8A4C8EF2CF0280E0B5C62
:10598000D8B0C8EF2CF0010E0901346F680E336FE8
:10599000000109013251010A680ED8B43119000121
:1059A000D8B430EF2DF009013451010A680ED8B493
:1059B00033190001D8B430EF2DF009013151335DB6
:1059C000325134590001D8B00CEF2DF00901335198
:1059D000315D366F34513259376FD89037333633A3
:1059E0003351362734513723010E375D0001D8A0DB
:1059F00009EF2DF0D8A404EF2DF0680E0901365DF3
:105A00000001D8A009EF2DF0680E0901365F010EE4
:105A1000375B000130EF2DF009013151335D366FF6
:105A200032513459376FD8903733363331513627A6
:105A300032513723010E375D0001D8A02FEF2DF032
:105A4000D8A42AEF2DF0680E0901365D0001D8A018
:105A50002FEF2DF0680E0901365F010E375B000154
:105A600009013751010A680ED8B436190001D8B4BB
:105A70005AEF2DF0D50EDE6E860EDE6E010EDE6E56
:105A8000F1EC54F08083BBC30BF0BCC30CF00BC033
:105A9000DEFF0CC0DEFF36C9DEFF37C9DEFF010EB8
:105AA000DE6E010EDE6EB5EC45F0809337C98BF0EB
:105AB00036C98AF07DEF1FF008EF32F0360E815DB7
:105AC000D8A496EF2DF012EC4AF0180EDE6EDE6AC6
:105AD000DE6AF1EC54F0D70EDE6E840EDE6E030E3D
:105AE000DE6EF1EC54F0D90EDE6E840EDE6E070E23
:105AF000DE6EF1EC54F01C0EDE6E7A0EDE6E050EDC
:105B0000DE6EF1EC54F0010E8C5DD8A48AEF2DF01E
:105B100056EF15F0D89680A3D886D8B692EF2DF020
:105B2000C2EC48F02AEF49F008EF32F0370E815D01
:105B3000D8A4A8EF2DF012EC4AF0010E8C5DD8A489
:105B4000A4EF2DF056EF15F056EF52F008EF32F0BB
:105B50003D0E815DD8A444EF31F0F30EDE6E0C0EE5
:105B6000DE6EDE6AF1EC54F0F90EDE6E160EDE6EBD
:105B7000060EDE6EF1EC54F0C80E82EC01F012EC71
:105B80004AF0010E8C5DD8A4C8EF2DF056EF15F049
:105B9000820E026E800E096E2A6A540E296E066805
:105BA00005687CEC00F0D8A0F3D70801CC6F640E38
:105BB000CC5D0001D8A42BEF2EF00801D06BCE6B8A
:105BC000CD6B00010801CE530001D8A419EF2EF0CF
:105BD000640E0801CD5D0001D8B019EF2EF0090167
:105BE00038512DEC01F00801CE51100DF3CF2CF0FF
:105BF000CD51100DF3CF2BF0F4502C262B4A2C2A2C
:105C00002C502DEC01F02B502DEC01F012EC01F09A
:105C1000CF6FDE0ECF5D0001D8A411EF2EF008018A
:105C2000D02B00010801CD2BD8B4CE2B0001D8A475
:105C3000C8D7820E026E400E096E2A6A540E296E73
:105C4000066A056A200E016E0801D051BEEC00F014
:105C5000000140EF31F0650E0801CC5D0001D8A4D1
:105C6000AAEF2EF00801D06BCE6BCD6B00010801BE
:105C7000CE530001D8A46EEF2EF0640E0801CD5D66
:105C80000001D8B06EEF2EF0090138512DEC01F073
:105C90000801CE51100DF3CF2CF0CD51100DF3CFE4
:105CA0002BF0F4502C262B4A2C2A2C502DEC01F0F2
:105CB0002B502DEC01F012EC01F0CF6FDE0ECF5D1A
:105CC0000001D8A466EF2EF00801D02B00010801D6
:105CD000CD2BD8B4CE2B0001D8A4C8D70801D05101
:105CE000100DF3CF2BF0F4CF2CF02B040B6E000E25
:105CF0002C580C6ECE6BCD6B00010801CD510B5CA6
:105D0000CE510C580001D8A0A8EF2EF0090138514F
:105D10002DEC01F00801CE512DEC01F0CD512DEC10
:105D200001F012EC01F0CF6F820E026E400E096E90
:105D30002A6A540E296E066A056A200E016ECF513A
:105D4000BEEC00F0CD2BD8B4CE2B0001D8A4D4D714
:105D500040EF31F0660E0801CC5D0001D8A4B9EF28
:105D60002EF0CDEC69F00A0E816F56EF15F040EF82
:105D700031F0670E0801CC5D0001D8A41EEF2FF0B2
:105D80000801CE6BCD6B00010801CD4BCE2BCE535D
:105D90000001D8A4D3EF2EF00B0E0801CD5D000159
:105DA000D8A0D4EF2EF0F4D6820E026E800E096ECB
:105DB0002A6A540E296E130E066E880E056E7CEC50
:105DC00000F0D8A0E0D70801CC6FCCC8DEFF0001FE
:105DD00033EC42F0FF0EDB50DD520801BA87E8A039
:105DE000BA97820E026E400E096E2A6A540E296E10
:105DF000066A056A200E016E7B0EBEEC00F0820E74
:105E0000026E400E096E2A6A540E296E066A056AF1
:105E1000200E016E7B0EBEEC00F0820E026E400E74
:105E2000096E2A6A540E296E066A056A200E016EF2
:105E30007B0EBEEC00F0000140EF31F0680E08016F
:105E4000CC5D0001D8A41FEF30F0820E026E800EF0
:105E5000096E2A6A540E296E130E066E880E056EA0
:105E60007CEC00F0D8A094D60801D46F820E026EAC
:105E7000800E096E2A6A540E296E130E066E880E65
:105E8000056E7CEC00F00001D8A082D60801D36F2B
:105E9000820E026E800E096E2A6A540E296E130E4F
:105EA000066E880E056E7CEC00F00001D8A070D65E
:105EB0000801D56F820E026E800E096E2A6A540E9A
:105EC000296E130E066E880E056E7CEC00F0000144
:105ED000D8A05ED60801D66F820E026E800E096EC3
:105EE0002A6A540E296E130E066E880E056E7CEC1F
:105EF00000F00001D8A04CD60801D76F820E026EC8
:105F0000800E096E2A6A540E296E130E066E880ED4
:105F1000056E7CEC00F00001D8A03AD60801D86FDD
:105F2000820E026E800E096E2A6A540E296E130EBE
:105F3000066E880E056E7CEC00F00001D8A028D615
:105F40000801D96F820E026E800E096E2A6A540E05
:105F5000296E130E066E880E056E7CEC00F00001B3
:105F6000D8A016D6BF6F820E026E800E096E2A6A06
:105F7000540E296E130E066E880E056E7CEC00F032
:105F8000D8A006D6C06FAA6A460EA96E0801D451E1
:105F900074EC01F0AA6A4C0EA96ED35174EC01F0B6
:105FA000AA6A470EA96ED55174EC01F0AA6A480E90
:105FB000A96ED65174EC01F0AA6A490EA96ED751A8
:105FC00074EC01F0AA6A4A0EA96ED85174EC01F083
:105FD000AA6A4B0EA96ED95174EC01F0AA6A4D0E53
:105FE000A96E0001BF5174EC01F0AA6A4E0EA96EB1
:105FF000C05174EC01F0820E026E400E096E2A6AE6
:10600000540E296E066A056A200E016EFF0EBEEC64
:1060100000F0010E0801D65D0001D8A415EF30F0A4
:10602000BD6BD5C8BCF01CEF30F00801D5513C0D5C
:10603000F3CFBCF0F4CFBDF0000140EF31F0690EBA
:106040000801CC5D0001D8A452EF30F0820E026E40
:10605000400E096E2A6A540E296E066A056A200EE1
:10606000016E000EBEEC00F0820E026E400E096E54
:106070002A6A540E296E066A056A200E016E020E07
:10608000BEEC00F0820E026E400E096E2A6A540EBB
:10609000296E066A056A200E016E000EBEEC00F045
:1060A00040EF31F06A0E0801CC5D0001D8A4FFEF8B
:1060B00030F0460E6BEC01F00801D46F820E026ED8
:1060C000400E096E2A6A540E296E066A056A200E71
:1060D000016ED451BEEC00F04C0E6BEC01F0D36FAE
:1060E000820E026E400E096E2A6A540E296E066AEE
:1060F000056A200E016ED351BEEC00F0470E6BEC2A
:1061000001F0D56F820E026E400E096E2A6A540E9F
:10611000296E066A056A200E016ED551BEEC00F0AC
:10612000480E6BEC01F0D66F820E026E400E096EC7
:106130002A6A540E296E066A056A200E016ED6512F
:10614000BEEC00F0490E6BEC01F0D76F820E026ED0
:10615000400E096E2A6A540E296E066A056A200EE0
:10616000016ED751BEEC00F04A0E6BEC01F0D86F17
:10617000820E026E400E096E2A6A540E296E066A5D
:10618000056A200E016ED851BEEC00F04B0E6BEC90
:1061900001F0D96F820E026E400E096E2A6A540E0B
:1061A000296E066A056A200E016ED951BEEC00F018
:1061B0004D0E6BEC01F00001BF6F820E026E400EBF
:1061C000096E2A6A540E296E066A056A200E016E4F
:1061D000BF51BEEC00F04E0E6BEC01F0C06F820EB2
:1061E000026E400E096E2A6A540E296E066A056A0E
:1061F000200E016EC051BEEC00F040EF31F06B0E8E
:106200000801CC5D0001D8A418EF31F07BEC40F020
:10621000820E026E400E096E2A6A540E296E066ABC
:10622000056A200E016EFF0EBEEC00F040EF31F06B
:106230006C0E0801CC5D0001D8A437EF31F0820E5E
:10624000026E400E096E2A6A540E296E066A056AAD
:10625000200E016EFF0EBEEC00F0FA0EDE6E160E82
:10626000DE6E060EDE6EF1EC54F040EF31F06D0E96
:106270000801CC5D0001D8A440EF31F0D3EC40F030
:10628000C8EF2DF008EF32F03E0E815DD8A453EF39
:1062900031F0CDEC69F03DEC4CF00A0E816F56EF19
:1062A00015F008EF32F03F0E815DD8A462EF31F0B7
:1062B000CDEC69F065EC4DF00A0E816F56EF15F0EC
:1062C00008EF32F0400E815DD8A471EF31F0CDECD3
:1062D00069F0DFEC4AF00A0E816F56EF15F008EF17
:1062E00032F0410E815DD8A49CEF31F0BE2B020E3E
:1062F000BE5DD8A487EF31F0BE6BF70EDE6E370EB1
:10630000DE6E060EDE6EF1EC54F08FEF31F0F50E1E
:10631000DE6E370EDE6E060EDE6EF1EC54F0010E10
:106320001E6E2C0E83EC01F0CDEC69F00A0E816F2D
:1063300056EF15F008EF32F0420E815DD8A4C7EF9A
:1063400031F07B2B020E7B5DD8A4B2EF31F07B6B7A
:10635000F70EDE6E390EDE6E060EDE6EF1EC54F0D8
:10636000BAEF31F0F50EDE6E390EDE6E060EDE6E21
:10637000F1EC54F0010E1E6E2C0E83EC01F0CDEC0E
:1063800069F00A0E816F56EF15F008EF32F0430EF8
:10639000815DD8A4D6EF31F0CDEC69F098EC4FF0E8
:1063A0000A0E816F56EF15F008EF32F0440E815D52
:1063B000D8A401EF32F0852B020E855DD8A4ECEF56
:1063C00031F0856BF70EDE6E390EDE6E060EDE6E78
:1063D000F1EC54F0F4EF31F0F50EDE6E390EDE6EB6
:1063E000060EDE6EF1EC54F0010E1E6E2C0E83ECE8
:1063F00001F0CDEC69F00A0E816F56EF15F008EF51
:1064000032F0470E815DD8A408EF32F053EF50F020
:106410007DEF1FF00801BA9909013C6B0001D89685
:106420000801BAB9D8860001D8B62CEF32F000EED8
:106430003AF009013C51EB500B6E2C0E0B5C000145
:10644000D8A428EF32F00801BA8900012AEF32F00F
:1064500009013C2B0001E2D709013C2900EE3AF08A
:10646000EBCF0BF00BC040F9020E3C2500EE3AF0EA
:10647000EBCF0BF00BC041F9030E3C2500EE3AF0D8
:10648000EBCF0BF00BC042F9040E3C2500EE3AF0C6
:10649000EBCF0BF00BC043F9050E3C2500EE3AF0B4
:1064A000EBCF0BF00BC044F9060E3C2500EE3AF0A2
:1064B000EBCF0BF00BC045F9070E3C2500EE3AF090
:1064C000EBCF0BF00BC046F9080E3C2500EE3AF07E
:1064D000EBCF0BF00BC047F9090E3C2500EE3AF06C
:1064E000EBCF0BF00BC048F90A0E3C2500EE3AF05A
:1064F000EBCF0BF00BC049F90801BA9909013D6BCC
:1065000000010A0E09013D5D0001D8B0B3EF32F081
:1065100009EE40F009013D51EB500B6E2C0E0B5C67
:106520000001D8A49DEF32F0F36A09EE40F00901B2
:106530003D51F3CFEBFF0801BA890001D89608015D
:10654000BAA9D8860001D8B6ADEF32F0F36A09EEE9
:1065500040F009013D51F3CFEBFF000109013D2B54
:106560000001D8A4CDD70801BA9B09013E6B0001F8
:10657000D8960801BABBD8860001D8B604EF33F02C
:1065800009EE40F009013E51EB500B6E2E0E0B5CF4
:106590000001D8A400EF33F0060E09013E5D09EEBC
:1065A00040F0EB500101106F050E09013E5D09EE50
:1065B00040F0EB500101116F040E09013E5D09EE40
:1065C00040F0EB500101126F030E09013E5D09EE30
:1065D00040F0EB500101136F020E09013E5D09EE20
:1065E00040F0EB500101146F09013E0509EE40F047
:1065F000EB500101156F0801BA8B000102EF33F077
:1066000009013E2B0001B3D70801BA9909013C2BBF
:106610000001D8960801BAB9D8860001D8B626EF8D
:1066200033F000EE3AF009013C51EB500B6E2C0EAA
:106630000B5C0001D8A422EF33F00801BA890001F5
:1066400024EF33F009013C2B0001E2D709013C297A
:1066500000EE3AF0EB500B6E560E0B5C0001D8A426
:1066600034EF33F0E0EF5FF009013C2900EE3AF03F
:10667000EB500B6E410E0B5C0001D8B442EF33F0CF
:10668000E0EF5FF009013C2B0801BA990001D896B0
:106690000801BAB9D8860001D8B664EF33F000EE2D
:1066A0003AF009013C51EB500B6E2C0E0B5C0001D3
:1066B000D8A460EF33F00801BA89000162EF33F02B
:1066C00009013C2B0001E2D709013C2900EE3AF018
:1066D000EBCF0BF00BC04AF9020E3C2500EE3AF06E
:1066E000EBCF0BF00BC04BF9030E3C2500EE3AF05C
:1066F000EBCF0BF00BC04CF9040E3C2500EE3AF04A
:10670000EBCF0BF00BC04DF9050E3C2500EE3AF037
:10671000EBCF0BF00BC04EF9060E3C2500EE3AF025
:10672000EBCF0BF00BC04FF9070E3C2500EE3AF013
:10673000EBCF0BF00BC050F9080E3C2500EE3AF001
:10674000EBCF0BF00BC051F9090E3C2500EE3AF0EF
:10675000EBCF0BF00BC052F90A0E3C2500EE3AF0DD
:10676000EBCF0BF00BC053F90B0E3C2500EE3AF0CB
:10677000EBCF0BF00BC054F90801BA9909013D6B3E
:1067800000010B0E09013D5D0001D8B0F3EF33F0BD
:1067900009EE4AF009013D51EB500B6E2C0E0B5CDB
:1067A0000001D8A4DDEF33F0F36A09EE4AF00901E5
:1067B0003D51F3CFEBFF0801BA890001D8960801DB
:1067C000BAA9D8860001D8B6EDEF33F0F36A09EE26
:1067D0004AF009013D51F3CFEBFF000109013D2BC8
:1067E0000001D8A4CDD70801BA9B09013E6B000176
:1067F000D8960801BABBD8860001D8B653EF34F05A
:1068000009EE4AF009013E51EB500B6E2E0E0B5C67
:106810000001D8A44FEF34F0040E09013E5D09EEEB
:106820004AF0EB500101176F030E09013E5D09EEBE
:106830004AF0EB500101186F020E09013E5D09EEAE
:106840004AF0EB500101196F09013E0509EE4AF0CB
:10685000EB5001011A6F09013E2909EE4AF0EB5095
:1068600001011B6F020E09013E2509EE4AF0EB50B3
:1068700001011C6F030E09013E2509EE4AF0EB50A1
:1068800001011D6F040E09013E2509EE4AF0EB508F
:1068900001011E6F0801BA8B000151EF34F00901AC
:1068A0003E2B0001A4D71C6A1B6A1A6A19C119F091
:1068B000246A010E236E860E226EA00E216E49EC14
:1068C00002F01CC090F01BC08FF01AC08EF019C0EF
:1068D0008DF01C6A1B6A1A6A1AC119F0246A236AAD
:1068E000270E226E100E216E49EC02F01CC02EF015
:1068F0001BC02DF01AC02CF019C02BF02B508D2787
:106900002C508E232D508F232E5090231C6A1B6AEF
:106910001A6A1BC119F0246A236A030E226EE80E5C
:10692000216E49EC02F01CC02EF01BC02DF01AC0E5
:106930002CF019C02BF02B508D272C508E232D506E
:106940008F232E5090231C6A1B6A1A6A1CC119F0EF
:10695000246A236A226A640E216E49EC02F01CC08C
:106960002EF01BC02DF01AC02CF019C02BF02B50AC
:106970008D272C508E232D508F232E5090231C6A50
:106980001B6A1A6A1DC119F0246A236A226A0A0E58
:10699000216E49EC02F01CC02EF01BC02DF01AC075
:1069A0002CF019C02BF02B508D272C508E232D50FE
:1069B0008F232E50902301011E5100018D258D6FD4
:1069C000000E8E218E6F000E8F218F6F000E902192
:1069D000906F010117510A0DF3CF2BF0F4CF2CF07B
:1069E00018512B240001C16F09013C2B0801BA99F1
:1069F0000001D8960801BAB9D8860001D8B616EFBA
:106A000035F000EE3AF009013C51EB500B6E2C0EC4
:106A10000B5C0001D8A412EF35F00801BA8900011F
:106A200014EF35F009013C2B0001E2D709013C29A4
:106A300000EE3AF0EB5001011F6F09013C2B0801F9
:106A4000BA990001D8960801BAB9D8860001D8B61B
:106A50003FEF35F000EE3AF009013C51EB500B6E80
:106A60002C0E0B5C0001D8A43BEF35F00801BA896D
:106A700000013DEF35F009013C2B0001E2D709018F
:106A80003C2900EE3AF0EBCF0BF00BC055F9020EAB
:106A90003C2500EE3AF0EBCF0BF00BC056F9030E9D
:106AA0003C2500EE3AF0EBCF0BF00BC057F9040E8B
:106AB0003C2500EE3AF0EBCF0BF00BC058F9050E79
:106AC0003C2500EE3AF0EBCF0BF00BC059F9060E67
:106AD0003C2500EE3AF0EBCF0BF00BC05AF9070E55
:106AE0003C2500EE3AF0EBCF0BF00BC05BF9080E43
:106AF0003C2500EE3AF0EBCF0BF00BC05CF9090E31
:106B00003C2500EE3AF0EBCF0BF00BC05DF90A0E1E
:106B10003C2500EE3AF0EBCF0BF00BC05EF90B0E0C
:106B20003C2500EE3AF0EBCF0BF00BC05FF90C0EFA
:106B30003C2500EE3AF0EBCF0BF00BC060F90801FA
:106B4000BA9909013D6B00010B0E09013D5D000181
:106B5000D8B0D6EF35F009EE55F009013D51EB50B4
:106B60000B6E2C0E0B5C0001D8A4C0EF35F0F36A5D
:106B700009EE55F009013D51F3CFEBFF0801BA8949
:106B80000001D8960801BAA9D8860001D8B6D0EF7E
:106B900035F0F36A09EE55F009013D51F3CFEBFFF3
:106BA000000109013D2B0001D8A4CDD70801BA9BF3
:106BB00009013E6B0001D8960801BABBD8860001D6
:106BC000D8B63EEF36F009EE55F009013E51EB50D4
:106BD0000B6E2E0E0B5C0001D8A43AEF36F0050EBA
:106BE00009013E5D09EE55F0EB500101206F040EE6
:106BF00009013E5D09EE55F0EB500101216F030ED6
:106C000009013E5D09EE55F0EB500101226F020EC5
:106C100009013E5D09EE55F0EB500101236F0901BA
:106C20003E0509EE55F0EB500101246F09013E29A4
:106C300009EE55F0EB500101256F020E09013E25CA
:106C400009EE55F0EB500101266F030E09013E25B8
:106C500009EE55F0EB500101276F040E09013E25A6
:106C600009EE55F0EB500101286F0801BA8B0001C5
:106C70003CEF36F009013E2B00019CD71C6A1B6AD1
:106C80001A6A23C119F0246A010E236E860E226E41
:106C9000A00E216E49EC02F01CC094F01BC093F0D2
:106CA0001AC092F019C091F01C6A1B6A1A6A24C1BA
:106CB00019F0246A236A270E226E100E216E49EC09
:106CC00002F01CC02EF01BC02DF01AC02CF019C011
:106CD0002BF02B5091272C5092232D5093232E5084
:106CE00094231C6A1B6A1A6A25C119F0246A236A54
:106CF000030E226EE80E216E49EC02F01CC02EF04D
:106D00001BC02DF01AC02CF019C02BF02B5091276E
:106D10002C5092232D5093232E5094231C6A1B6ACF
:106D20001A6A26C119F0246A236A226A640E216E47
:106D300049EC02F01CC02EF01BC02DF01AC02CF044
:106D400019C02BF02B5091272C5092232D509323B8
:106D50002E5094231C6A1B6A1A6A27C119F0246AF0
:106D6000236A226A0A0E216E49EC02F01CC02EF042
:106D70001BC02DF01AC02CF019C02BF02B509127FE
:106D80002C5092232D5093232E50942301012851EF
:106D900000019125916F000E9221926F000E9321B8
:106DA000936F000E9421946F09013C2B0801BA994E
:106DB0000001D8960801BAB9D8860001D8B6F6EF16
:106DC00036F000EE3AF009013C51EB500B6E2C0E00
:106DD0000B5C0001D8A4F2EF36F00801BA8900017B
:106DE000F4EF36F009013C2B0001E2D709013C2900
:106DF00000EE3AF0EB500101296F09013C2B08012C
:106E0000BA990001D8960801BAB9D8860001D8B657
:106E10001FEF37F000EE3AF009013C51EB500B6EDA
:106E20002C0E0B5C0001D8A41BEF37F00801BA89C7
:106E300000011DEF37F009013C2B0001E2D70901E9
:106E40003C2900EE3AF0EBCF0BF00BC061F9020EDB
:106E50003C2500EE3AF0EBCF0BF00BC062F9030ECD
:106E60003C2500EE3AF0EBCF0BF00BC063F9040EBB
:106E70003C2500EE3AF0EBCF0BF00BC064F9050EA9
:106E80003C2500EE3AF0EBCF0BF00BC065F9060E97
:106E90003C2500EE3AF0EBCF0BF00BC066F9070E85
:106EA0003C2500EE3AF0EBCF0BF00BC067F9080180
:106EB000BA9909013D6B0001070E09013D5D000112
:106EC000D8B08EEF37F009EE61F009013D51EB507B
:106ED0000B6E2C0E0B5C0001D8A478EF37F0F36A30
:106EE00009EE61F009013D51F3CFEBFF0801BA89CA
:106EF0000001D8960801BAA9D8860001D8B688EF53
:106F000037F0F36A09EE61F009013D51F3CFEBFF71
:106F1000000109013D2B0001D8A4CDD70801BA9B7F
:106F200009013E6B0001D8960801BABBD886000162
:106F3000D8B6E8EF37F009EE61F009013E51EB50A9
:106F40000B6E2E0E0B5C0001D8A4E4EF37F0020E9E
:106F500009013E5D0001D8B0B3EF37F001012A6BA3
:106F60000001BBEF37F0020E09013E5D09EE61F052
:106F7000EB5001012A6F0001010E09013E5D000185
:106F8000D8B0C8EF37F001012B6B0001CFEF37F01D
:106F900009013E0509EE61F0EB5001012B6F000184
:106FA00009013E2909EE61F0EB5001012C6F020E40
:106FB00009013E2509EE61F0EB5001012D6F08013A
:106FC000BA8B0001E6EF37F009013E2B0001AAD78A
:106FD0000A0E01012A5D0001D8A0F1EF37F001018E
:106FE0002A6B00010A0E01012B5D0001D8A0FBEF06
:106FF00037F001012B6B00010A0E01012C5D00012D
:10700000D8A005EF38F001012C6B00010A0E010138
:107010002D5D0001D8A00FEF38F001012D6B0001AC
:107020002C6A2AC12BF02CC028F02B50276EE80DBB
:10703000F3CF2BF0F4CF2CF02850E80DF3502C2692
:107040002750030DF3502C26306A2BC12FF03050FF
:10705000640DF3CF30F02F50640DF3CF2FF0F450C8
:1070600030262F502B2630502C22306A2CC12FF086
:1070700030500A0DF3CF30F02F500A0DF3CF2FF020
:10708000F45030262F502B2630502C2201012D5148
:107090002B242E6F000E2C202F6F130E09013F6F33
:1070A000000109013F290B6E01EE65F0D8903F35D4
:1070B000E926000EEA22EECF0DF0EFCF0EF001EE42
:1070C00065F0D8900B34E926000EEA220DC0EEFFE1
:1070D0000EC0EFFF010E3F5F0001D8B0E1D72FC116
:1070E00066F12EC165F1B46BB36BB26BB16B090184
:1070F000716B0001090171510801D75D0001D8A031
:107100009BEF38F001EE65F0D89009017135E92662
:10711000000EEA22EECF0BF0EFCF0CF00B50000187
:10712000B1270C50B223000EB323B4230901712BF5
:107130000001D8A4DED72D6A2E6A0801D7292B6E4C
:10714000000E2C6A2C22B4C01CF0B3C01BF0B2C0DD
:107150001AF0B1C019F02EC024F02DC023F02CC0BD
:1071600022F02BC021F0D2EC01F01AC0B6F019C009
:10717000B5F07E0E09013F6F000109013F290B6E3A
:1071800002EEB9F0D8903F35E926000EEA22EECFA4
:107190000DF0EFCF0EF002EEB9F0D8900B34E926E7
:1071A000000EEA220DC0EEFF0EC0EFFF010E3F5FA2
:1071B0000001D8B0E1D7B6C0BAF2B5C0B9F2090142
:1071C0003C2B0801BA990001D8960801BAB9D886B3
:1071D0000001D8B601EF39F000EE3AF009013C5158
:1071E000EB500B6E2C0E0B5C0001D8A4FDEF38F0B9
:1071F0000801BA890001FFEF38F009013C2B0001BA
:10720000E2D709013C2900EE3AF0EBCF0BF00BC0BE
:1072100068F9020E3C2500EE3AF0EBCF0BF00BC004
:1072200069F9030E3C2500EE3AF0EBCF0BF00BC0F2
:107230006AF9040E3C2500EE3AF0EBCF0BF00BC0E0
:107240006BF9050E3C2500EE3AF0EBCF0BF00BC0CE
:107250006CF9060E3C2500EE3AF0EBCF0BF00BC0BC
:107260006DF9070E3C2500EE3AF0EBCF0BF00BC0AA
:107270006EF90801BA9909013D6B0001070E090179
:107280003D5D0001D8B070EF39F009EE68F00901FA
:107290003D51EB500B6E2C0E0B5C0001D8A45AEF45
:1072A00039F0F36A09EE68F009013D51F3CFEBFFC5
:1072B0000801BA890001D8960801BAA9D886000148
:1072C000D8B66AEF39F0F36A09EE68F009013D516A
:1072D000F3CFEBFF000109013D2B0001D8A4CDD76E
:1072E0000801BA9B09013E6B0001D8960801BABBA0
:1072F000D8860001D8B6D0EF39F009EE68F0090160
:107300003E51EB500B6E2E0E0B5C0001D8A4CCEF5F
:1073100039F0030E09013E5D0001D8B095EF39F058
:107320000101306B00019DEF39F0030E09013E5D54
:1073300009EE68F0EB500101306F0001020E090107
:107340003E5D0001D8B0AAEF39F00101316B0001B8
:10735000B2EF39F0020E09013E5D09EE68F0EB5024
:107360000101316F0001010E09013E5D0001D8B03D
:10737000BFEF39F00101326B0001C6EF39F00901AE
:107380003E0509EE68F0EB500101326F0001080183
:10739000BA8B0001CEEF39F009013E2B0001A4D7D2
:1073A000040E0101305D0001D8A0D9EF39F00101D0
:1073B000306B00010A0E0101315D0001D8A0E3EF3E
:1073C00039F00101316B00010A0E0101325D00014B
:1073D000D8A0EDEF39F00101326B00012C6A30C109
:1073E0002BF02C50640DF3CF2CF02B50640DF3CF09
:1073F0002BF0F4502C26306A31C12FF030500A0D9A
:10740000F3CF30F02F500A0DF3CF2FF0F450302689
:107410002F502B2630502C22010132512B24336F58
:10742000000E2C20346F0801D3530001D8A443EF81
:107430003AF0010134530001D8A427EF3AF00801D3
:10744000D4510101335D0001D8A030EF3AF00801BA
:10745000D4510101335F000E345B000140EF3AF07C
:10746000010133510801D45D0101336F341DD8B0DF
:10747000010F346F33516808336F010E3455346F88
:1074800000015FEF3AF00801D45101013327000EEB
:107490003423010E345D0001D8A05EEF3AF0D8A489
:1074A00059EF3AF0680E0101335D0001D8A05EEF9C
:1074B0003AF0680E0101335F010E345B0001130ED8
:1074C00009013F6F000109013F290B6E01EE8FF0AA
:1074D000D8903F35E926000EEA22EECF0DF0EFCF2F
:1074E0000EF001EE8FF0D8900B34E926000EEA2260
:1074F0000DC0EEFF0EC0EFFF010E3F5F0001D8B0E0
:10750000E1D734C190F133C18FF109019A6B9B6BC4
:10751000716B0001090171510801D75D0001D8A00C
:10752000DEEF3AF001EE8FF0D89009017135E926CF
:10753000000EEA22EECF0BF0EFCF0CF009EE72F066
:10754000D8907135E926000EEA220BC0EEFF0CC080
:10755000EFFF09EE72F0D8907135E926000EEA22AD
:10756000EECF19F0EFCF1AF0020EBCEC01F00B6E6B
:10757000030E0B5C0001D8A4C0EF3AF009019A2B6E
:10758000000109EE72F0D89009017135E926000E6C
:10759000EA22EECF19F0EFCF1AF0020EBCEC01F0A8
:1075A0000B6E0B520001D8A4D8EF3AF009019B2BC7
:1075B00000010901712B0001D8A4ABD709019A532E
:1075C0000001D8B444EF3BF009019B530001D8B44B
:1075D00044EF3BF009019A519B250B6E0C6A0C3667
:1075E0000801D7290F6E000E106A102210500C5C93
:1075F0000001D8A444EF3BF00F500B5CD8A444EF3B
:107600003BF00901716B0001090171510801D75D5F
:107610000001D8A044EF3BF009EE72F0D8900901C8
:107620007135E926000EEA22EECF19F0EFCF1AF0FD
:10763000020EBCEC01F00B6E0B520001D8A43EEF21
:107640003BF009EE72F0D89009017135E926000E81
:10765000EA22EECF0DF0EFCF0EF0680E0D240B6E88
:10766000010E0E200C6E09EE72F0D8907135E926ED
:10767000000EEA220BC0EEFF0CC0EFFF0001090173
:10768000712B0001D8A4BFD7B46BB36BB26BB16BD5
:107690000901716B0001090171510801D75D0001F9
:1076A000D8A06CEF3BF009EE72F0D890090171356B
:1076B000E926000EEA22EECF0BF0EFCF0CF00B50D4
:1076C0000001B1270C50B223000EB323B4230901EB
:1076D000712B0001D8A4DED72D6A2E6A0801D729A4
:1076E0002B6E000E2C6A2C22B4C01CF0B3C01BF011
:1076F000B2C01AF0B1C019F02EC024F02DC023F092
:107700002CC022F02BC021F0D2EC01F01AC0BAF04C
:1077100019C0B9F0010E0001BA5DD8A09CEF3BF092
:10772000D8A498EF3BF0680EB95DD8A09CEF3BF071
:10773000680EB95F010EBA5B7E0E09013F6F000152
:1077400009013F290B6E03EEB9F0D8903F35E926C9
:10775000000EEA22EECF0DF0EFCF0EF003EEB9F0FF
:10776000D8900B34E926000EEA220DC0EEFF0EC0C1
:10777000EFFF010E3F5F0001D8B0E1D7BAC0BAF306
:10778000B9C0B9F309013C2B0801BA990001D89698
:107790000801BAB9D8860001D8B6E4EF3BF000EE94
:1077A0003AF009013C51EB500B6E2C0E0B5C0001C2
:1077B000D8A4E0EF3BF00801BA890001E2EF3BF00A
:1077C00009013C2B0001E2D709013C2900EE3AF007
:1077D000EB500101356F020E09013C2500EE3AF035
:1077E000EB500101366F030E09013C2500EE3AF023
:1077F000EB500101376F040E09013C2500EE3AF011
:10780000EB500101386F050E09013C2500EE3AF0FE
:10781000EB500101396F060E09013C2500EE3AF0EC
:10782000EB5001013A6F00018953D8B424EF3CF0CA
:107830008B51010A900ED8B48A19D8A424EF3CF0D9
:10784000B9C38AF0BAC38BF08953D8B430EF3CF097
:10785000DCEC0AF019EE6FF0A2EC02F033EF3CF032
:107860000901706B6F6B0001130E09013F6F00017E
:1078700009013F290B6E01EE3BF0D8903F35E92618
:10788000000EEA22EECF0DF0EFCF0EF001EE3BF04E
:10789000D8900B34E926000EEA220DC0EEFF0EC090
:1078A000EFFF010E3F5F0001D8B0E1D770C93CF196
:1078B0006FC93BF1B46BB36BB26BB16B0901716B08
:1078C0000001090171510801D75D0001D8A082EFC4
:1078D0003CF001EE3BF0D89009017135E926000E2D
:1078E000EA22EECF0BF0EFCF0CF00B500001B127E6
:1078F0000C50B223000EB323B4230901712B0001F5
:10790000D8A4DED72D6A2E6A0801D7292B6E000E67
:107910002C6A2C22B4C01CF0B3C01BF0B2C01AF009
:10792000B1C019F02EC024F02DC023F02CC022F0DD
:107930002BC021F0D2EC01F01AC0B8F019C0B7F09A
:107940007E0E09013F6F000109013F290B6E01EE18
:10795000B9F0D8903F35E926000EEA22EECF0DF0BF
:10796000EFCF0EF001EEB9F0D8900B34E926000EFF
:10797000EA220DC0EEFF0EC0EFFF010E3F5F0001D7
:10798000D8B0E1D7B8C0BAF1B7C0B9F170C91AF030
:107990006FC919F0030EBCEC01F00401B96F70C996
:1079A0001AF06FC919F0020EBCEC01F0BA6F70C981
:1079B0001AF06FC919F0010EBCEC01F0BB6F70C971
:1079C0001AF06FC919F0000EBCEC01F0BC6F020E8A
:1079D0000001A95DD8A4FCEF3CF0D89680B3D8860E
:1079E000D8B6FCEF3CF0BB53D8A4FBEF3CF05CEC0A
:1079F00013F0BCC0BBF0BB0712000901A96BA86B58
:107A00009E6B9D6B0001060E09019E5D0001D8A0D2
:107A100014EF3DF0D8A432EF3DF0400E09019D5D1A
:107A20000001D8B032EF3DF0090138512DEC01F0E2
:107A30009E512DEC01F09D512DEC01F012EC01F066
:107A40009C6FDE0E9C5D0001D8A42BEF3DF09EC91B
:107A5000A9F99DC9A8F909019D2BD8B49E2B000155
:107A6000D8A4D0D70901A951A8110001D8A43DEF8D
:107A70003DF0FEEC3EF0FCEF3EF0090138512DECFC
:107A800001F0A8052B6E000EA9592C6E2C502DEC80
:107A900001F02B502DEC01F012EC01F09C6F9C2BAF
:107AA00039512DEC01F00F0EA8252B6E000EA921E7
:107AB0002C6E2C502DEC01F02B502DEC01F09C5134
:107AC0002BEC01F0050E82EC01F039512DEC01F0A8
:107AD000100EA8252B6E000EA9212C6E2C502DEC1B
:107AE00001F02B502DEC01F0DE0E2BEC01F0050E19
:107AF00082EC01F0010110510A0DF3CF2BF0F4CF0D
:107B00002CF011512B240901AF6F39512DEC01F0EC
:107B1000110EA8252B6E000EA9212C6E2C502DECD9
:107B200001F02B502DEC01F0AF512BEC01F0050EC4
:107B300082EC01F0010112510A0DF3CF2BF0F4CFCA
:107B40002CF013512B240901AF6F39512DEC01F0AA
:107B5000120EA8252B6E000EA9212C6E2C502DEC98
:107B600001F02B502DEC01F0AF512BEC01F0050E84
:107B700082EC01F0010114510A0DF3CF2BF0F4CF88
:107B80002CF015512B240901AF6F39512DEC01F068
:107B9000130EA8252B6E000EA9212C6E2C502DEC57
:107BA00001F02B502DEC01F0AF512BEC01F0050E44
:107BB00082EC01F0010135510A0DF3CF2BF0F4CF27
:107BC0002CF036512B240901AF6F39512DEC01F007
:107BD000140EA8252B6E000EA9212C6E2C502DEC16
:107BE00001F02B502DEC01F0AF512BEC01F0050E04
:107BF00082EC01F0010137510A0DF3CF2BF0F4CFE5
:107C00002CF038512B240901AF6F39512DEC01F0C4
:107C1000150EA8252B6E000EA9212C6E2C502DECD4
:107C200001F02B502DEC01F0AF512BEC01F0050EC3
:107C300082EC01F0010139510A0DF3CF2BF0F4CFA2
:107C40002CF03A512B240901AF6F39512DEC01F082
:107C5000160EA8252B6E000EA9212C6E2C502DEC93
:107C600001F02B502DEC01F0AF512BEC01F0050E83
:107C700082EC01F038512DEC01F00B0EA8252B6E93
:107C8000000EA9212C6E2C502DEC01F02B502DEC68
:107C900001F012EC01F0AB6FABC9AEF038512DEC36
:107CA00001F00C0EA8252B6E000EA9212C6E2C5075
:107CB0002DEC01F02B502DEC01F012EC01F0AC6F2B
:107CC000ACC9ADF038512DEC01F00D0EA8252B6E8E
:107CD000000EA9212C6E2C502DEC01F02B502DEC18
:107CE00001F012EC01F0AD6FADC9ACF038512DECE4
:107CF00001F00E0EA8252B6E000EA9212C6E2C5023
:107D00002DEC01F02B502DEC01F012EC01F0AE6FD8
:107D1000AEC9ABF00001AB2B000EAC23AD23AE23FC
:107D2000AEC0ABF9ADC0ACF9ACC0ADF9ABC0AEF90B
:107D3000AB07000EAC5BAD5BAE5B1B0E0901A8256B
:107D40000001AF6F000E0901A9210001B06F090108
:107D500039512DEC01F0170EA8252B6E000EA9212C
:107D60002C6E2C502DEC01F02B502DEC01F0AB5172
:107D70002BEC01F0050E82EC01F039512DEC01F0F5
:107D8000180EA8252B6E000EA9212C6E2C502DEC60
:107D900001F02B502DEC01F0AC512BEC01F0050E55
:107DA00082EC01F039512DEC01F0190EA8252B6E53
:107DB000000EA9212C6E2C502DEC01F02B502DEC37
:107DC00001F0AD512BEC01F0050E82EC01F03951C0
:107DD0002DEC01F01A0EA8252B6E000EA9212C6E99
:107DE0002C502DEC01F02B502DEC01F0AE512BEC72
:107DF00001F0050E82EC01F000011200A30E090152
:107E0000B16FA20EB26FB46BB36BB2512DEC01F037
:107E1000B4512DEC01F0B3512DEC01F0010E2BEC1F
:107E200001F0050E82EC01F0B1512DEC01F0B451DE
:107E30002DEC01F0B3512DEC01F012EC01F0B56F17
:107E4000B2512DEC01F0010EB3252B6E000EB421C2
:107E50002C6E2C502DEC01F02B502DEC01F0DE0E91
:107E60002BEC01F0050E82EC01F0B1512DEC01F08C
:107E7000010EB3252B6E000EB4212C6E2C502DEC70
:107E800001F02B502DEC01F012EC01F0B56F010167
:107E900010510A0DF3CF2BF0F4CF2CF011512B24FD
:107EA0000901B66FB2512DEC01F0020EB3252B6E15
:107EB000000EB4212C6E2C502DEC01F02B502DEC2B
:107EC00001F0B6512BEC01F0050E82EC01F001013E
:107ED00012510A0DF3CF2BF0F4CF2CF013512B24B9
:107EE0000901B66FB2512DEC01F0030EB3252B6ED4
:107EF000000EB4212C6E2C502DEC01F02B502DECEB
:107F000001F0B6512BEC01F0050E82EC01F00101FD
:107F100014510A0DF3CF2BF0F4CF2CF015512B2474
:107F20000901B66FB2512DEC01F0040EB3252B6E92
:107F3000000EB4212C6E2C502DEC01F02B502DECAA
:107F400001F0B6512BEC01F0050E82EC01F00101BD
:107F500035510A0DF3CF2BF0F4CF2CF036512B24F2
:107F60000901B66FB2512DEC01F0050EB3252B6E51
:107F7000000EB4212C6E2C502DEC01F02B502DEC6A
:107F800001F0B6512BEC01F0050E82EC01F001017D
:107F900037510A0DF3CF2BF0F4CF2CF038512B24AE
:107FA0000901B66FB2512DEC01F0060EB3252B6E10
:107FB000000EB4212C6E2C502DEC01F02B502DEC2A
:107FC00001F0B6512BEC01F0050E82EC01F001013D
:107FD00039510A0DF3CF2BF0F4CF2CF03A512B246A
:107FE0000901B66FB2512DEC01F0070EB3252B6ECF
:107FF000000EB4212C6E2C502DEC01F02B502DECEA
:1080000001F0B6512BEC01F0050E82EC01F0A36BF0
:10801000A26B060EA16F400EA06FA3C9B6F9B251B4
:108020002DEC01F0080EB3252B6E000EB4212C6E42
:108030002C502DEC01F02B502DEC01F0B6512BEC17
:1080400001F0050E82EC01F0A2C9B6F9B2512DEC97
:1080500001F0090EB3252B6E000EB4212C6E2C50AE
:108060002DEC01F02B502DEC01F0B6512BEC01F072
:10807000050E82EC01F0A1C9B6F9B2512DEC01F068
:108080000A0EB3252B6E000EB4212C6E2C502DEC55
:1080900001F02B502DEC01F0B6512BEC01F0050E48
:1080A00082EC01F0A0C9B6F9B2512DEC01F00B0E33
:1080B000B3252B6E000EB4212C6E2C502DEC01F04C
:1080C0002B502DEC01F0B6512BEC01F0050E82EC9B
:1080D00001F00001AE6BAD6B060EAC6F3F0EAB6FE7
:1080E0000C0E0901B3250001AF6F000E0901B42188
:1080F0000001B06F12000901B86BB76B0001060EEA
:108100000901B85D0001D8A090EF40F0D8A4A6EF17
:1081100040F0410E0901B75D0001D8B0A6EF40F074
:10812000A20E2DEC01F00901B8512DEC01F0B75170
:108130002DEC01F0000E2BEC01F0050E82EC01F0AD
:10814000B72BD8B4B82B0001D8A4D8D71200090196
:10815000BB6BBA6B0001FF0E0901BB5D0001D8A02B
:10816000BCEF40F0D8A4D2EF40F0FF0E0901BA5D99
:108170000001D8B0D2EF40F0A20E2DEC01F00901C1
:10818000BB512DEC01F0BA512DEC01F0000E2BEC9F
:1081900001F0050E82EC01F0BA2BD8B4BB2B000124
:1081A000D8A4D8D712000901BE6BBD6B00017F0EA9
:1081B0000901BE5D0001D8A0E8EF40F0D8A429EF86
:1081C00041F0F00E0901BD5D0001D8B029EF41F08A
:1081D000820E026E800E096E2A6A540E296E130EEC
:1081E000066E880E056E7CEC00F0D8A0C8EF2DF06E
:1081F0000901BC6FA00E2DEC01F0BE512DEC01F079
:10820000BD512DEC01F0BC512BEC01F00A0E82ECBB
:1082100001F0A10E2DEC01F0BE512DEC01F0BD518D
:108220002DEC01F012EC01F0BF6F820E026E400ED9
:10823000096E2A6A540E296E066A056A200E016EBE
:10824000BF51BEEC00F0BD2BD8B4BE2B0001D8A4AA
:10825000ADD712000901C36BC76BC66BC56BC46B8E
:108260000001D8960901C7BFD8860001D8B64AEFE9
:1082700041F00901C7530001D8A432EF42F0FE0ECD
:108280000901C45DFF0EC559010EC6590001D8B0E1
:1082900032EF42F0D8960901C7BFD8860001D8B6A0
:1082A000B0EF41F00901C7530AE1C65108E1FF0EE2
:1082B000C45DFF0EC5590001D8A0B0EF41F009011F
:1082C000C429C16F000EC521C26FAB0E2DEC01F0A9
:1082D000C2512DEC01F0C1512DEC01F012EC01F076
:1082E000C06F820E026E400E096E2A6A540E296E0D
:1082F000066A056A200E016E2D0EBEEC00F0820E9D
:10830000026E400E096E2A6A540E296E066A056ACC
:10831000200E016E086AC2C922F0C1C921F024EC06
:1083200000F0820E026E400E096E2A6A540E296E0B
:10833000066A056A200E016E2C0EBEEC00F0820E5D
:10834000026E400E096E2A6A540E296E066A056A8C
:10835000200E016EC05121EC00F0000101EF42F04F
:10836000C5C9C2F9C4C9C1F9A30E2DEC01F00901B8
:10837000C2512DEC01F0C1512DEC01F012EC01F0D5
:10838000C06F820E026E400E096E2A6A540E296E6C
:10839000066A056A200E016E2E0EBEEC00F0820EFB
:1083A000026E400E096E2A6A540E296E066A056A2C
:1083B000200E016E086AC7C92EF0C6C92DF0C5C9C6
:1083C0002CF0C4C92BF053EC00F0820E026E400E6C
:1083D000096E2A6A540E296E066A056A200E016E1D
:1083E0002C0EBEEC00F0820E026E400E096E2A6A60
:1083F000540E296E066A056A200E016EC05121ECEA
:1084000000F000010901C32B100EC35D0001D8A4C8
:1084100028EF42F0820E026E400E096E2A6A540E58
:10842000296E066A056A200E016E0D0EBEEC00F084
:10843000820E026E400E096E2A6A540E296E066A7A
:10844000056A200E016E0A0EBEEC00F00901C36B36
:1084500000010901C42B000EC523C623C723000158
:10846000D8A0FED61200A30E0901D16FA20ED26FC2
:10847000AB0ED36FAA0ED46FFF0EDBCFC8F9DD525F
:108480000801BA9D0901C851100DF3CF2BF0F4CFAC
:108490002CF0080E2B5CE66F000E2C58E76FD151C4
:1084A0002DEC01F0E7512DEC01F0E6512DEC01F03F
:1084B00012EC01F0DE6FC851100DF3CF2BF0F4CFAA
:1084C0002CF0070E2B5CE66F000E2C58E76FD15195
:1084D0002DEC01F0E7512DEC01F0E6512DEC01F00F
:1084E00012EC01F0DF6FC851100DF3CF2BF0F4CF79
:1084F0002CF0060E2B5CE66F000E2C58E76FD15166
:108500002DEC01F0E7512DEC01F0E6512DEC01F0DE
:1085100012EC01F0E06FC851100DF3CF2BF0F4CF47
:108520002CF0050E2B5CE66F000E2C58E76FD15136
:108530002DEC01F0E7512DEC01F0E6512DEC01F0AE
:1085400012EC01F0E16FDEC9CCF9DFC9CBF9E0C96B
:10855000CAF9E1C9C9F9C851100DF3CF2BF0F4CF16
:108560002CF0040E2B5CE66F000E2C58E76FD151F7
:108570002DEC01F0E7512DEC01F0E6512DEC01F06E
:1085800012EC01F0DE6FC851100DF3CF2BF0F4CFD9
:108590002CF0030E2B5CE66F000E2C58E76FD151C8
:1085A0002DEC01F0E7512DEC01F0E6512DEC01F03E
:1085B00012EC01F0DF6FC851100DF3CF2BF0F4CFA8
:1085C0002CF0020E2B5CE66F000E2C58E76FD15199
:1085D0002DEC01F0E7512DEC01F0E6512DEC01F00E
:1085E00012EC01F0E06FC851100DF3CF2BF0F4CF77
:1085F0002CF02B04E66F000E2C58E76FD1512DECB8
:1086000001F0E7512DEC01F0E6512DEC01F012ECF8
:1086100001F0E16FDEC9D0F9DFC9CFF9E0C9CEF9C9
:10862000E1C9CDF9CCC9DDF9CBC9DCF9CAC9DBF99F
:10863000C9C9DAF900010901DA51CD5DDB51CE5922
:10864000DC51CF59DD51D059DD51D019D8B0800A55
:108650000001D8A88DEF43F0D8960901DDBFD88678
:108660000001D8B664EF43F00901DD530AE1DC51A3
:1086700008E1FF0EDA5DFF0EDB590001D8A064EFC0
:1086800043F00901DA29E66F000EDB21E76FD351D1
:108690002DEC01F0E7512DEC01F0E6512DEC01F04D
:1086A00012EC01F0D96F820E026E400E096E2A6A3A
:1086B000540E296E066A056A200E016ED951BEEC71
:1086C00000F0000183EF43F0DBC9E7F9DAC9E6F90E
:1086D0000901D1512DEC01F0E7512DEC01F0E651EB
:1086E0002DEC01F012EC01F0D96F820E026E400EFB
:1086F000096E2A6A540E296E066A056A200E016EFA
:10870000D951BEEC00F000010901DA2B000EDB2389
:10871000DC23DD230001D8A08DD70801BA8DE86ADB
:10872000BABD010EDE6E00011200D89680A3D88675
:10873000D8B69CEF43F0808DD89680A1D886D8B665
:10874000D1EF43F0B9C30BF0BAC30CF00BC0DEFF9E
:108750000CC0DEFF7EC0DEFF7FC0DEFF45EC0AF00E
:1087600019EEECF0A2EC02F00901ED530001D8A4DF
:10877000C1EF43F01F0E0901EC5D0001D8A0C7EF67
:1087800043F08091808DD6EC61F0CFEF43F0D6ECD2
:1087900061F0ECC9DEFFEDC9DEFF46EC62F0D3EF1D
:1087A00043F050EC0BF01200890EDE6E200EDE6EF0
:1087B000DE6AF1EC54F08A0EDE6E2F0EDE6E030ED2
:1087C000DE6EF1EC54F01C0EDE6E060EDE6E080E50
:1087D000DE6EF1EC54F0D70EDE6E870EDE6E080E04
:1087E000DE6EF1EC54F0040EDE6E350EDE6E080E19
:1087F000DE6EF1EC54F012EC4AF0010E8C5DD8A460
:1088000004EF44F056EF15F0020E8C5DD8B40AEF79
:1088100044F0F1D788EC07F00AEC32F090C098F001
:108820008FC097F08EC096F08DC095F094C09CF0EC
:1088300093C09BF092C09AF091C099F0CDEC69F092
:10884000890EDE6E200EDE6EDE6AF1EC54F08A0ECA
:10885000DE6E2F0EDE6E030EDE6EF1EC54F01C0E9B
:10886000DE6E060EDE6E080EDE6EF1EC54F0D90EF2
:10887000DE6E870EDE6E080EDE6EF1EC54F0060E34
:10888000DE6E350EDE6E080EDE6EF1EC54F012EC8C
:108890004AF0010E8C5DD8A450EF44F056EF15F06D
:1088A000030E8C5DD8B456EF44F0F1D788EC07F096
:1088B0000AEC32F090C0A0F08FC09FF08EC09EF006
:1088C0008DC09DF094C0A4F093C0A3F092C0A2F01C
:1088D00091C0A1F0BAC0C6F0B9C0C5F0CDEC69F046
:1088E0008083808B7DEF1FF0120019EEF4F0A2EC74
:1088F00002F019EEF6F0A2EC02F0D89680A3D8862A
:10890000D8B68AEF44F0380E0901F16F380EF26FD5
:10891000380EF36F0001F5C91AF0F4C919F0030E0F
:108920001E6EE80E1D6E32EC02F00901EE6FF5C905
:108930002CF0F4C92BF0306AEEC92FF030C028F0CB
:108940002F50276EE80DF3CF2FF0F4CF30F02850E2
:10895000E80DF35030262750030DF35030262F50EA
:108960002B5E30502C5A2CC01AF02BC019F01E6A06
:10897000640E1D6E32EC02F0EF6FF5C92CF0F4C9F5
:108980002BF0306AEEC92FF030C028F02F50276E40
:10899000E80DF3CF2FF0F4CF30F02850E80DF3506E
:1089A00030262750030DF35030262F502B5E3050C9
:1089B0002C5A306AEFC92FF03050640DF3CF30F0ED
:1089C0002F50640DF3CF2FF0F45030262F502B5E34
:1089D00030502C5A2CC01AF02BC019F01E6A0A0E07
:1089E0001D6E32EC02F0F06FDE6A570EDE6E000193
:1089F00035EC60F0170E0901F86FEF51F25D0001E0
:108A0000D8B409EF45F0EFC9DEFFF8C9DEFF59EC35
:108A100066F0EFC9F2F9620E0901F86FF051F35DEB
:108A20000001D8B41AEF45F0F0C9DEFFF8C9DEFF47
:108A300059EC66F0F0C9F3F90801BA9F0901EE5349
:108A40000001D8B438EF45F0010E0901F96FF86B59
:108A5000EE51F15D0001D8B436EF45F0EEC9DEFF0E
:108A6000F8C9DEFFF9C9DEFF8AEC68F00801BA8FA9
:108A70000001E86A0801BABF010EDE6E00011200B3
:108A800019EEFAF0A2EC02F019EEFCF0A2EC02F002
:108A90000901FC51FA5DFD51FB590001D8B059EFB5
:108AA00045F0050EDE6EDE6ADE6AF1EC54F077EF1B
:108AB00045F00901FB51FD5D0001D8A470EF45F0C0
:108AC0000901FA51FC5D0001D8A470EF45F0070ED2
:108AD000DE6EDE6A070EDE6EF1EC54F077EF45F0E5
:108AE000090EDE6EDE6A0A0EDE6EF1EC54F0120044
:108AF00019EEFEF0A2EC02F01AEE01F0A2EC02F088
:108B00000A0101510901FE5D0A0102510901FF59E3
:108B10000001D8B094EF45F0AF0EDE6EDE6ADE6A7B
:108B2000F1EC54F0B4EF45F00901FF510A01025D88
:108B30000001D8A4ADEF45F00901FE510A01015D25
:108B40000001D8A4ADEF45F0B10EDE6EDE6A030E73
:108B5000DE6EF1EC54F0B4EF45F0B30EDE6EDE6A7B
:108B6000040EDE6EF1EC54F01200FF0EDB50DD520D
:108B70000A010D83E8A00D93FF0EDB50DD520D813D
:108B8000E8A00D911AEE0EF0A2EC02F01AEE10F031
:108B9000A2EC02F0D896000180A3D886D8B6DEEF0A
:108BA00045F0430E0A010A6F430E0B6F430E0C6F24
:108BB000430E076F430E086F430E096F00010A0151
:108BC000036B046B056B066BD8960DA1D88600016C
:108BD000D8B608EF47F0090E0A01126F0D0E00011A
:108BE000815DD8A4F7EF45F0040E0A01126F000171
:108BF000D8960A010DA3D8860001D8B654EF46F0E6
:108C00000FCA1AF00ECA19F0020EBCEC01F00A01EC
:108C1000036F0FCA1AF00ECA19F0010EBCEC01F076
:108C2000046F0FCA1AF00ECA19F0000EBCEC01F066
:108C3000056F066B0A0E136F0351075D0001D8B470
:108C40002AEF46F012CADEFF13CADEFF03CADEFFB8
:108C500043EC66F003CA07FA330E0A01136F04519E
:108C6000085D0001D8B43DEF46F012CADEFF13CA1A
:108C7000DEFF04CADEFF43EC66F004CA08FA5C0EAD
:108C80000A01136F0551095D0001D8B450EF46F099
:108C900012CADEFF13CADEFF05CADEFF43EC66F030
:108CA00005CA09FA06EF47F00FCA1AF00ECA19F002
:108CB000030EBCEC01F00A01036F0FCA1AF00ECAD2
:108CC00019F0020EBCEC01F0046F0FCA1AF00ECAC4
:108CD00019F0010EBCEC01F0056F0FCA1AF00ECAB4
:108CE00019F0000EBCEC01F0066F03530001D8A48C
:108CF000C1EF46F0140E0A01136F0451075D000125
:108D0000D8B48BEF46F012CADEFF13CADEFF04CAE6
:108D1000DEFF43EC66F004CA07FA410E0A01136F46
:108D20000551085D0001D8B49EEF46F012CADEFF7F
:108D300013CADEFF05CADEFF43EC66F005CA08FA77
:108D40006E0E0A01136F0651095D0001D8B4B1EF30
:108D500046F012CADEFF13CADEFF06CADEFF43EC8E
:108D600066F006CA09FA060EDE6E6F0EDE6EE6ECDF
:108D700060F0060EDE6E420EDE6EC2EC60F006EFB4
:108D800047F0140E0A01136F0351075D0001D8B4B8
:108D9000D2EF46F012CADEFF13CADEFF03CADEFFBF
:108DA00043EC66F003CA07FA410E0A01136F04513F
:108DB000085D0001D8B4E5EF46F012CADEFF13CA21
:108DC000DEFF04CADEFF43EC66F004CA08FA6E0E4A
:108DD0000A01136F0551095D0001D8B4F8EF46F0A0
:108DE00012CADEFF13CADEFF05CADEFF43EC66F0DF
:108DF00005CA09FA060EDE6E420EDE6EE6EC60F083
:108E0000060EDE6E6F0EDE6EC2EC60F01EEF48F0F6
:108E10000A01126B0D0E0001815DD8A413EF47F01B
:108E2000040E0A01126F0001D8960A010DA3D8861C
:108E30000001D8B670EF47F00FCA1AF00ECA19F049
:108E4000020EBCEC01F00A01036F0FCA1AF00ECA41
:108E500019F0010EBCEC01F0046F0FCA1AF00ECA33
:108E600019F0000EBCEC01F0056F066B0A0E136FD3
:108E700003510A5D0001D8B446EF47F012CADEFF85
:108E800013CADEFF03CADEFF43EC66F003CA0AFA28
:108E9000330E0A01136F04510B5D0001D8B459EF72
:108EA00047F012CADEFF13CADEFF04CADEFF43EC3E
:108EB00066F004CA0BFA5C0E0A01136F05510C5DD3
:108EC0000001D8B46CEF47F012CADEFF13CADEFF10
:108ED00005CADEFF43EC66F005CA0CFA1EEF48F047
:108EE0000FCA1AF00ECA19F0030EBCEC01F00A0109
:108EF000036F0FCA1AF00ECA19F0020EBCEC01F093
:108F0000046F0FCA1AF00ECA19F0010EBCEC01F082
:108F1000056F0FCA1AF00ECA19F0000EBCEC01F072
:108F2000066F03530001D8A4DBEF47F00C0E0A01D3
:108F3000136F04510A5D0001D8B4A7EF47F012CABD
:108F4000DEFF13CADEFF04CADEFF43EC66F004CA8C
:108F50000AFA390E0A01136F05510B5D0001D8B4EE
:108F6000BAEF47F012CADEFF13CADEFF05CADEFF02
:108F700043EC66F005CA0BFA660E0A01136F065140
:108F80000C5D0001D8B4CDEF47F012CADEFF13CA62
:108F9000DEFF06CADEFF43EC66F006CA0CFADE6AA4
:108FA0005F0EDE6E2DEC61F0DE6A320EDE6E09ECD5
:108FB00061F01EEF48F00C0E0A01136F03510A5DB9
:108FC0000001D8B4ECEF47F012CADEFF13CADEFF8F
:108FD00003CADEFF43EC66F003CA0AFA390E0A013F
:108FE000136F04510B5D0001D8B4FFEF47F012CAB4
:108FF000DEFF13CADEFF04CADEFF43EC66F004CADC
:109000000BFA660E0A01136F05510C5D0001D8B40E
:1090100012EF48F012CADEFF13CADEFF05CADEFFF8
:1090200043EC66F005CA0CFADE6A320EDE6E2DECF9
:1090300061F0DE6A5F0EDE6E09EC61F01200FF0E79
:10904000DBCF17FADD52FF0EDBCF16FADD52FF0E33
:10905000DBCF15FADD52FF0EDBCF14FADD52D896C6
:1090600080A3D886D8B675EF48F0630E0A011B6F4F
:10907000630E1A6F630E196F630E186F010EDE6EAA
:10908000000158EC6CF04E0EDE6E74EC6CF00A01D0
:109090001E6B0001040E0A011E5D0001D8B05AEFDC
:1090A00048F03F0EDE6EE4EC6CF00A011E2B00016E
:1090B000D8A4EFD7040EDE6E58EC6CF04E0EDE6EC8
:1090C00074EC6CF00A011E6B0001040E0A011E5DB7
:1090D0000001D8B075EF48F0FC0EDE6EE4EC6CF0E9
:1090E0000A011E2B0001D8A4EFD70A011D6B1C6BCF
:1090F0001451185D0001D8B486EF48F01DCADEFF98
:109100001CCADEFF14CADEFF43EC66F014CA18FA6C
:10911000280E0A011C6F1551195D0001D8B499EF92
:1091200048F01DCADEFF1CCADEFF15CADEFF43EC95
:1091300066F015CA19FA540E0A011C6F16511A5D11
:109140000001D8B4ACEF48F01DCADEFF1CCADEFF38
:1091500016CADEFF43EC66F016CA1AFA7C0E0A0144
:109160001C6F17511B5D0001D8B4BFEF48F01DCA3A
:10917000DEFF1CCADEFF17CADEFF43EC66F017CA2B
:109180001BFA1200030EC36F840EC26FC3C01AF025
:10919000C2C019F01E6A3C0E1D6E32EC02F00A01CC
:1091A000236F1A6A23CA19F0010EBCEC01F01F6F7D
:1091B0001A6A23CA19F0000EBCEC01F0206F216B73
:1091C000226B1FCADEFF20CADEFF21CADEFF22CAD1
:1091D000DEFF000134DF12EC4AF0010E8C5DD8A4F2
:1091E000F7EF48F080932AEF49F025EF49F0020E9F
:1091F0008C5DD8A413EF49F02C0EC227010EC323B7
:10920000030EC35DD8A011EF49F0D8A40DEF49F0CB
:10921000850EC25DD8A011EF49F0010EC36F2C0E70
:10922000C26F25EF49F0030E8C5DD8A425EF49F0FD
:109230002C0EC25F010EC35BC351C211D8A425EF2F
:1092400049F0030EC36F840EC26FC80E82EC01F0AA
:109250009DD712001A0EDE6E790EDE6E050EDE6EE2
:10926000F1EC54F0C80E82EC01F00A01296B000108
:10927000F2A4E0EF49F00A01292B030E295D000159
:10928000D8A445EF49F00A01296B0001C20ED76E40
:10929000F70ED66EF294C207000EC35BC3C01AF07D
:1092A000C2C019F01E6A3C0E1D6E32EC02F00A01BB
:1092B000246F1A6A24CA19F0010EBCEC01F0256F64
:1092C0001A6A24CA19F0000EBCEC01F0266FC3C064
:1092D0001AF0C2C019F01E6A3C0E1D6E32EC02F08C
:1092E00021C024FA1A6A24CA19F0010EBCEC01F05C
:1092F000276F1A6A24CA19F0000EBCEC01F0286F1F
:1093000025CADEFF26CADEFF27CADEFF28CADEFF27
:10931000000195DEC351C211D8A491EF49F0E3EFEB
:1093200049F012EC4AF0010E8C5DD8A4A5EF49F08B
:10933000020E0A01295D0001D8A4A3EF49F0330E03
:10934000816F56EF15F0DEEF49F0020E8C5DD8A468
:10935000B8EF49F0030EC35D480ED8B4C25DD8B073
:10936000B6EF49F03C0EC227000EC323DEEF49F0F2
:10937000030E8C5DD8A4D2EF49F0C353D8A4C6EF36
:1093800049F03D0EC25DD8A0CCEF49F03C0EC25F63
:10939000000EC35BD0EF49F00A0E816F56EF15F057
:1093A000DEEF49F0040E8C5DD8A4D9EF49F0DEEF72
:1093B00049F0050E8C5DD8A4DEEF49F0E1EF49F0ED
:1093C00056D755D712000A012A6B00011A0E0A015E
:1093D0002A5D0001D8B0FCEF49F01CEC6DF0640E82
:1093E00082EC01F023EC6DF0640E82EC01F00A01D6
:1093F0002A2B0001D8A4E9D7010EAA5DD8A40CEF4E
:109400004AF0030EA95DD8A40CEF4AF0020EA96F32
:10941000FDEC3CF0020EAA6F82C081F080837DEFEC
:109420001FF0120080B616EF4AF08087D89680A70A
:10943000D886D8B623EF4AF03B0EDE6E980EDE6E6D
:10944000DE6AF1EC54F080B22FEF4AF0050E82ECA8
:1094500001F080B22FEF4AF0808953EF50F08C6B0F
:109460000A010D97000180A03BEF4AF00A010D8729
:10947000030E00018C6F81A243EF4AF00A010D87B1
:10948000040E00018C6F80AA4BEF4AF00A010D8791
:10949000010E00018C6F82A253EF4AF00A010D8782
:1094A000020E00018C6F82A05BEF4AF00A010D876B
:1094B000050E00018C6FD8960A010DB7D886000101
:1094C000D8B6DEEF4AF0810E026E010E096E400E34
:1094D0002A6E200E296E066A640E056E0B6AD8800D
:1094E0007CEC00F0D8A0DEEF4AF00AEE2BF00B5037
:1094F0001DC0EBFF0B2A0B501008F1E10A013B6B7A
:109500000001100E0A013B5D0001D8B0DEEF4AF009
:109510000AEE2BF00A013B51EB500B6E030E0B5C75
:109520000001D8A4D9EF4AF0030E0A013B250AEE48
:109530002BF0EB503D6F1A6A3DCA19F0080E6BEC28
:1095400002F03C6F800E3C5D0001D8A4ACEF4AF005
:10955000010E8C6FD9EF4AF0400E0A013C5D00010C
:10956000D8A4B7EF4AF0020E8C6FD9EF4AF0200E64
:109570000A013C5D0001D8A4C2EF4AF0030E8C6FD3
:10958000D9EF4AF0100E0A013C5D0001D8A4CDEFDE
:109590004AF0040E8C6FD9EF4AF0080E0A013C5DC8
:1095A0000001D8A4D8EF4AF0050E8C6FD9EF4AF02D
:1095B0008C6B0A013B2B0001D8A4A2D71200D896CD
:1095C00080A3D886D8B686EF4BF0890EDE6E090EE2
:1095D000DE6E010EDE6EF1EC54F0D70EDE6E860EFE
:1095E000DE6E0A0EDE6EF1EC54F00E0EDE6E860EAE
:1095F000DE6E0C0EDE6EF1EC54F0D90EDE6E860ED1
:10960000DE6E0E0EDE6EF1EC54F0DB0EDE6E350E0D
:10961000DE6E070EDE6EF1EC54F0DF0EDE6E640ED1
:10962000DE6E070EDE6EF1EC54F0E30EDE6E3A0EE7
:10963000DE6E040EDE6EF1EC54F0DD0EDE6E580EC2
:10964000DE6E040EDE6EF1EC54F04E0E6BEC01F0AB
:10965000C06F0A01406BC0C03FFA3FCADEFF40CA7C
:10966000DEFF3FCADEFF40CADEFFDE6A010EDE6EAD
:109670000001B5EC45F00A0E82EC01F04D0E6BECEA
:1096800001F0BF6FBF53D8A453EF4BF00C0EDE6E4A
:10969000490EDE6E070EDE6EF1EC54F0C80E82EC61
:1096A00001F082EF4BF0010EBF5DD8A465EF4BF0E7
:1096B0000A0EDE6E490EDE6E070EDE6EF1EC54F021
:1096C000C80E82EC01F082EF4BF0020EBF5DD8A411
:1096D00077EF4BF00E0EDE6E490EDE6E070EDE6E7D
:1096E000F1EC54F0C80E82EC01F082EF4BF00C0E5E
:1096F000DE6E490EDE6E070EDE6EF1EC54F0C80E23
:1097000082EC01F08093C80E82EC01F0C0510A0196
:109710003E5D0001D8B4A2EF4BF00A01406BC0C01F
:109720003FFA3FCADEFF40CADEFF3FCADEFF40CA43
:10973000DEFFDE6A010EDE6E0001B5EC45F00A0EBA
:1097400082EC01F00A0141510001BF5DD8B4E9EF9C
:109750004BF0BF53D8A4BAEF4BF00C0EDE6E490E9F
:10976000DE6E070EDE6EF1EC54F0C80E82EC01F0F6
:10977000E9EF4BF0010EBF5DD8A4CCEF4BF00A0E21
:10978000DE6E490EDE6E070EDE6EF1EC54F0C80E92
:1097900082EC01F0E9EF4BF0020EBF5DD8A4DEEFE2
:1097A0004BF00E0EDE6E490EDE6E070EDE6EF1EC35
:1097B00054F0C80E82EC01F0E9EF4BF00C0EDE6EB7
:1097C000490EDE6E070EDE6EF1EC54F0C80E82EC30
:1097D00001F028DE010E8C5DD8A405EF4CF0AA6ADA
:1097E0004D0EA96EBF5174EC01F0050E82EC01F034
:1097F000AA6A4E0EA96EC05174EC01F0050E82ECFF
:1098000001F03C0E816F56EF15F0020E8C5DD8A46E
:1098100012EF4CF0C0C03EFAC02BC029D8A412EF02
:109820004CF0C06B030E8C5DD8A41FEF4CF0D4C875
:109830003EFAC053D8A41EEF4CF0C069C007040E16
:109840008C5DD8A42DEF4CF0BFC041FABF2B030EA6
:10985000BF5DD8A42DEF4CF0BF6B050E8C5DD8A476
:109860003BEF4CF0BFC041FABF2B030EBF5DD8A445
:109870003BEF4CF0BF6BA3D61200D89680A3D886DE
:10988000D8B6B9EF4CF0E90EDE6E1C0EDE6EDE6A65
:10989000F1EC54F0D70EDE6E860EDE6E0A0EDE6E32
:1098A000F1EC54F03F0EDE6E890EDE6E0C0EDE6EB5
:1098B000F1EC54F0D90EDE6E860EDE6E0E0EDE6E0C
:1098C000F1EC54F0DB0EDE6E1B0EDE6E070EDE6E6C
:1098D000F1EC54F0DF0EDE6E740EDE6E070EDE6EFF
:1098E000F1EC54F0E30EDE6E3A0EDE6E040EDE6E28
:1098F000F1EC54F0DD0EDE6E580EDE6E040EDE6E00
:10990000F1EC54F0460E6BEC01F00801D46F0A0143
:10991000446BD4C843FA43CADEFF44CADEFF43CADD
:10992000DEFF44CADEFFDE6A010EDE6E0001B5EC2A
:1099300045F00A0E82EC01F04C0E6BEC01F00801D0
:10994000D36FD3530001D8A4B0EF4CF0E50EDE6E18
:109950002F0EDE6E060EDE6EF1EC54F0B8EF4CF01A
:10996000E70EDE6E2F0EDE6E060EDE6EF1EC54F0AC
:1099700080930801D4510A01425D0001D8B4D6EFAA
:109980004CF00A01446BD4C843FA43CADEFF44CA10
:10999000DEFF43CADEFF44CADEFFDE6A010EDE6E72
:1099A0000001B5EC45F00A0E82EC01F00A014551C8
:1099B0000801D35D0001D8B4FCEF4CF00801D3538B
:1099C0000001D8A4F1EF4CF0E50EDE6E2F0EDE6E36
:1099D000060EDE6EF1EC54F0640E82EC01F0FCEF4A
:1099E0004CF0E70EDE6E2F0EDE6E060EDE6EF1EC34
:1099F00054F0640E82EC01F012EC4AF0010E8C5D22
:109A0000D8A41BEF4DF0AA6A460EA96E0801D451E6
:109A100074EC01F0050E82EC01F0AA6A4C0EA96EFE
:109A2000D35174EC01F0050E82EC01F03C0E000104
:109A3000816F56EF15F0020E8C5DD8A42CEF4DF01F
:109A4000D4C842FA0801D42BD4290001D8A42BEFA2
:109A50004DF00801D46B0001030E8C5DD8A43EEFDD
:109A60004DF0D4C842FA0801D4530001D8A43BEF0A
:109A70004DF00801D46900010801D4070001040E6B
:109A80008C5DD8A451EF4DF0D3C845FA0801D32B13
:109A9000020ED35D0001D8A450EF4DF00801D36B46
:109AA0000001050E8C5DD8A463EF4DF0D3C845FAD4
:109AB0000801D32B020ED35D0001D8A462EF4DF054
:109AC0000801D36B0001D9D61200D89680A3D8869E
:109AD000D8B6D9EF4DF0EB0EDE6E2A0EDE6EDE6AE2
:109AE000F1EC54F0D70EDE6E860EDE6E0A0EDE6EE0
:109AF000F1EC54F0D90EDE6E860EDE6E0E0EDE6ECA
:109B0000F1EC54F0DB0EDE6E250EDE6E070EDE6E1F
:109B1000F1EC54F0DF0EDE6E6A0EDE6E070EDE6EC6
:109B2000F1EC54F0E30EDE6E3A0EDE6E040EDE6EE5
:109B3000F1EC54F0DD0EDE6E580EDE6E040EDE6EBD
:109B4000F1EC54F0470E6BEC01F00801D56F0A01FF
:109B5000486BD5C847FA47CADEFF48CADEFF47CA86
:109B6000DEFF48CADEFFDE6A010EDE6E0001B5ECE4
:109B700045F00A0E82EC01F0480E6BEC01F0080192
:109B8000D66FD6530001D8A4D0EF4DF0F10EDE6EA3
:109B9000390EDE6E060EDE6EF1EC54F0D8EF4DF0AD
:109BA000EF0EDE6E390EDE6E060EDE6EF1EC54F058
:109BB00080930801D5510A01465D0001D8B4F6EF43
:109BC0004DF00A01486BD5C847FA47CADEFF48CABC
:109BD000DEFF47CADEFF48CADEFFDE6A010EDE6E28
:109BE0000001B5EC45F00A0E82EC01F00A01495182
:109BF0000801D65D0001D8B41CEF4EF00801D65321
:109C00000001D8A411EF4EF0F10EDE6E390EDE6EBB
:109C1000060EDE6EF1EC54F0640E82EC01F01CEFE7
:109C20004EF0EF0EDE6E390EDE6E060EDE6EF1ECDD
:109C300054F0640E82EC01F012EC4AF0010E8C5DDF
:109C4000D8A44DEF4EF0AA6A470EA96E0801D5516F
:109C500074EC01F0050E82EC01F0AA6A480EA96EC0
:109C6000D65174EC01F0050E82EC01F0010ED65DC8
:109C70000001D8A441EF4EF0BD6BD5C8BCF048EF51
:109C80004EF00801D5513C0DF3CFBCF0F4CFBDF040
:109C900000013C0E816F56EF15F0020E8C5DD8A4CA
:109CA0005FEF4EF0D5C846FA0801D5290001D8A4C7
:109CB0005CEF4EF00801D56B00010801D52B0001C7
:109CC000030E8C5DD8A471EF4EF0D5C846FA08019A
:109CD000D507D5530001D8A470EF4EF00801D5691F
:109CE0000001040E8C5DD8A483EF4EF0D6C849FA6B
:109CF0000801D62B020ED65D0001D8A482EF4EF0EB
:109D00000801D66B0001050E8C5DD8A495EF4EF0CE
:109D1000D6C849FA0801D62B020ED65D0001D8A498
:109D200094EF4EF00801D66B0001CFD612000A0165
:109D30004A690001A86BA76BA653D8A4A7EF4EF001
:109D4000A5510A014A5D0001D8B4B7EF4EF0A5C095
:109D5000DEFFA6C0DEFFA5C0DEFFA6C0DEFFDE6A16
:109D6000010EDE6EB5EC45F00A0E82EC01F012EC4D
:109D70004AF0010E8C5DD8A4C1EF4EF080837DEFD8
:109D80001FF0020E8C5DD8A4D4EF4EF0A5C04AFAA5
:109D9000A54BA62BA529A611D8A4D1EF4EF0A66BF2
:109DA000A56B640E82EC01F0C7D712000A014B6963
:109DB0000001A66BA56BA853D8A4E6EF4EF0A751FF
:109DC0000A014B5D0001D8B4F6EF4EF0A7C0DEFFEC
:109DD000A8C0DEFFA7C0DEFFA8C0DEFFDE6A010E5E
:109DE000DE6EB5EC45F00A0E82EC01F012EC4AF0A2
:109DF000010E8C5DD8A400EF4FF080837DEF1FF043
:109E0000030E8C5DD8A413EF4FF0A7C04BFAA74BFD
:109E1000A82BA729A811D8A410EF4FF0A86BA76B07
:109E2000640E82EC01F0C7D71200830EDE6E190EAD
:109E3000DE6EDE6AF1EC54F0D70EDE6E860EDE6E5C
:109E40000A0EDE6EF1EC54F0D90EDE6E860EDE6E7A
:109E50000E0EDE6EF1EC54F0E30EDE6E3A0EDE6EA8
:109E6000040EDE6EF1EC54F0DD0EDE6E580EDE6E8A
:109E7000040EDE6EF1EC54F08B510A014D5D0001D1
:109E8000D8A44AEF4FF08A510A014C5D0001D8B4C2
:109E90005AEF4FF08AC0DEFF8BC0DEFF8AC0DEFFC4
:109EA0008BC0DEFFDE6A010EDE6EB5EC45F0050EFE
:109EB00082EC01F012EC4AF0010E8C5DD8A464EF44
:109EC0004FF080837DEF1FF0020E8C5DD8A47CEFF5
:109ED0004FF08BC04DFA8AC04CFA8A4B8B2B8B51BA
:109EE000010A680ED8B48A19D8A479EF4FF08B6BA9
:109EF0008A6B050E82EC01F0030E8C5DD8A496EF00
:109F00004FF08BC04DFA8AC04CFA8B518A11D8A4FD
:109F100090EF4FF0010E8B6F670E8A6F93EF4FF04B
:109F20008A07000E8B5B050E82EC01F0A5D71200AC
:109F3000D89680A3D886D8B6E8EF4FF0120EDE6E22
:109F4000150EDE6EDE6AF1EC54F01E0EDE6E390E7A
:109F5000DE6E070EDE6EF1EC54F0D70EDE6E860E6E
:109F6000DE6E0A0EDE6EF1EC54F0D90EDE6E860E59
:109F7000DE6E0E0EDE6EF1EC54F0E30EDE6E3A0E87
:109F8000DE6E040EDE6EF1EC54F0DD0EDE6E580E69
:109F9000DE6E040EDE6EF1EC54F0490E6BEC01F057
:109FA0000801D76F0A01516BD7C850FA50CADEFFBB
:109FB00051CADEFF50CADEFF51CADEFFDE6A010E63
:109FC000DE6E0001B5EC45F00A0E82EC01F08093E4
:109FD0000A014F530001D8A4F6EF4FF00A014E5189
:109FE0000801D75D0001D8B40BEF50F00A01516BA6
:109FF000D7C850FA50CADEFF51CADEFF50CADEFF92
:10A0000051CADEFFDE6A010EDE6E0001B5EC45F0DE
:10A010000A0E82EC01F012EC4AF0010E8C5DD8A41D
:10A0200021EF50F0AA6A490EA96E0801D75174ECCD
:10A0300001F0050E82EC01F03C0E0001816F56EF3D
:10A0400015F0020E8C5DD8A438EF50F00A014F6B6A
:10A05000D7C84EFA0801D72B150ED75D0001D8A43A
:10A0600034EF50F00801D76B0001050E82EC01F0CF
:10A07000030E8C5DD8A450EF50F00A014F6BD7C887
:10A080004EFA0801D7530001D8A44AEF50F0140E3D
:10A090000801D76F00010801D707050E82EC01F017
:10A0A000000146D7120084968494C80E82EC01F019
:10A0B000CDEC69F0D89680A9D886D8B66AEF50F072
:10A0C0008D0EDE6E1A0EDE6E050EDE6EF1EC54F0B5
:10A0D0007AEF50F0810EDE6E290EDE6E020EDE6E1D
:10A0E000F1EC54F08F0EDE6E260EDE6E050EDE6E87
:10A0F000F1EC54F0070E1E6ED00E83EC01F0869446
:10A100008692DE6A58EC6CF0DE6A66EC6CF0DE6A11
:10A1100074EC6CF0DE6A9EEC6CF000EC6DF0030EFB
:10A120001E6EE80E83EC01F08698180E82EC01F0AA
:10A130008686180E82EC01F08696180E82EC01F0ED
:10A140008698010E1E6EF40E83EC01F08698270EA1
:10A150001E6E100E83EC01F01200630EDE6E230EF5
:10A16000DE6E0A0EDE6EF1EC54F0D70EDE6E6E0E71
:10A17000DE6E080EDE6EF1EC54F0D90EDE6E6E0E61
:10A18000DE6E0C0EDE6EF1EC54F0E30EDE6E3F0E72
:10A19000DE6E0E0EDE6EF1EC54F0DD0EDE6E650E40
:10A1A000DE6E0E0EDE6EF1EC54F01C0EDE6E170E3F
:10A1B000DE6E010EDE6EF1EC54F0EB0EDE6E3D0E47
:10A1C000DE6EDE6AF1EC54F0010EA95DD8A4FCEF5E
:10A1D00050F0DE6A0F0EDE6E380EDE6E040EDE6E9E
:10A1E00018EC5FF04D0EDE6E3F0EDE6E040EDE6E7E
:10A1F000F1EC54F02AEF51F0020EA95DD8A414EF4F
:10A2000051F0DE6A0F0EDE6E380EDE6E040EDE6E6C
:10A2100018EC5FF0590EDE6E450EDE6E040EDE6E3B
:10A22000F1EC54F02AEF51F0030EA95DD8A42AEF07
:10A2300051F0DE6A0F0EDE6E380EDE6E040EDE6E3C
:10A2400018EC5FF0550EDE6E380EDE6E040EDE6E1C
:10A25000F1EC54F08C6B630EDE6E230EDE6E0A0E94
:10A26000DE6EF1EC54F0D70EDE6E6E0EDE6E080E72
:10A27000DE6EF1EC54F0D90EDE6E6E0EDE6E0C0E5C
:10A28000DE6EF1EC54F0E30EDE6E3F0EDE6E0E0E6F
:10A29000DE6EF1EC54F0DD0EDE6E650EDE6E0E0E3F
:10A2A000DE6EF1EC54F012EC4AF0010E8C5DD8A495
:10A2B0008BEF51F0010EAA5DD8A468EF51F0020EA9
:10A2C000A95DD8A468EF51F0FDEC3CF0020EAA6F36
:10A2D000020EAA5DD8A476EF51F0030EA95DD8A4B2
:10A2E00076EF51F0010EA96F010EAA6F1A6A82C0B3
:10A2F00019F0000EBCEC01F00B6E0B52D8B487EFD6
:10A3000051F082C081F07DEF1FF089EF51F056EFE0
:10A3100015F054EF52F0020E8C5DD8A4E5EF51F029
:10A32000A92B040EA95DD8A498EF51F0010EA96FD6
:10A33000010EA95DD8A4B0EF51F0DE6A0F0EDE6EFB
:10A34000380EDE6E040EDE6E18EC5FF04D0EDE6E23
:10A350003F0EDE6E040EDE6EF1EC54F0DEEF51F0D7
:10A36000020EA95DD8A4C8EF51F0DE6A0F0EDE6EB2
:10A37000380EDE6E040EDE6E18EC5FF0590EDE6EE7
:10A38000450EDE6E040EDE6EF1EC54F0DEEF51F0A1
:10A39000030EA95DD8A4DEEF51F0DE6A0F0EDE6E6B
:10A3A000380EDE6E040EDE6E18EC5FF0550EDE6EBB
:10A3B000380EDE6E040EDE6EF1EC54F0010E1E6EF1
:10A3C000900E83EC01F054EF52F0030E8C5DD8A494
:10A3D0003EEF52F0A907A953D8A4F1EF51F0030EB4
:10A3E000A96F010EA95DD8A409EF52F0DE6A0F0E25
:10A3F000DE6E380EDE6E040EDE6E18EC5FF04D0E73
:10A40000DE6E3F0EDE6E040EDE6EF1EC54F037EFC2
:10A4100052F0020EA95DD8A421EF52F0DE6A0F0EB1
:10A42000DE6E380EDE6E040EDE6E18EC5FF0590E36
:10A43000DE6E450EDE6E040EDE6EF1EC54F037EF8C
:10A4400052F0030EA95DD8A437EF52F0DE6A0F0E6A
:10A45000DE6E380EDE6E040EDE6E18EC5FF0550E0A
:10A46000DE6E380EDE6E040EDE6EF1EC54F0010E80
:10A470001E6E900E83EC01F054EF52F0040E8C5DD2
:10A48000D8A445EF52F054EF52F0050E8C5DD8A4DD
:10A490004CEF52F054EF52F08C53D8A453EF52F0DB
:10A4A0005CD654EF52F059D658D612001D0EDE6E0F
:10A4B000080EDE6E020EDE6EF1EC54F08C6B86A49C
:10A4C0006CEF52F0510EDE6E460EDE6E050EDE6E45
:10A4D000F1EC54F081EF52F086A279EF52F0530E76
:10A4E000DE6E460EDE6E050EDE6EF1EC54F081EF90
:10A4F00052F04D0EDE6E460EDE6E050EDE6EF1EC97
:10A5000054F0630EDE6E230EDE6E0A0EDE6EF1EC8C
:10A5100054F0D70EDE6E6E0EDE6E080EDE6EF1ECBF
:10A5200054F0D90EDE6E6E0EDE6E0C0EDE6EF1ECA9
:10A5300054F0E30EDE6E3F0EDE6E0E0EDE6EF1ECBC
:10A5400054F0DD0EDE6E650EDE6E0E0EDE6EF1EC8C
:10A5500054F012EC4AF0010E8C5DD8A4C5EF52F015
:10A560001A6A82C019F0000EBCEC01F00B6E0B529F
:10A57000D8B4C1EF52F082C081F07DEF1FF0C3EF7D
:10A5800052F056EF15F06BEF53F0020E8C5DD8A42D
:10A59000FAEF52F086B4E9EF52F086B2DAEF52F0F9
:10A5A00086848692510EDE6E460EDE6E050EDE6EDF
:10A5B000F1EC54F086A2E7EF52F0869486924D0EAD
:10A5C000DE6E460EDE6E050EDE6EF1EC54F0F3EF3D
:10A5D00052F086948682530EDE6E460EDE6E050EB7
:10A5E000DE6EF1EC54F0010E1E6E900E83EC01F065
:10A5F0006BEF53F0030E8C5DD8A42FEF53F086B4AD
:10A600001EEF53F086B20FEF53F086848692510E00
:10A61000DE6E460EDE6E050EDE6EF1EC54F086A2A6
:10A620001CEF53F0869486924D0EDE6E460EDE6E63
:10A63000050EDE6EF1EC54F028EF53F0869486821E
:10A64000530EDE6E460EDE6E050EDE6EF1EC54F03D
:10A65000010E1E6E900E83EC01F06BEF53F0040EB2
:10A660008C5DD8A449EF53F01A6A82C019F0000E2D
:10A67000BCEC01F00B6E0B52D8B445EF53F082C026
:10A6800081F07DEF1FF047EF53F056EF15F06BEFC1
:10A6900053F0050E8C5DD8A463EF53F01A6A82C0A4
:10A6A00019F0000EBCEC01F00B6E0B52D8B45FEF4A
:10A6B00053F082C081F07DEF1FF061EF53F056EF51
:10A6C00015F06BEF53F08C53D8A46AEF53F0EED62D
:10A6D0006BEF53F0EBD6EAD61200C69A94869488B4
:10A6E000060EE82EFED700008288060EE82EFED762
:10A6F00000008286060EE82EFED700008298060E25
:10A70000E82EFED700008296060EE82EFED7000047
:10A710000A01526B0001090E0A01525D0001D8B016
:10A72000ABEF53F08288060EE82EFED7000082863B
:10A73000060EE82EFED700008296060EE82EFED703
:10A7400000008294060EE82EFED700000A01522B6C
:10A750000001D8A4DFD78288060EE82EFED70000BD
:10A760008286060EE82EFED700008298060EE82E9E
:10A77000FED700008296060EE82EFED700008298D3
:10A78000060EE82EFED700008296060EE82EFED7B3
:10A7900000008286060EE82EFED700008288060E94
:10A7A000E82EFED70000C68AA1A6D8EF53F0A196E6
:10A7B0001200FF0EDBCF5BFADD52FF0EDBCF5CFA3F
:10A7C000DD52FF0EDBCF5DFADD52FF0EDBCF5EFA0E
:10A7D000DD521AEE5FF0A2EC02F01AEE61F0A2EC8C
:10A7E00002F00A01536B546B5ECA57FA00010A016A
:10A7F00057515D5D0001D8A0F0EF54F00A015B51A4
:10A800000F082B6E000ED8A0FF0F2C6E53512B5C3F
:10A81000546F080E545D0001D8A083EF54F0080E69
:10A820000A01545D0001D8A41CEF54F0070E0A0180
:10A83000586F000174EF54F0090E0A01545D0001D5
:10A84000D8A429EF54F0060E0A01586F000174EFE6
:10A8500054F00A0E0A01545D0001D8A436EF54F0FA
:10A86000050E0A01586F000174EF54F00B0E0A0137
:10A87000545D0001D8A443EF54F0040E0A01586F50
:10A88000000174EF54F00C0E0A01545D0001D8A4CD
:10A8900050EF54F0030E0A01586F000174EF54F0AA
:10A8A0000D0E0A01545D0001D8A45DEF54F0020EB4
:10A8B0000A01586F000174EF54F00E0E0A01545D46
:10A8C0000001D8A46AEF54F0010E0A01586F00018C
:10A8D00074EF54F00F0E0A01545D0001D8A473EF19
:10A8E00054F00A01586B000158CADEFF66EC6CF0A8
:10A8F000080E0A015C255A6F5ACADEFF00019EEC61
:10A900006CF08FEF54F054CA58FA58CADEFF58EC76
:10A910006CF05CCA5AFA5ACADEFF74EC6CF062CA78
:10A9200056FA61CA55FA0A0155515F5D5651605990
:10A930000001D8A0EAEF54F0080E0A01545D0001AE
:10A94000D8A0C4EF54F0A10E2DEC01F00A0157512C
:10A9500055252B6E000E56212C6E2C502DEC01F03F
:10A960002B502DEC01F012EC01F0596F1A6A59CA04
:10A9700019F0080E6BEC02F0596F59CADEFF0001A6
:10A98000F2EC6CF0DEEF54F0A10E2DEC01F00A01B8
:10A99000575155252B6E000E56212C6E2C502DEC48
:10A9A00001F02B502DEC01F012EC01F0596F59CA57
:10A9B000DEFF0001E4EC6CF00A01596B0001100E9F
:10A9C0000A0155270001D8A0AED70A01562B000175
:10A9D000D8A4A9D70A01532B572B0001D8A406D716
:10A9E0001200FF0EDBCF63FADD52FF0EDBCF64FAFD
:10A9F000DD52FF0EDBCF65FADD52010E0A01655D07
:10AA00000001D8A413EF55F0DE6A500EDE6E090E79
:10AA1000DE6EDE6A0F0EDE6E64CADEFF63CADEFF24
:10AA2000C8DE17EF5FF0050E0A01655D0001D8A4CE
:10AA30002CEF55F0700EDE6E0A0EDE6EA00EDE6E8E
:10AA40000B0EDE6EDE6A050EDE6E64CADEFF63CAC2
:10AA5000DEFFAFDE17EF5FF0070E0A01655D000154
:10AA6000D8A446EF55F0700EDE6E0A0EDE6EA00E14
:10AA7000DE6E0B0EDE6E070EDE6E080EDE6E64CA34
:10AA8000DEFF63CADEFF95DE17EF5FF0090E0A01F5
:10AA9000655D0001D8A460EF55F0700EDE6E0A0E01
:10AAA000DE6EA00EDE6E0B0EDE6E0A0EDE6E0F0E7A
:10AAB000DE6E64CADEFF63CADEFF7BDE17EF5FF087
:10AAC0000D0E0A01655D0001D8A478EF55F0DE6A2D
:10AAD000570EDE6EB00EDE6E600EDE6EDE6A0F0E9C
:10AAE000DE6E64CADEFF63CADEFF63DE17EF5FF06F
:10AAF0000F0E0A01655D0001D8A481EF55F017EF34
:10AB00005FF0110E0A01655D0001D8A48AEF55F0CF
:10AB100017EF5FF0130E0A01655D0001D8A493EFF3
:10AB200055F017EF5FF0150E0A01655D0001D8A41E
:10AB30009CEF55F017EF5FF0170E0A01655D0001FD
:10AB4000D8A4A5EF55F017EF5FF0190E0A01655D67
:10AB50000001D8A4AEEF55F017EF5FF01B0E0A010D
:10AB6000655D0001D8A4C8EF55F0F00EDE6E0B0E47
:10AB7000DE6E500EDE6E140EDE6E020EDE6E030E04
:10AB8000DE6E64CADEFF63CADEFF13DE17EF5FF01E
:10AB90001D0E0A01655D0001D8A4E2EF55F0F00E2C
:10ABA000DE6E0B0EDE6EF00EDE6E140EDE6EDE6AF4
:10ABB000010EDE6E64CADEFF63CADEFFD9EC53F01D
:10ABC00017EF5FF0210E0A01655D0001D8A4EBEFDD
:10ABD00055F017EF5FF0230E0A01655D0001D8A460
:10ABE00006EF56F0600EDE6E180EDE6E900EDE6E14
:10ABF000200EDE6E080EDE6E0A0EDE6E64CADEFF0A
:10AC000063CADEFFD9EC53F017EF5FF0250E0A019F
:10AC1000655D0001D8A420EF56F0600EDE6E180EC0
:10AC2000DE6EDE6A1F0EDE6E040EDE6E060EDE6E59
:10AC300064CADEFF63CADEFFD9EC53F017EF5FF0A2
:10AC4000270E0A01655D0001D8A43AEF56F0600EA8
:10AC5000DE6E180EDE6ED00EDE6E200EDE6EDE6A4A
:10AC6000020EDE6E64CADEFF63CADEFFD9EC53F06B
:10AC700017EF5FF02B0E0A01655D0001D8A455EFB8
:10AC800056F0600EDE6E180EDE6E900EDE6E200E3A
:10AC9000DE6E080EDE6E0A0EDE6E64CADEFF63CA6A
:10ACA000DEFFD9EC53F017EF5FF02D0E0A01655D62
:10ACB0000001D8A46FEF56F0600EDE6E180EDE6E47
:10ACC000DE6A1F0EDE6E040EDE6E060EDE6E64CAD7
:10ACD000DEFF63CADEFFD9EC53F017EF5FF02F0EF3
:10ACE0000A01655D0001D8A489EF56F0600EDE6EA2
:10ACF000180EDE6ED00EDE6E200EDE6EDE6A020EE6
:10AD0000DE6E64CADEFF63CADEFFD9EC53F017EFD4
:10AD10005FF0330E0A01655D0001D8A4A4EF56F080
:10AD2000600EDE6E180EDE6E900EDE6E200EDE6E93
:10AD3000080EDE6E0A0EDE6E64CADEFF63CADEFF38
:10AD4000D9EC53F017EF5FF0350E0A01655D000195
:10AD5000D8A4BEEF56F0600EDE6E180EDE6EDE6A10
:10AD60001F0EDE6E040EDE6E060EDE6E64CADEFFA1
:10AD700063CADEFFD9EC53F017EF5FF0370E0A011C
:10AD8000655D0001D8A4C7EF56F017EF5FF03B0EEA
:10AD90000A01655D0001D8A4E2EF56F0100EDE6EE8
:10ADA000210EDE6E800EDE6E210EDE6E0E0EDE6E6B
:10ADB0000F0EDE6E64CADEFF63CADEFFD9EC53F00D
:10ADC00017EF5FF03D0E0A01655D0001D8A4FDEFAD
:10ADD00056F0100EDE6E210EDE6EB00EDE6E210E0F
:10ADE000DE6E0C0EDE6E0D0EDE6E64CADEFF63CA12
:10ADF000DEFFD9EC53F017EF5FF03F0E0A01655DFF
:10AE00000001D8A418EF57F0100EDE6E210EDE6E92
:10AE1000B00EDE6E210EDE6E0C0EDE6E0D0EDE6EE0
:10AE200064CADEFF63CADEFFD9EC53F017EF5FF0B0
:10AE3000410E0A01655D0001D8A421EF57F017EF1C
:10AE40005FF0430E0A01655D0001D8A42AEF57F0B8
:10AE500017EF5FF0450E0A01655D0001D8A433EFDE
:10AE600057F017EF5FF0470E0A01655D0001D8A4A7
:10AE70003CEF57F017EF5FF0490E0A01655D0001E6
:10AE8000D8A456EF57F0100EDE6E210EDE6E800E47
:10AE9000DE6E220EDE6EDE6A010EDE6E64CADEFF3C
:10AEA00063CADEFFD9EC53F017EF5FF04D0E0A01D5
:10AEB000655D0001D8A470EF57F0DE6A230EDE6EE8
:10AEC000100EDE6E250EDE6E0E0EDE6E0F0EDE6EC8
:10AED00064CADEFF63CADEFFD9EC53F017EF5FF000
:10AEE0004F0E0A01655D0001D8A48AEF57F0DE6AB3
:10AEF000230EDE6E100EDE6E250EDE6E0C0EDE6E86
:10AF00000D0EDE6E64CADEFF63CADEFFD9EC53F0BD
:10AF100017EF5FF0510E0A01655D0001D8A4A4EFA0
:10AF200057F0DE6A230EDE6E100EDE6E250EDE6E2C
:10AF30000A0EDE6E0B0EDE6E64CADEFF63CADEFF33
:10AF4000D9EC53F017EF5FF0530E0A01655D000175
:10AF5000D8A4BEEF57F0DE6A230EDE6E100EDE6E52
:10AF6000250EDE6E080EDE6E090EDE6E64CADEFF92
:10AF700063CADEFFD9EC53F017EF5FF0550E0A01FC
:10AF8000655D0001D8A4D9EF57F0900EDE6E250E56
:10AF9000DE6E800EDE6E280EDE6E060EDE6E070E94
:10AFA000DE6E64CADEFF63CADEFFD9EC53F017EF32
:10AFB0005FF0570E0A01655D0001D8A4F4EF57F069
:10AFC000A00EDE6E250EDE6ED00EDE6E280EDE6E5C
:10AFD000040EDE6E050EDE6E64CADEFF63CADEFF9F
:10AFE000D9EC53F017EF5FF0590E0A01655D0001CF
:10AFF000D8A40FEF58F0400EDE6E310EDE6EA00EBC
:10B00000DE6E320EDE6E040EDE6E050EDE6E64CA7D
:10B01000DEFF63CADEFFD9EC53F017EF5FF05B0E83
:10B020000A01655D0001D8A42AEF58F0A00EDE6E7B
:10B03000250EDE6ED00EDE6E280EDE6E020EDE6E89
:10B04000030EDE6E64CADEFF63CADEFFD9EC53F086
:10B0500017EF5FF05F0E0A01655D0001D8A433EFC2
:10B0600058F017EF5FF0610E0A01655D0001D8A48A
:10B070003CEF58F017EF5FF0630E0A01655D0001C9
:10B08000D8A457EF58F0900EDE6E250EDE6E100E2F
:10B09000DE6E2A0EDE6E080EDE6E090EDE6E64CAED
:10B0A000DEFF63CADEFFD9EC53F017EF5FF0650EE9
:10B0B0000A01655D0001D8A460EF58F017EF5FF05A
:10B0C000670E0A01655D0001D8A469EF58F017EF1B
:10B0D0005FF0690E0A01655D0001D8A472EF58F0B7
:10B0E00017EF5FF06B0E0A01655D0001D8A47BEFDE
:10B0F00058F017EF5FF06F0E0A01655D0001D8A4EC
:10B1000084EF58F017EF5FF0710E0A01655D0001E2
:10B11000D8A48DEF58F017EF5FF0730E0A01655D4C
:10B120000001D8A496EF58F017EF5FF0750E0A01F2
:10B13000655D0001D8A49FEF58F017EF5FF0770E20
:10B140000A01655D0001D8A4A8EF58F017EF5FF081
:10B15000790E0A01655D0001D8A4B1EF58F017EF30
:10B160005FF07D0E0A01655D0001D8A4BAEF58F0CA
:10B1700017EF5FF07F0E0A01655D0001D8A4C3EFF1
:10B1800058F017EF5FF0810E0A01655D0001D8A449
:10B19000DEEF58F0C00EDE6E2D0EDE6EA00EDE6EFF
:10B1A000340EDE6E040EDE6E050EDE6E64CADEFF49
:10B1B00063CADEFFD9EC53F017EF5FF0830E0A018C
:10B1C000655D0001D8A4F9EF58F0C00EDE6E2D0EBB
:10B1D000DE6E900EDE6E340EDE6E060EDE6E070E36
:10B1E000DE6E64CADEFF63CADEFFD9EC53F017EFF0
:10B1F0005FF0850E0A01655D0001D8A414EF59F0D7
:10B20000800EDE6E300EDE6E900EDE6E340EDE6E62
:10B21000060EDE6E070EDE6E64CADEFF63CADEFF58
:10B22000D9EC53F017EF5FF0870E0A01655D00015E
:10B23000D8A41DEF59F017EF5FF0890E0A01655D84
:10B240000001D8A438EF59F0B00EDE6E2D0EDE6E80
:10B25000900EDE6E360EDE6E0A0EDE6E0C0EDE6EAA
:10B2600064CADEFF63CADEFFD9EC53F017EF5FF06C
:10B270008A0E0A01655D0001D8A453EF59F0B00EA3
:10B28000DE6E2E0EDE6E900EDE6E360EDE6E0D0E55
:10B29000DE6E0F0EDE6E64CADEFF63CADEFFD9EC1F
:10B2A00053F017EF5FF08D0E0A01655D0001D8A421
:10B2B0006DEF59F0900EDE6E380EDE6E500EDE6EC3
:10B2C0003F0EDE6EDE6A050EDE6E64CADEFF63CA06
:10B2D000DEFFD9EC53F017EF5FF08F0E0A01655DCA
:10B2E0000001D8A488EF59F0900EDE6E380EDE6EA5
:10B2F000E00EDE6E3D0EDE6E060EDE6E0F0EDE6EB4
:10B3000064CADEFF63CADEFFD9EC53F017EF5FF0CB
:10B31000930E0A01655D0001D8A4A2EF59F0D00E8A
:10B32000DE6E3F0EDE6EB00EDE6E450EDE6EDE6A47
:10B33000030EDE6E64CADEFF63CADEFFD9EC53F093
:10B3400017EF5FF0950E0A01655D0001D8A4BDEF0F
:10B3500059F0D00EDE6E3F0EDE6EB00EDE6E450E84
:10B36000DE6E040EDE6E070EDE6E64CADEFF63CA9A
:10B37000DEFFD9EC53F017EF5FF0970E0A01655D21
:10B380000001D8A4D8EF59F0D00EDE6E3F0EDE6E6D
:10B39000B00EDE6E450EDE6E080EDE6E0B0EDE6E3D
:10B3A00064CADEFF63CADEFFD9EC53F017EF5FF02B
:10B3B000990E0A01655D0001D8A4F3EF59F0D00E93
:10B3C000DE6E3F0EDE6EB00EDE6E450EDE6E0C0ED5
:10B3D000DE6E0F0EDE6E64CADEFF63CADEFFD9ECDE
:10B3E00053F017EF5FF09D0E0A01655D0001D8A4D0
:10B3F0000DEF5AF0A00EDE6E460EDE6EA00EDE6E73
:10B400004C0EDE6EDE6A060EDE6E64CADEFF63CAB6
:10B41000DEFFD9EC53F017EF5FF09F0E0A01655D78
:10B420000001D8A428EF5AF0A00EDE6E460EDE6EA4
:10B43000100EDE6E4E0EDE6E080EDE6E0F0EDE6E2F
:10B4400064CADEFF63CADEFFD9EC53F017EF5FF08A
:10B45000A30E0A01655D0001D8A442EF5AF0900ED8
:10B46000DE6E4E0EDE6E700EDE6E560EDE6EDE6A26
:10B47000020EDE6E64CADEFF63CADEFFD9EC53F053
:10B4800017EF5FF0A50E0A01655D0001D8A45DEF1E
:10B490005AF0900EDE6E4E0EDE6EA00EDE6E560E72
:10B4A000DE6E040EDE6E070EDE6E64CADEFF63CA59
:10B4B000DEFFD9EC53F017EF5FF0A70E0A01655DD0
:10B4C0000001D8A466EF5AF017EF5FF0AB0E0A0147
:10B4D000655D0001D8A46FEF5AF017EF5FF0AF0E73
:10B4E0000A01655D0001D8A48AEF5AF0600EDE6E95
:10B4F000700EDE6E600EDE6E710EDE6E060EDE6E9D
:10B50000090EDE6E64CADEFF63CADEFFD9EC53F0BB
:10B5100017EF5FF0B10E0A01655D0001D8A4A5EF39
:10B520005AF0600EDE6E700EDE6E600EDE6E710E14
:10B53000DE6E0A0EDE6E0B0EDE6E64CADEFF63CABE
:10B54000DEFFD9EC53F017EF5FF0B30E0A01655D33
:10B550000001D8A4C0EF5AF0600EDE6E700EDE6EF1
:10B56000600EDE6E710EDE6E0C0EDE6E0F0EDE6E87
:10B5700064CADEFF63CADEFFD9EC53F017EF5FF059
:10B58000B50E0A01655D0001D8A4C9EF5AF017EFA6
:10B590005FF0B70E0A01655D0001D8A4D2EF5AF042
:10B5A00017EF5FF0BB0E0A01655D0001D8A4DBEF69
:10B5B0005AF017EF5FF0BF0E0A01655D0001D8A4D5
:10B5C000E4EF5AF017EF5FF0C30E0A01655D00016A
:10B5D000D8A4EDEF5AF017EF5FF0C70E0A01655DD2
:10B5E0000001D8A4F6EF5AF017EF5FF0C90E0A0178
:10B5F000655D0001D8A4FFEF5AF017EF5FF0CD0EA4
:10B600000A01655D0001D8A41AEF5BF0A00EDE6EA2
:10B61000710EDE6E700EDE6E720EDE6E0A0EDE6E65
:10B620000F0EDE6E64CADEFF63CADEFFD9EC53F094
:10B6300017EF5FF0CF0E0A01655D0001D8A435EF6A
:10B640005BF0A00EDE6E710EDE6E700EDE6E720EA0
:10B65000DE6E0A0EDE6E0F0EDE6E64CADEFF63CA99
:10B66000DEFFD9EC53F017EF5FF0D10E0A01655DF4
:10B670000001D8A450EF5BF0B00EDE6E720EDE6EED
:10B68000400EDE6E730EDE6E0A0EDE6E0F0EDE6E86
:10B6900064CADEFF63CADEFFD9EC53F017EF5FF038
:10B6A000D30E0A01655D0001D8A46BEF5BF0B00E0C
:10B6B000DE6E720EDE6E400EDE6E730EDE6E0A0EF3
:10B6C000DE6E0F0EDE6E64CADEFF63CADEFFD9ECEB
:10B6D00053F017EF5FF0D50E0A01655D0001D8A4A5
:10B6E00085EF5BF0400EDE6E4D0EDE6E200EDE6EE0
:10B6F0004E0EDE6EDE6A050EDE6E64CADEFF63CAC3
:10B70000DEFFD9EC53F017EF5FF0D70E0A01655D4D
:10B710000001D8A4A0EF5BF0E00EDE6E600EDE6EDE
:10B72000E00EDE6E610EDE6E080EDE6E090EDE6E5F
:10B7300064CADEFF63CADEFFD9EC53F017EF5FF097
:10B74000D90E0A01655D0001D8A4BBEF5BF0E00EE5
:10B75000DE6E600EDE6EE00EDE6E610EDE6E0A0ED6
:10B76000DE6E0B0EDE6E64CADEFF63CADEFFD9EC4E
:10B7700053F017EF5FF0DB0E0A01655D0001D8A4FE
:10B78000D6EF5BF0E00EDE6E600EDE6E500EDE6E0B
:10B79000610EDE6E0C0EDE6E0D0EDE6E64CADEFF16
:10B7A00063CADEFFD9EC53F017EF5FF0DD0E0A013C
:10B7B000655D0001D8A4F1EF5BF0E00EDE6E600E77
:10B7C000DE6EB00EDE6E610EDE6E0E0EDE6E0F0EE3
:10B7D000DE6E64CADEFF63CADEFFD9EC53F017EFFA
:10B7E0005FF0DF0E0A01655D0001D8A40CEF5CF08C
:10B7F000800EDE6E610EDE6EF00EDE6E610EDE6EAF
:10B800000C0EDE6E0D0EDE6E64CADEFF63CADEFF56
:10B81000D9EC53F017EF5FF0E10E0A01655D00010E
:10B82000D8A427EF5CF0600EDE6E2A0EDE6E700E7E
:10B83000DE6E2C0EDE6E0E0EDE6E0F0EDE6E64CA37
:10B84000DEFF63CADEFFD9EC53F017EF5FF0E30EC3
:10B850000A01655D0001D8A441EF5CF0600EDE6E68
:10B860002A0EDE6EDE6A2C0EDE6E0C0EDE6E0D0E05
:10B87000DE6E64CADEFF63CADEFFD9EC53F017EF59
:10B880005FF0E50E0A01655D0001D8A45BEF5CF096
:10B89000500EDE6E610EDE6E600EDE6E650EDE6ECA
:10B8A000DE6A030EDE6E64CADEFF63CADEFFD9EC19
:10B8B00053F017EF5FF0E70E0A01655D0001D8A4B1
:10B8C00076EF5CF0500EDE6E610EDE6E600EDE6EA8
:10B8D000650EDE6E040EDE6E070EDE6E64CADEFFDF
:10B8E00063CADEFFD9EC53F017EF5FF0E90E0A01EF
:10B8F000655D0001D8A491EF5CF0700EDE6E620E03
:10B90000DE6EE00EDE6E680EDE6E080EDE6E0B0E74
:10B91000DE6E64CADEFF63CADEFFD9EC53F017EFB8
:10B920005FF0EB0E0A01655D0001D8A4ACEF5CF09E
:10B93000700EDE6E620EDE6E300EDE6E670EDE6E36
:10B940000C0EDE6E0F0EDE6E64CADEFF63CADEFF13
:10B95000D9EC53F017EF5FF0ED0E0A01655D0001C1
:10B96000D8A4C7EF5CF0200EDE6E690EDE6E400ECE
:10B97000DE6E6F0EDE6E0A0EDE6E0D0EDE6E64CAB9
:10B98000DEFF63CADEFFD9EC53F017EF5FF0EF0E76
:10B990000A01655D0001D8A4E1EF5CF0F00EDE6EF7
:10B9A000650EDE6EC00EDE6E680EDE6EDE6A030EA3
:10B9B000DE6E64CADEFF63CADEFFD9EC53F017EF18
:10B9C0005FF0F10E0A01655D0001D8A4FCEF5CF0A8
:10B9D000F00EDE6E650EDE6EC00EDE6E680EDE6E82
:10B9E000040EDE6E070EDE6E64CADEFF63CADEFF83
:10B9F000D9EC53F017EF5FF0F30E0A01655D00011B
:10BA0000D8A416EF5DF0200EDE6E690EDE6EE00E3D
:10BA1000DE6E6F0EDE6EDE6A030EDE6E64CADEFF61
:10BA200063CADEFFD9EC53F017EF5FF0F50E0A01A1
:10BA3000655D0001D8A431EF5DF0200EDE6E690E69
:10BA4000DE6E600EDE6E6B0EDE6E040EDE6E070EB8
:10BA5000DE6E64CADEFF63CADEFFD9EC53F017EF77
:10BA60005FF0F70E0A01655D0001D8A44CEF5DF0B0
:10BA7000E00EDE6E6B0EDE6E200EDE6E6E0EDE6E85
:10BA8000040EDE6E070EDE6E64CADEFF63CADEFFE2
:10BA9000D9EC53F017EF5FF0F90E0A01655D000174
:10BAA000D8A467EF5DF0200EDE6E690EDE6E200E0C
:10BAB000DE6E6F0EDE6E080EDE6E090EDE6E64CA7E
:10BAC000DEFF63CADEFFD9EC53F017EF5FF0FA0E2A
:10BAD0000A01655D0001D8A482EF5DF0700EDE6E94
:10BAE0006A0EDE6E700EDE6E700EDE6E080EDE6E9C
:10BAF000090EDE6E64CADEFF63CADEFFD9EC53F0C6
:10BB000017EF5FF0FB0E0A01655D0001D8A48BEF13
:10BB10005DF017EF5FF0FD0E0A01655D0001D8A42E
:10BB200094EF5DF017EF5FF00A0165290001D8A4DA
:10BB30009CEF5DF017EF5FF0020E0A01655D0001FA
:10BB4000D8A4B7EF5DF0900EDE6E730EDE6E100EB1
:10BB5000DE6E790EDE6E0C0EDE6E0F0EDE6E64CAC9
:10BB6000DEFF63CADEFFD9EC53F017EF5FF0040E7F
:10BB70000A01655D0001D8A4D1EF5DF0A00EDE6E74
:10BB8000710EDE6E800EDE6E760EDE6EDE6A010EE9
:10BB9000DE6E64CADEFF63CADEFFD9EC53F017EF36
:10BBA0005FF0060E0A01655D0001D8A4ECEF5DF0C0
:10BBB000A00EDE6E710EDE6E800EDE6E760EDE6E16
:10BBC000020EDE6E030EDE6E64CADEFF63CADEFFA7
:10BBD000D9EC53F017EF5FF0080E0A01655D000124
:10BBE000D8A407EF5EF0F00EDE6E670EDE6E800EFC
:10BBF000DE6E6F0EDE6E0E0EDE6E0F0EDE6E64CA31
:10BC0000DEFF63CADEFFD9EC53F017EF5FF00A0ED8
:10BC10000A01655D0001D8A421EF5EF0200EDE6E02
:10BC2000700EDE6E500EDE6E710EDE6EDE6A010E7E
:10BC3000DE6E64CADEFF63CADEFFD9EC53F017EF95
:10BC40005FF00C0E0A01655D0001D8A43CEF5EF0C8
:10BC5000200EDE6E700EDE6E500EDE6E710EDE6E2B
:10BC6000020EDE6E030EDE6E64CADEFF63CADEFF06
:10BC7000D9EC53F017EF5FF00E0E0A01655D00017D
:10BC8000D8A457EF5EF0200EDE6E700EDE6E500E02
:10BC9000DE6E710EDE6E040EDE6E050EDE6E64CAA2
:10BCA000DEFF63CADEFFD9EC53F017EF5FF0100E32
:10BCB0000A01655D0001D8A460EF5EF017EF5FF048
:10BCC000120E0A01655D0001D8A47BEF5EF0A00EA4
:10BCD000DE6E710EDE6EF00EDE6E780EDE6E040E1F
:10BCE000DE6E060EDE6E64CADEFF63CADEFFD9ECCE
:10BCF00053F017EF5FF0140E0A01655D0001D8A440
:10BD000096EF5EF0D00EDE6E2D0EDE6EC00EDE6E95
:10BD1000330EDE6E0A0EDE6E0F0EDE6E64CADEFFBE
:10BD200063CADEFFD9EC53F017EF5FF0160E0A017D
:10BD3000655D0001D8A4B0EF5EF0C00EDE6E790E36
:10BD4000DE6E200EDE6E7F0EDE6EDE6A050EDE6EAD
:10BD500064CADEFF63CADEFFD9EC53F017EF5FF071
:10BD6000180E0A01655D0001D8A4CBEF5EF0500EFD
:10BD7000DE6E790EDE6E800EDE6E7F0EDE6E0A0ED9
:10BD8000DE6E0F0EDE6E64CADEFF63CADEFFD9EC24
:10BD900053F017EF5FF01A0E0A01655D0001D8A499
:10BDA000E5EF5EF0900EDE6E730EDE6EDE6A760EEE
:10BDB000DE6E0A0EDE6E0B0EDE6E64CADEFF63CA36
:10BDC000DEFFD9EC53F017EF5FF01C0E0A01655D42
:10BDD0000001D8A4FEEF5EF0F00EDE6E0B0EDE6EFC
:10BDE000DE6A0E0EDE6EDE6A010EDE6E64CADEFFF5
:10BDF00063CADEFFD9EC53F017EF5FF01E0E0A01A5
:10BE0000655D0001D8A417EF5FF0100EDE6E140E12
:10BE1000DE6EE00EDE6E160EDE6E0A0EDE6E0B0EAF
:10BE2000DE6E64CADEFF63CADEFFD9EC53F0120097
:10BE3000FF0EDBCF66FADD52FF0EDBCF67FADD5275
:10BE40001AEE68F0A2EC02F0F00EDE6E0B0EDE6E63
:10BE500068CADEFF69CADEFF0E0EDE6E0F0EDE6EF2
:10BE600067CADEFF66CADEFFD9EC53F01200630E2C
:10BE7000DE6E190EDE6E0A0EDE6EF1EC54F0D70E99
:10BE8000DE6E6E0EDE6E080EDE6EF1EC54F0D90E34
:10BE9000DE6E6E0EDE6E0C0EDE6EF1EC54F0DF0E1A
:10BEA000DE6E800EDE6E0A0EDE6EF1EC54F0DB0EFE
:10BEB000DE6E650EDE6E0A0EDE6EF1EC54F0E30E01
:10BEC000DE6E3F0EDE6E0E0EDE6EF1EC54F0DD0E19
:10BED000DE6E650EDE6E0E0EDE6EF1EC54F01200BC
:10BEE000630EDE6E190EDE6E0A0EDE6EF1EC54F09D
:10BEF000D70EDE6E6E0EDE6E080EDE6EF1EC54F0C6
:10BF0000D90EDE6E6E0EDE6E0C0EDE6EF1EC54F0AF
:10BF1000DF0EDE6E800EDE6E0A0EDE6EF1EC54F089
:10BF2000DB0EDE6E650EDE6E0A0EDE6EF1EC54F098
:10BF30001200630EDE6E190EDE6E050EDE6EF1EC83
:10BF400054F0D70EDE6E6E0EDE6E030EDE6EF1EC7A
:10BF500054F0D90EDE6E6E0EDE6E070EDE6EF1EC64
:10BF600054F0DF0EDE6E800EDE6E050EDE6EF1EC3E
:10BF700054F0DB0EDE6E650EDE6E050EDE6EF1EC4D
:10BF800054F0E30EDE6E3F0EDE6E090EDE6EF1EC57
:10BF900054F0DD0EDE6E650EDE6E090EDE6EF1EC27
:10BFA00054F01200DE6A500EDE6E090EDE6EDE6A9E
:10BFB0000F0EDE6E050EDE6EDE6AD9EC53F0120057
:10BFC00012EC4AF0010E8C5DD8A4E9EF5FF056EF59
:10BFD00015F07A53D8A4F6EF5FF0CDEC69F00D0EB2
:10BFE000DE6E010EDE6EDE6AF1EC54F0010E7A6F49
:10BFF000030EDE6E58EC6CF03D0EDE6E74EC6CF0F1
:10C000000A016A6B00015B0E0A016A5D0001D8B08B
:10C0100015EF60F0DE68E4EC6CF00A0E82EC01F0E3
:10C020000A016A2B0001D8A4EDD73D0EDE6E74EC38
:10C030006CF00A016A6B00015B0E0A016A5D000187
:10C04000D8B02EEF60F0DE6AE4EC6CF00A0E82EC01
:10C0500001F00A016A2B0001D8A4EDD7320E82EC60
:10C0600001F080837DEF1FF01200FF0EDBCF6CFA32
:10C07000DD52FF0EDBCF6BFADD526BCADEFF58ECF0
:10C080006CF06CCADEFF74EC6CF00A016D6B0001A1
:10C09000080E0A016D5D0001D8B057EF60F0DE6850
:10C0A000E4EC6CF00A016D2B0001D8A4F0D712006B
:10C0B000FF0EDBCF6FFADD52FF0EDBCF6EFADD52E3
:10C0C0006ECADEFF66EC6CF06FCADEFF9EEC6CF0B1
:10C0D0000A01706B0001060E0A01705D0001D8B004
:10C0E0007BEF60F01F0EDE6EF2EC6CF00A01702B3D
:10C0F0000001D8A4EFD71200FF0EDBCF72FADD5299
:10C10000FF0EDBCF71FADD5271CADEFF58EC6CF026
:10C1100072CADEFF74EC6CF00A01736B0001080E4A
:10C120000A01735D0001D8B09EEF60F0DE6AE4ECB6
:10C130006CF00A01732B0001D8A4F0D71200FF0E97
:10C14000DBCF75FADD52FF0EDBCF74FADD5274CA15
:10C15000DEFF66EC6CF075CADEFF9EEC6CF00A0147
:10C16000766B0001080E0A01765D0001D8B0C1EFC0
:10C1700060F0DE6AF2EC6CF00A01762B0001D8A4C4
:10C18000F0D71200FF0EDBCF78FADD52FF0EDBCFC7
:10C1900077FADD5277CADEFF66EC6CF078CADEFF14
:10C1A0009EEC6CF00A01796B0001050E0A01795DC5
:10C1B0000001D8B0E5EF60F0F00EDE6EF2EC6CF04E
:10C1C0000A01792B0001D8A4EFD71200FF0EDBCFB4
:10C1D0007BFADD52FF0EDBCF7AFADD527ACADEFF40
:10C1E00066EC6CF07BCADEFF9EEC6CF00A017C6BA7
:10C1F0000001050E0A017C5D0001D8B008EF61F076
:10C20000DE6AF2EC6CF00A017C2B0001D8A4F0D7B6
:10C210001200FF0EDBCF7EFADD52FF0EDBCF7DFA80
:10C22000DD527DCADEFF58EC6CF07ECADEFF74EC96
:10C230006CF00A017F6B0001050E0A017F5D0001B1
:10C24000D8B02CEF61F00F0EDE6EE4EC6CF00A015A
:10C250007F2B0001D8A4EFD71200FF0EDBCF81FAAD
:10C26000DD52FF0EDBCF80FADD5280CADEFF58ECD4
:10C270006CF081CADEFF74EC6CF00A01826B000185
:10C28000050E0A01825D0001D8B04FEF61F0DE6A51
:10C29000E4EC6CF00A01822B0001D8A4F0D7120064
:10C2A0000A01836B0001080E0A01835D0001D8B00A
:10C2B0007CEF61F083CADEFF58EC6CF00A01846BFE
:10C2C00084CADEFF000174EC6CF00A01856B00018A
:10C2D000170E0A01855D0001D8B077EF61F0DE6AC4
:10C2E000E4EC6CF00A01852B0001D8A4F0D70A0118
:10C2F000832B0001D8A4D6D70A01836B0001080E56
:10C300000A01835D0001D8B0A9EF61F083CADEFFA6
:10C3100066EC6CF0080E0A01846F84CADEFF00012F
:10C320009EEC6CF00A01856B0001170E0A01855D19
:10C330000001D8B0A4EF61F0DE6AF2EC6CF00A0103
:10C34000852B0001D8A4F0D70A01832B0001D8A4C3
:10C35000D5D71200040E0A01866F0001060E0A01ED
:10C36000865D0001D8B0D4EF61F086CADEFF66ECCE
:10C370006CF01C0EDE6E9EEC6CF00A01876B000107
:10C38000260E0A01875D0001D8B0CFEF61F0DE6AAA
:10C39000F2EC6CF00A01872B0001D8A4F0D70A0157
:10C3A000862B0001D8A4D9D712001200030E0A016F
:10C3B000886F0001060E0A01885D0001D8B0FFEF0A
:10C3C00061F088CADEFF58EC6CF0DE6A74EC6CF049
:10C3D0000A018B6B0001A00E0A018B5D0001D8B031
:10C3E000FAEF61F0DE6AE4EC6CF00A018B2B0001DD
:10C3F000D8A4F0D70A01882B0001D8A4DAD7180EE8
:10C400008FEC01F00A01896B00019F0E0A01895D22
:10C410000001D8B042EF62F0020E0A01886F0001FD
:10C42000070E0A01885D0001D8B03CEF62F089CAAE
:10C43000DEFF74EC6CF088CADEFF58EC6CF0030E83
:10C440000A01885D0001D8A42CEF62F03F0E0A01BA
:10C450008A6F00012EEF62F00A018A6900018ACA20
:10C46000DEFFE4EC6CF08ACADEFFE4EC6CF00A015B
:10C47000882B0001D8A4D3D74F0E0A0189270001C9
:10C48000D8A0C2D7180E8FEC01F012001AEE8CF073
:10C49000A2EC02F00A018D530001D8A457EF62F01C
:10C4A000140E0A018C5D0001D8A05BEF62F00A0156
:10C4B0008D6B130E8C6F0001520E7D5DD8A467EF5B
:10C4C00062F0500E0A018E6F000173EF62F0D89097
:10C4D0000A018C352B6E8D352C6ED8902B362C3670
:10C4E0002B504D088E6F00010A018D518C110001F7
:10C4F000D8B4B5EF62F0030E0A018F6F0001060E8B
:10C500000A018F5D0001D8B0B5EF62F08FCADEFF7F
:10C5100058EC6CF08ECADEFF74EC6CF00A01906B84
:10C5200000010A018D530001D8A49EEF62F00A01B8
:10C5300090518C5D0001D8A0B0EF62F0DE68E4ECB1
:10C540006CF0CF0EDE6EE4EC6CF0DE68E4EC6CF0C8
:10C55000DE68E4EC6CF00A01902B0001D8A4E0D76F
:10C560000A018F2B0001D8A4C9D7180E8FEC01F057
:10C570001200FF0EDBCF9DFADD52D89680A3D8863D
:10C58000D8B6C6EF62F00A01936B926B00010A0104
:10C590000D99010E9D5D0001D8A41AEF63F00A0108
:10C5A000916B0001800E0A01915D0001D8B018EF77
:10C5B00063F002EEB9F0D8900A019135E926000E39
:10C5C000EA22EECF0DF0EFCF0EF00E500A0DF3CFB2
:10C5D0000CF00D500A0DF3CF0BF0F4500C2604EEC6
:10C5E000BDF0D8909135E926000EEA220BC0EEFF8F
:10C5F0000CC0EFFF04EEBDF0D8909135E926000E97
:10C60000EA22EECF0BF0EFCF0CF0000112EF63F057
:10C6100004EEBDF0D8900A019135E926000EEA2219
:10C62000EE68EF6800010A01912B0001D8A4B9D788
:10C630002EEF64F0020E0A019D5D0001D8A46CEF9C
:10C6400063F00A01916B0001800E0A01915D000107
:10C65000D8B06AEF63F001EEB9F0D8900A019135D5
:10C66000E926000EEA22EECF0DF0EFCF0EF00E50CD
:10C670000A0DF3CF0CF00D500A0DF3CF0BF0F45070
:10C680000C2604EEBDF0D8909135E926000EEA2282
:10C690000BC0EEFF0CC0EFFF04EEBDF0D89091355B
:10C6A000E926000EEA22EECF0BF0EFCF0CF00001EE
:10C6B00064EF63F004EEBDF0D8900A019135E926ED
:10C6C000000EEA22EE68EF6800010A01912B0001DA
:10C6D000D8A4B9D72EEF64F0030E0A019D5D0001C6
:10C6E000D8A42EEF64F00A01916B0001800E0A01BC
:10C6F000915D0001D8B0A2EF63F003EEB9F0D890DD
:10C700000A019135E926000EEA22EECF0DF0EFCFB7
:10C710000EF00E50640DF3CF0CF00D50640DF3CFFE
:10C720000BF0F4500C2604EEBDF0D8909135E926BC
:10C73000000EEA220BC0EEFF0CC0EFFF912B0001B0
:10C74000D8A4D3D70A01916B0001800E0A01915D34
:10C750000001D8B0E3EF63F004EEBDF0D8900A0119
:10C760009135E926000EEA22EECF0BF0EFCF0CF068
:10C77000750E0C5C300ED8B40B5C0001D8B0DEEF47
:10C7800063F004EEBDF0D8900A019135E926000E61
:10C79000EA22EECF0BF0EFCF0CF0270E0C5C00017D
:10C7A000D8A0DDEF63F0D8A4DBEF63F0100E0B5CD4
:10C7B000D8A0DDEF63F00A010D8900010A01912B79
:10C7C0000001D8A4C1D7D8960A010DB9D8860001B6
:10C7D000D8B62EEF64F0010E0A01916F0001800EB1
:10C7E0000A01915D0001D8B02EEF64F004EEBDF0B7
:10C7F000D8900A019135E926000EEA22EECF0BF01F
:10C80000EFCF0CF0270E0C5C0F0ED8B40B5C0001C0
:10C81000D8B028EF64F004EEBDF0D8900A0191354D
:10C82000E926000EEA22EECF0DF0EFCF0EF0A00EBB
:10C830000D240B6E8C0E0E200C6E04EEBDF0D89005
:10C840009135E926000EEA220BC0EEFF0CC0EFFF87
:10C8500000010A01912B0001D8A4C0D70A01936BF3
:10C86000070E926F976996699F6B0001800E0A010F
:10C870009F5D0001D8B084EF64F004EEBDF0D89065
:10C880000A019F35E926000EEA22EECF0BF0EFCF2A
:10C890000CF00B50925D0C5093590001D8B05DEF35
:10C8A00064F004EEBDF0D8900A019F35E926000E31
:10C8B000EA22EECF92FAEFCF93FA000104EEBDF038
:10C8C000D8900A019F35E926000EEA22EECF0BF040
:10C8D000EFCF0CF096510B5C97510C580001D8B07B
:10C8E0007EEF64F004EEBDF0D8900A019F35E92692
:10C8F000000EEA22EECF96FAEFCF97FA00010A0176
:10C900009F2B0001D8A4B1D7010EBE5DD8A49FEF24
:10C9100064F00A019651925D2B6E975193592C6EDB
:10C920002CC01AF02BC019F01E6A070E1D6E32ECD7
:10C9300002F0946F1AC095FA0001ACEF64F093CA4C
:10C940001AF092CA19F01E6A070E1D6E32EC02F040
:10C950000A01946F1AC095FA00017F0E0A01916FC7
:10C960000001010EBE5DD8A416EF65F00A019151D9
:10C970007F080D6E04EEBDF0D8900D34E926000E50
:10C98000EA22EECF0BF0EFCF0CF096510B5C2B6E42
:10C9900097510C582C6E2CC01AF02BC019F095CA68
:10C9A0001EF094CA1DF032EC02F0986F1AC099FA8A
:10C9B00091517F080D6E04EEBDF0D8900D34E9263C
:10C9C000000EEA22EECF0BF0EFCF0CF00CC02CF0F3
:10C9D0000BC02BF096512B5E97512C5A2CC01AF09D
:10C9E0002BC019F095CA1EF094CA1DF032EC02F06B
:10C9F00022C02CF021C02BF02C500A0DF3CF2CF0CC
:10CA00002B500A0DF3CF2BF0F4502C262CC01AF02B
:10CA10002BC019F095CA1EF094CA1DF032EC02F03A
:10CA20009A6F1AC09BFA000169EF65F00A019151F3
:10CA30007F080D6E04EEBDF0D8900D34E926000E8F
:10CA4000EA22EECF0BF0EFCF0CF00CC01AF00BC0C7
:10CA500019F095CA1EF094CA1DF032EC02F0986FDE
:10CA60001AC099FA91517F080D6E04EEBDF0D8906E
:10CA70000D34E926000EEA22EECF0BF0EFCF0CF0DA
:10CA80000CC02CF00BC02BF02CC01AF02BC019F0EE
:10CA900095CA1EF094CA1DF032EC02F022C02CF0B0
:10CAA00021C02BF02C500A0DF3CF2CF02B500A0D87
:10CAB000F3CF2BF0F4502C262CC01AF02BC019F019
:10CAC00095CA1EF094CA1DF032EC02F09A6F1AC09B
:10CAD0009BFA00010A019C6B0001070E0A019C5D94
:10CAE0000001D8B03BEF66F09CCADEFF58EC6CF05A
:10CAF00091CADEFF74EC6CF00A0199530001D8A4CE
:10CB000089EF65F00A0198519C5D0001D8B08EEF65
:10CB100065F00A019E6900019EEF65F00A019953D4
:10CB20000001D8A49DEF65F00A019C51985D0001B9
:10CB3000D8B09DEF65F00A019E6B00010A01995182
:10CB40000001D8A432EF66F00A0198519C5D000103
:10CB5000D8A432EF66F00A019B519A110001D8A4C3
:10CB6000B7EF65F00A019E6B000132EF66F00A0133
:10CB70009A059B110001D8A4C4EF65F0010E0A01CB
:10CB80009E6F000132EF66F00A019A51020A9B1172
:10CB90000001D8A4D2EF65F0030E0A019E6F0001D8
:10CBA00032EF66F00A019A51030A9B110001D8A4E2
:10CBB000E0EF65F0070E0A019E6F000132EF66F0AC
:10CBC0000A019A51040A9B110001D8A4EEEF65F006
:10CBD0001F0E0A019E6F000132EF66F00A019A51A2
:10CBE000050A9B110001D8A4FCEF65F01F0E0A0195
:10CBF0009E6F000132EF66F00A019A51060A9B11FE
:10CC00000001D8A40AEF66F03F0E0A019E6F0001F2
:10CC100032EF66F00A019A51070A9B110001D8A46D
:10CC200018EF66F03F0E0A019E6F000132EF66F0CA
:10CC30000A019A51080A9B110001D8A426EF66F058
:10CC40007F0E0A019E6F000132EF66F00A019A51D1
:10CC5000090A9B110001D8A431EF66F07F0E0A018A
:10CC60009E6F00019ECADEFFE4EC6CF00A019C2B73
:10CC70000001D8A431D7010E0A01915F0001D8B09C
:10CC80006FD612001200FF0EDBCFA0FADD52FF0EAE
:10CC9000DBCFA1FADD52FF0EDBCFA2FADD52A0CA34
:10CCA000DEFFA1CADEFFA2CADEFFDE6A74EC66F018
:10CCB0001200FF0EDBCFA4FADD52FF0EDBCFA3FA8A
:10CCC000DD52A3CADEFFA4CADEFFDE6A010EDE6EFD
:10CCD00074EC66F0A3CADEFFA4CADEFFDE6A020EB1
:10CCE000DE6E74EC66F01200FF0EDBCFA6FADD52AA
:10CCF000FF0EDBCFA7FADD52FF0EDBCFA8FADD5225
:10CD0000FF0EDBCFAAFADD520A01AB6B0001060E63
:10CD10000A01AB5D0001D8B0CBEF67F0A8CAA9FA51
:10CD2000A9CADEFF74EC6CF0080E0A01A825A96FF1
:10CD3000A9CADEFF00019EEC6CF00A01B16B000194
:10CD4000060E0A01B15D0001D8B0C6EF67F0AACAAD
:10CD5000DEFFABCADEFFDE6A30EC6AF087C019F096
:10CD60000A01B151E82A1932E82EFDD7010ED8A0E8
:10CD7000E86AB081E8A0B09187C019F0B151E82A03
:10CD80001932E82EFDD7010ED8A0E86AB083E8A0DA
:10CD9000B09387C019F0B151E82A1932E82EFDD7B7
:10CDA000010ED8A0E86AB085E8A0B09587C019F058
:10CDB000B151E82A1932E82EFDD7010ED8A0E86A51
:10CDC000B087E8A0B09787C019F0B151E82A1932AE
:10CDD000E82EFDD7010ED8A0E86AB089E8A0B09986
:10CDE00087C019F0B151E82A1932E82EFDD7010E9B
:10CDF000D8A0E86AB08BE8A0B09B87C019F0B15109
:10CE0000E82A1932E82EFDD7010ED8A0E86AB08DC5
:10CE1000E8A0B09D87C019F0B151E82A1932E82E78
:10CE2000FDD7010ED8A0E86AB08FE8A0B09FA65346
:10CE30000001D8A423EF67F00A01A751AB25AC6F1E
:10CE400000014BEF67F0010E0A01A65D0001D8A4B6
:10CE500037EF67F00A01AB51020DF3CF2BF0F4CF9F
:10CE60002CF0A7512B24AC6F00014BEF67F0020EA2
:10CE70000A01A65D0001D8A44AEF67F02C6AABCA8C
:10CE80002BF0D8902B362C362B4A2C2A0A01A7518E
:10CE90002B24AC6F0001080E0A01AC5D0001D8A084
:10CEA00089EF67F01E6AACCA1DF0E60EF66ECE0E74
:10CEB000F76E2168212A21500708D8A083EF67F078
:10CEC0000900F5CF19F00900F5CF1AF00900F55067
:10CED0000900A3EC01F0020E12EC00F0EBE021C01F
:10CEE000B3FA83EF67F00F0000000E0000000D00A2
:10CEF00000000C0000000B0000000A000000090008
:10CF0000000008000000B3CADEFF66EC6CF08FEF93
:10CF100067F0ACCAB3FAB3CADEFF58EC6CF00A0192
:10CF2000A6530001D8A49BEF67F0050E0A01AD6F70
:10CF300000019EEF67F0090E0A01AD6F00010A01C2
:10CF4000AE6B00010A01AE51AD5D0001D8A0C1EF8A
:10CF500067F0B0CAB2FA080E0A01AC5D0001D8A0B1
:10CF6000B8EF67F0B2CADEFFF2EC6CF0BCEF67F02E
:10CF7000B2CADEFFE4EC6CF00A01AE2B0001D8A4CB
:10CF8000E0D70A01B12B0001D8A4D9D60A01AB2BF6
:10CF90000001D8A4BBD61200FF0EDBCFB4FADD52DD
:10CFA000FF0EDBCFB5FADD52FF0EDBCFB6FADD5256
:10CFB0000A01B86B0001060E0A01B85D0001D8B085
:10CFC00089EF68F0B5CAB7FAB7CADEFF74EC6CF047
:10CFD0000A01BE6B0001060E0A01BE5D0001D8B059
:10CFE00082EF68F0B6CADEFFB8CADEFF010EDE6E61
:10CFF00030EC6AF087C019F00A01BE51E82A1932F4
:10D00000E82EFDD7010ED8A0E86ABD81E8A0BD9149
:10D0100087C019F0BE51E82A1932E82EFDD7010E5B
:10D02000D8A0E86ABD83E8A0BD9387C019F0BE51BF
:10D03000E82A1932E82EFDD7010ED8A0E86ABD858E
:10D04000E8A0BD9587C019F0BE51E82A1932E82E34
:10D05000FDD7010ED8A0E86ABD87E8A0BD9788C0BB
:10D0600019F0BE51E82A1932E82EFDD7010ED8A0DA
:10D07000E86ABD89E8A0BD9988C019F0BE51E82AC8
:10D080001932E82EFDD7010ED8A0E86ABD8BE8A0C2
:10D09000BD9B88C019F0BE51E82A1932E82EFDD791
:10D0A000010ED8A0E86ABD8DE8A0BD9D88C019F02A
:10D0B000BE51E82A1932E82EFDD7010ED8A0E86A41
:10D0C000BD8FE8A0BD9FB4CADEFF000158EC6CF034
:10D0D0000A01BB6B0001040E0A01BB5D0001D8B060
:10D0E0007DEF68F0BDCABFFABFCADEFFE4EC6CF0AA
:10D0F0000A01BB2B0001D8A4EDD70A01BE2B000109
:10D10000D8A468D70A01B42B020EB8270001D8A012
:10D1100051D71200FF0EDBCFC0FADD52FF0EDBCF7E
:10D12000C1FADD52FF0EDBCFC3FADD520A01C46B38
:10D130000001060E0A01C45D0001D8B09BEF69F042
:10D14000C1CAC2FAC2CADEFF74EC6CF0080E0A0152
:10D15000C125C26FC2CADEFF00019EEC6CF00A015D
:10D16000C96B0001060E0A01C95D0001D8B096EF37
:10D1700069F0C3CADEFFC4CADEFFDE6A30EC6AF0C3
:10D1800087C019F00A01C951E82A1932E82EFDD7E3
:10D19000010ED8A0E86AC881E8A0C89187C019F03C
:10D1A000C951E82A1932E82EFDD7010ED8A0E86A45
:10D1B000C883E8A0C89387C019F0C951E82A19327A
:10D1C000E82EFDD7010ED8A0E86AC885E8A0C8956A
:10D1D00087C019F0C951E82A1932E82EFDD7010E8F
:10D1E000D8A0E86AC887E8A0C89787C019F0C951D5
:10D1F000E82A1932E82EFDD7010ED8A0E86AC889BE
:10D20000E8A0C89987C019F0C951E82A1932E82E58
:10D21000FDD7010ED8A0E86AC88BE8A0C89B87C0DC
:10D2200019F0C951E82A1932E82EFDD7010ED8A00D
:10D23000E86AC88DE8A0C89D87C019F0C951E82ADE
:10D240001932E82EFDD7010ED8A0E86AC88FE8A0F1
:10D25000C89FC051C425C56F080EC55D0001D8A088
:10D2600069EF69F01E6AC5CA1DF0A60EF66ED20EF1
:10D27000F76E2168212A21500708D8A063EF69F0D2
:10D280000900F5CF19F00900F5CF1AF00900F550A3
:10D290000900A3EC01F0020E12EC00F0EBE021C05B
:10D2A000CBFA63EF69F00F0000000E0000000D00E4
:10D2B00000000C0000000B0000000A000000090044
:10D2C000000008000000CBCADEFF66EC6CF06FEFD8
:10D2D00069F0C5CACBFACBCADEFF58EC6CF00A0184
:10D2E000C66B0001030E0A01C65D0001D8B091EFC4
:10D2F00069F0C8CACAFA080E0A01C55D0001D8A0C3
:10D3000088EF69F0CACADEFFF2EC6CF08CEF69F0CE
:10D31000CACADEFFE4EC6CF00A01C62B0001D8A4F7
:10D32000E0D70A01C92B0001D8A41BD70A01C42BDE
:10D330000001D8A4FDD612000A01CC6B0001080E32
:10D340000A01CC5D0001D8B0CCEF69F0CCCADEFF99
:10D3500058EC6CF00A01CD6BCDCADEFF000174EC15
:10D360006CF00A01CE6B0001A00E0A01CE5D000137
:10D37000D8B0C7EF69F00A01CF6BCFCADEFF00015A
:10D38000E4EC6CF00A01CE2B0001D8A4ECD70A0122
:10D39000CC2B0001D8A4D2D712000A01D06B000117
:10D3A000080E0A01D05D0001D8B0FDEF69F0D0CAC7
:10D3B000DEFF58EC6CF00A01D16BD1CADEFF000130
:10D3C00074EC6CF00A01D26B0001A00E0A01D25D70
:10D3D0000001D8B0F8EF69F00A01D36BD3CADEFFC1
:10D3E0000001E4EC6CF00A01D22B0001D8A4ECD7C8
:10D3F0000A01D02B0001D8A4D2D70A01D06B0001BA
:10D40000080E0A01D05D0001D8B02FEF6AF0D0CA33
:10D41000DEFF66EC6CF0080E0A01D16FD1CADEFFA8
:10D4200000019EEC6CF0070E0A01D26F0001A80EFD
:10D430000A01D25D0001D8B02AEF6AF00A01D36B6D
:10D44000D3CADEFF0001F2EC6CF00A01D22B00011E
:10D45000D8A4ECD70A01D02B0001D8A4D0D7120051
:10D46000FF0EDB50DD520A010D8BE8A00D9BFF0E75
:10D47000DBCFD4FADD52FF0EDBCFD5FADD52D55328
:10D480000001D8A462EF6AF0020E0A01D42500EE72
:10D49000CBF0EB500001876FD8960A010DABD88610
:10D4A0000001D8B660EF6AF0020E0A01D4252C6A9A
:10D4B0002B6E2C362B2800EECBF0EB500001886F42
:10D4C00007EF6CF0010E0A01D55D0001D8A48DEFC5
:10D4D0006AF0020E0A01D4252C6A2B6E2C36060E39
:10D4E0002B2400EECBF0EB500001876FD8960A0199
:10D4F0000DABD8860001D8B68BEF6AF0020E0A0198
:10D50000D4252C6A2B6E2C36070E2B2400EECBF084
:10D51000EB500001886F07EF6CF0020E0A01D55D39
:10D520000001D8A4B8EF6AF0020E0A01D4252C6AD3
:10D530002B6E2C360C0E2B2400EECBF0EB500001A2
:10D54000876FD8960A010DABD8860001D8B6B6EF22
:10D550006AF0020E0A01D4252C6A2B6E2C360D0EB1
:10D560002B2400EECBF0EB500001886F07EF6CF03E
:10D57000030E0A01D55D0001D8A4E3EF6AF0020EA4
:10D580000A01D4252C6A2B6E2C36120E2B2400EEA9
:10D59000CBF0EB500001876FD8960A010DABD8860F
:10D5A0000001D8B6E1EF6AF0020E0A01D4252C6A18
:10D5B0002B6E2C36130E2B2400EECBF0EB5000011B
:10D5C000886F07EF6CF0040E0A01D55D0001D8A446
:10D5D0000EEF6BF0020E0A01D4252C6A2B6E2C364E
:10D5E000180E2B2400EECBF0EB500001876FD8967D
:10D5F0000A010DABD8860001D8B60CEF6BF0020E15
:10D600000A01D4252C6A2B6E2C36190E2B2400EE21
:10D61000CBF0EB500001886F07EF6CF0050E0A01AC
:10D62000D55D0001D8A439EF6BF0020E0A01D425B4
:10D630002C6A2B6E2C361E0E2B2400EECBF0EB50FA
:10D640000001876FD8960A010DABD8860001D8B6C5
:10D6500037EF6BF0020E0A01D4252C6A2B6E2C36A4
:10D660001F0E2B2400EECBF0EB500001886F07EF6C
:10D670006CF0060E0A01D55D0001D8A464EF6BF0D2
:10D68000020E0A01D4252C6A2B6E2C36240E2B2474
:10D6900000EECBF0EB500001876FD8960A010DAB7E
:10D6A000D8860001D8B662EF6BF0020E0A01D425CD
:10D6B0002C6A2B6E2C36250E2B2400EECBF0EB5073
:10D6C0000001886F07EF6CF0070E0A01D55D0001BD
:10D6D000D8A48FEF6BF0020E0A01D4252C6A2B6EB2
:10D6E0002C362A0E2B2400EECBF0EB500001876F76
:10D6F000D8960A010DABD8860001D8B68DEF6BF035
:10D70000020E0A01D4252C6A2B6E2C362B0E2B24EC
:10D7100000EECBF0EB500001886F07EF6CF0080EC5
:10D720000A01D55D0001D8A4BAEF6BF0020E0A0120
:10D73000D4252C6A2B6E2C36300E2B2400EECBF029
:10D74000EB500001876FD8960A010DABD886000117
:10D75000D8B6B8EF6BF0020E0A01D4252C6A2B6EF6
:10D760002C36310E2B2400EECBF0EB500001886FED
:10D7700007EF6CF0090E0A01D55D0001D8A4E5EFB2
:10D780006BF0020E0A01D4252C6A2B6E2C36360E55
:10D790002B2400EECBF0EB500001876FD8960A01E6
:10D7A0000DABD8860001D8B6E3EF6BF0020E0A018C
:10D7B000D4252C6A2B6E2C36370E2B2400EECBF0A2
:10D7C000EB500001886F07EF6CF0020E0A01D425C0
:10D7D0002C6A2B6E2C363C0E2B2400EECBF0EB503B
:10D7E0000001876FD8960A010DABD8860001D8B624
:10D7F00007EF6CF0020E0A01D4252C6A2B6E2C3632
:10D800003D0E2B2400EECBF0EB500001886F120090
:10D810008490320E82EC01F084808A0E0A01D66F69
:10D82000D6CADEFF0001C8EC6CF00A01D66BD6CA7E
:10D83000DEFF0001C8EC6CF08A0E0A01D66FD6CA72
:10D84000DEFF0001D6EC6CF00A01D66BD6CADEFF13
:10D850000001D6EC6CF0840E0A01D66FD6CADEFF4A
:10D860000001C8EC6CF0840E0A01D66FD6CADEFF48
:10D870000001D6EC6CF0A00E0A01D66FD6CADEFF0E
:10D880000001C8EC6CF0A10E0A01D66FD6CADEFF0B
:10D890000001D6EC6CF0DE6A58EC6CF0DE6A66ECE7
:10D8A0006CF0DE6A74EC6CF0DE6A9EEC6CF01200D8
:10D8B000FF0EDBCFD7FADD52B00E0A01D725D86FA5
:10D8C000D8CADEFF0001C8EC6CF01200FF0EDBCFFF
:10D8D000D9FADD52B00E0A01D925DA6FDACADEFFB5
:10D8E0000001D6EC6CF01200FF0EDBCFDBFADD524C
:10D8F0000A01DB390F0BDC6F100EDC11DD6FDDCAA6
:10D90000DEFF0001C8EC6CF00A01DB39F00BDC6FC4
:10D91000000EDC112B6E000E2C6E2C30F46E2B30B2
:10D92000F36EF432F332F432F332F432F330DD6F6B
:10D93000DDCADEFF0001C8EC6CF01200FF0EDBCF89
:10D94000DEFADD520A01DE390F0BDF6F100EDF1138
:10D95000E06FE0CADEFF0001D6EC6CF00A01DE39B0
:10D96000F00BDF6F000EDF112B6E000E2C6E2C30D3
:10D97000F46E2B30F36EF432F332F432F332F432CD
:10D98000F330E06FE0CADEFF0001D6EC6CF012006D
:10D99000FF0EDBCFE1FADD52849A86908492E1CAD1
:10D9A00083FF000084828680848A1200FF0EDBCF12
:10D9B000E2FADD52849A84988492E2CA83FF0000DE
:10D9C00084828488848A1200FF0EDBCFE3FADD5262
:10D9D000848A86908492E3CA83FF000084828680D2
:10D9E000849A1200FF0EDBCFE4FADD52848A849819
:10D9F0008492E4CA83FF000084828488849A12009F
:10DA0000A90EDE6EC5DFA90EDE6ED0DF1200A80EF5
:10DA1000DE6EBEDFA80EDE6EC9DF1200AF0EDE6E58
:10DA2000B7DFAF0EDE6EC2DF1200AE0EDE6EB0DF0D
:10DA3000AE0EDE6EBBDF1200A70EDE6EA9DFA70EF4
:10DA4000DE6EB4DF1200A60EDE6EA2DFA60EDE6E64
:10DA5000ADDF1200848C86808488848A84828480EE
:10DA6000C80E82EC01F0D4DEA00E0A01E56FE5CA13
:10DA7000DEFF00018DDFA00E0A01E56FE5CADEFFC3
:10DA8000000194DFC40E0A01E56FE5CADEFF000164
:10DA90007FDFC40E0A01E56FE5CADEFF000186DF05
:10DAA000A60E0A01E56FE5CADEFF000171DFA60ED2
:10DAB0000A01E56FE5CADEFF000178DFA40E0A0166
:10DAC000E56FE5CADEFF000163DFA40E0A01E56F22
:10DAD000E5CADEFF00016ADF6D0E0A01E56FE5CAE7
:10DAE000DEFF000155DFF00E0A01E56FE5CADEFF3B
:10DAF00000014EDF6D0E0A01E56FE5CADEFF000191
:10DB000055DFF00E0A01E56FE5CADEFF00014EDFCA
:10DB1000240E0A01E56FE5CADEFF000139DF240E9D
:10DB20000A01E56FE5CADEFF000140DF810E0A0150
:10DB3000E56FE5CADEFF00012BDF3C0E0A01E56F51
:10DB4000E5CADEFF000124DF810E0A01E56FE5CAA8
:10DB5000DEFF00012BDF3C0E0A01E56FE5CADEFFA8
:10DB6000000124DF480E0A01E56FE5CADEFF00016F
:10DB70000FDF480E0A01E56FE5CADEFF000116DF80
:10DB8000720E0A01E56FE5CADEFF000101DF720EC9
:10DB90000A01E56FE5CADEFF000108DFAB0E0A01EE
:10DBA000E56FE5CADEFF0001F3DEAB0E0A01E56FAB
:10DBB000E5CADEFF0001FADE500E0A01E56FE5CA94
:10DBC000DEFF0001E5DE500E0A01E56FE5CADEFF6B
:10DBD0000001ECDE2F0E0A01E56FE5CADEFF000151
:10DBE000D7DE2F0E0A01E56FE5CADEFF0001DEDE9B
:10DBF00015DF120080A0FEEF6DF08090020E6BEC3E
:10DC000001F001010F6F8688180E82EC01F0868604
:10DC1000180E82EC01F08696180E82EC01F08698C0
:10DC2000010E1E6EF40E83EC01F08698859E020EA6
:10DC30000F5D0001D8A420EF6EF0858E2BEF6EF003
:10DC4000030E01010F5D0001D8A42AEF6EF0858E4E
:10DC50002BEF6EF0859E820E026E400E096E2A6AD0
:10DC6000540E296E066A056A200E016E480EBEEC3F
:10DC700000F0570EBEEC00F0720EBEEC00F0650E28
:10DC8000BEEC00F0760EBEEC00F03D0EBEEC00F0F7
:10DC9000820E026E400E096E2A6A540E296E066AC2
:10DCA000056A200E016E01010F5121EC00F0820E79
:10DCB000026E400E096E2A6A540E296E066A056AC3
:10DCC000200E016E0D0EBEEC00F0820E026E400EB4
:10DCD000096E2A6A540E296E066A056A200E016EC4
:10DCE0000A0EBEEC00F08496848486948692010E1F
:10DCF0001E6EF40E83EC01F00001ACDE0DEC6CF056
:10DD0000CDEC69F0D2EC5FF0070E1E6ED00E83EC06
:10DD100001F0CB6BCC6B3F0ECD6F210ECE6F210E81
:10DD2000CF6F210ED06F210ED16F3F0ED26F040E38
:10DD3000D36F040ED46F040ED56F040ED66F040E8D
:10DD4000D76F040ED86F3F0ED96F010EDA6F010E38
:10DD5000DB6F3F0EDC6F200EDD6F3F0EDE6F3F0E80
:10DD6000DF6F200EE06F200EE16F3C0EE26F200EA1
:10DD7000E36F3F0EE46F200EE56F200EE66F200E7E
:10DD8000E76F3F0EE86F210EE96F210EEA6F3F0E3D
:10DD9000EB6F200EEC6F200EED6F3F0EEE6F010E5D
:10DDA000EF6F3F0EF06F3F0EF16F210EF26F210EFD
:10DDB000F36F3F0EF46F010EF56F3F0EF66F200EFE
:10DDC000F76F200EF86F200EF96F200EFA6F200EFD
:10DDD000FB6F3F0EFC6F3F0EFD6F210EFE6F210E9D
:10DDE000FF6F3F0E0101006F210E016F3F0E026FAA
:10DDF0003F0E036F200E046F200E056F3F0E066F5F
:10DE0000210E076F3F0E086F096B0A6B0B6B0C6BD3
:10DE10000D6B0E6B0001CDEC69F010EC10F0460EAE
:10DE20006BEC01F00801D46FD4290001D8A421EFD4
:10DE30006FF00801D46BAA6A460EA96ED45174EC37
:10DE400001F000014C0E6BEC01F00801D36FD329F7
:10DE50000001D8A434EF6FF00801D36BAA6A4C0E0E
:10DE6000A96ED35174EC01F00001470E6BEC01F088
:10DE70000801D56FD5290001D8A448EF6FF0010E35
:10DE80000801D56FAA6A470EA96ED55174EC01F04E
:10DE90000001480E6BEC01F00801D66FD529000196
:10DEA000D8A45BEF6FF00801D66BAA6A480EA96E82
:10DEB000D65174EC01F00001010E0801D65D00019D
:10DEC000D8A468EF6FF0BD6BD5C8BCF06FEF6FF0F2
:10DED0000801D5513C0DF3CFBCF0F4CFBDF00001EB
:10DEE000490E6BEC01F00801D76FD7290001D8A4C7
:10DEF00083EF6FF0030E0801D76FAA6A490EA96E6F
:10DF0000D75174EC01F000014A0E6BEC01F00801EE
:10DF1000D86FD8290001D8A497EF6FF0010E08013F
:10DF2000D86FAA6A4A0EA96ED85174EC01F00001AC
:10DF30004B0E6BEC01F00801D96FD9290001D8A470
:10DF4000AAEF6FF00801D96BAA6A4B0EA96ED951DE
:10DF500074EC01F000014D0E6BEC01F0BF6FBF29B6
:10DF6000D8A4BAEF6FF0BF6BAA6A4D0EA96EBF516D
:10DF700074EC01F04E0E6BEC01F0C06FC029D8A418
:10DF8000C9EF6FF0C06BAA6A4E0EA96EC05174EC57
:10DF900001F00B0E0A01E66F0A0E0001816F56ECCC
:04DFA00015F0F7D7AA
:020000040030CA
:03000100020000FA
:020005008381F5
:06000800FFC0FFE0FF4015
:00000001FF
